:100000000C94D30F0C9404100C9404100C94041052
:100010000C9404100C9404100C9404100C94041010
:100020000C9404100C9404100C9404100C94041000
:100030000C9404100C943AB10C9404100C94041019
:100040000C9404100C94BA8F0C9404100C940410AB
:100050000C9404100C9404100C94E7260C9400AD3E
:100060000C9404100C94C58C0C9404100C94041083
:100070000C9404100C9404100C9404100C940410B0
:100080000C9404100C9404100C9404100C940410A0
:100090000C9404100C9404100C9404100C9432AAC8
:1000A0000C9404100C9404100C9404100C94041080
:1000B0000C9404100C9404100C9404100C94041070
:1000C0000C9404100C9404100C9404100C94041060
:1000D0000C9404100C9404100C9404100C94041050
:1000E0000C940410342742275E276C278627942718
:1000F000AE27B227B427B827C02784AB89AB8EAB15
:1001000098AB11ACA2ABAAABB2ABBCABC6ABD0AB9D
:10011000DFABE9AB11ACF3ABFDAB07AC2FAC32AC52
:1001200025AC29AC69AC36AC3AAC40AC44AC48AC7C
:100130004EAC52AC56AC69AC5CAC60AC64AC084A3A
:10014000D73B3BCE016E84BCBFFDC12F3D6C7431EB
:100150009ABD56833DDA3D00C77F11BED9E4BB4C42
:100160003E916BAAAABE000000803F05A84CCDB20C
:10017000D44EB93836A9020C50B9918688083CA6ED
:10018000AAAA2ABE000000803F007C3C3E5E2B3DB8
:100190003F2F5B5D3B2C2A225C004572723A204D5A
:1001A000415854454D50204245440054656D70659A
:1001B000726174757265206865617465642062653A
:1001C00064207377697463686564206F66662E20A7
:1001D0004D415854454D502074726967676572658A
:1001E00064202121004572723A204D494E54454DFC
:1001F00050003A204578747275646572207377698F
:100200007463686564206F66662E204D494E5445C0
:100210004D502074726967676572656420210045DE
:1002200072723A204D415854454D50003A2045785D
:10023000747275646572207377697463686564208D
:100240006F66662E204D415854454D50207472699A
:10025000676765726564202100202D20496E7661F4
:100260006C6964206578747275646572206E756D52
:10027000626572202100504944204175746F747585
:100280006E652066696E69736865642120507574B7
:1002900020746865206C617374204B702C204B694E
:1002A00020616E64204B6420636F6E7374616E74A2
:1002B000732066726F6D2061626F766520696E745F
:1002C0006F20436F6E66696775726174696F6E2E19
:1002D0006800504944204175746F74756E652066DE
:1002E00061696C6564212074696D656F75740020A7
:1002F000403A006F6B20543A006F6B20423A005036
:100300004944204175746F74756E65206661696C2F
:100310006564212054656D70657261747572652025
:10032000746F6F206869676800204B643A20002072
:100330004B693A2000204B703A200020436C6173D7
:100340007369632050494420002054753A200020EE
:100350004B753A2000206D61783A2000206D696E5F
:100360003A200020643A200020626961733A20003C
:100370001000C90210012C01400122017001180176
:10038000B0010E01F00104015002FA00B002F000C9
:100390003003E600D003DC009004D2007005C800F2
:1003A000A006BE000008B400B009AA00D00BA0004F
:1003B000600E960060118C000015820020197800F4
:1003C000C01D6E00A0226400B0275A00902C50007F
:1003D00000314600E0343C0010383200903A2800EA
:1003E000603C1E00A03D1400803E0A00203F00003B
:1003F00070012C0190012701B0012201C0011D01F3
:10040000F00118011002130130020E01600209010F
:1004100090020401C002FF000003FA004003F5004F
:100420008003F000D003EB002004E6007004E1003C
:10043000E004DC004005D700C005D2004006CD0036
:10044000D006C8008007C3003008BE00F008B9001D
:10045000C009B400B00AAF00B00BAA00D00CA500D0
:10046000000EA000500F9B00C0109600501291008B
:1004700000148C00C0158700B0178200B0197D00F1
:10048000D01B7800001E730040206E00902269008F
:10049000F024640040275F0090295A00E02B5500AB
:1004A000102E500020304B0010324600E033410047
:1004B00090353C001037370070383200A0392D00DD
:1004C000B03A2800A03B2300603C1E00103D1900FC
:1004D000903D1400103E0F00703E0A00C03E050023
:1004E000003F00004D383420582059205A20450044
:1004F00043616E6E6F7420656E74657220737562F1
:100500006469723A20004D3234004D323320257335
:10051000006175746F25692E67006572726F7220B5
:1005200077726974696E6720746F2066696C650004
:100530004E6F74207072696E74696E67000A002FC6
:10054000005344207072696E74696E67206279741A
:100550006520000A002E0044656C6574696F6E208A
:100560006661696C65642C2046696C653A200046BA
:10057000696C652064656C657465643A002E006F73
:1005800070656E206661696C65642C2046696C65D7
:100590003A200057726974696E6720746F2066692B
:1005A0006C653A20002E006F70656E206661696C84
:1005B00065642C2046696C653A20002E006F7065DA
:1005C0006E206661696C65642C2046696C653A2012
:1005D0000046696C652073656C6563746564002012
:1005E00053697A653A200046696C65206F70656EC4
:1005F00065643A20002E006F70656E206661696C3C
:1006000065642C2046696C653A20004E6F77206641
:10061000726573682066696C653A20004E6F7720BA
:10062000646F696E672066696C653A2000222070ED
:100630006F73002220706172656E743A2200535508
:1006400042524F5554494E452043414C4C20746111
:10065000726765743A2200747279696E6720746FEC
:100660002063616C6C207375622D67636F64652015
:1006700066696C6573207769746820746F6F206D8C
:10068000616E79206C6576656C732E204D41582023
:100690006C6576656C2069733A005344206361721F
:1006A00064206F6B006F70656E526F6F74206661AF
:1006B000696C656400766F6C756D652E696E697422
:1006C000206661696C656400534420696E6974201A
:1006D0006661696C0000002110422063308440A5EF
:1006E00050C660E770088129914AA16BB18CC1ADF9
:1006F000D1CEE1EFF13112100273325222B5529491
:1007000042F772D662399318837BB35AA3BDD39C48
:10071000C3FFF3DEE36224433420040114E664C71C
:1007200074A44485546AA54BB528850995EEE5CF98
:10073000F5ACC58DD55336722611163006D776F630
:10074000669556B4465BB77AA719973887DFF7FEE8
:10075000E79DD7BCC7C448E5588668A778400861BC
:100760001802282338CCC9EDD98EE9AFF948896938
:10077000990AA92BB9F55AD44AB77A966A711A50D0
:100780000A333A122AFDDBDCCBBFFB9EEB799B5888
:100790008B3BBB1AABA66C877CE44CC55C222C035C
:1007A0003C600C411CAEED8FFDECCDCDDD2AAD0BD8
:1007B000BD688D499D977EB66ED55EF44E133E3270
:1007C0002E511E700E9FFFBEEFDDDFFCCF1BBF3A28
:1007D000AF599F788F8891A981CAB1EBA10CD12D17
:1007E000C14EF16FE18010A100C230E3200450251A
:1007F0004046706760B9839893FBA3DAB33DC31C8E
:10080000D37FE35EF3B1029012F322D23235421469
:100810005277625672EAB5CBA5A89589856EF54FD9
:10082000E52CD50DC5E234C324A0148104667447B9
:100830006424540544DBA7FAB79987B8975FE77E2D
:10084000F71DC73CD7D326F2369106B01657667609
:1008500076154634564CD96DC90EF92FE9C899E979
:10086000898AB9ABA94458654806782768C018E159
:10087000088238A3287DCB5CDB3FEB1EFBF98BD8CD
:100880009BBBAB9ABB754A545A376A167AF10AD0A9
:100890001AB32A923A2EFD0FED6CDD4DCDAABD8B19
:1008A000ADE89DC98D267C076C645C454CA23C83F9
:1008B0002CE01CC10C1FEF3EFF5DCF7CDF9BAFBA6D
:1008C000BFD98FF89F176E367E554E745E932EB249
:1008D0003ED10EF01E53544F505045442E20005030
:1008E00072696E7465722073746F707065642064D1
:1008F000756520746F206572726F72732E20466961
:100900007820746865206572726F7220616E642051
:10091000757365204D39393920746F207265737491
:100920006172742E202854656D70657261747572E1
:10093000652069732072657365742E205365742079
:100940006974206166746572207265737461727473
:10095000696E6729004B494C4C45442E200050726B
:10096000696E7465722068616C7465642E206B69B1
:100970006C6C28292063616C6C656421006F6B00CE
:10098000526573656E643A20002200556E6B6E6F7F
:10099000776E20636F6D6D616E643A2022004D3278
:1009A000323020532569005A204F666673657420E3
:1009B0003A20007A5F6D61783A20007A5F6D696E47
:1009C0003A20005A204F6666736574005A204F66BD
:1009D00066736574206F6B002200556E6B6E6F77C7
:1009E0006E20636F6D6D616E643A2022007A5F6DD8
:1009F00061783A20007A5F6D696E3A2000795F6D08
:100A000061783A2000795F6D696E3A2000785F6DF9
:100A100061783A2000785F6D696E3A2000205A3A7A
:100A20000020593A0020436F756E7420583A200018
:100A300020453A00205A3A0020593A00583A0046D8
:100A400049524D574152455F4E414D453A4D6172B5
:100A50006C696E2056312E302E323B2053707269F5
:100A60006E7465722F6772626C206D617368757049
:100A700020666F722067656E36204649524D574199
:100A800052455F55524C3A68747470733A2F2F6711
:100A900069746875622E636F6D2F4D61726C696E3B
:100AA0004669726D776172652F4D61726C696E2057
:100AB00050524F544F434F4C5F56455253494F4E3F
:100AC0003A312E30204D414348494E455F545950EC
:100AD000453A507275736120693320455854525518
:100AE0004445525F434F554E543A31205555494481
:100AF0003A30303030303030302D303030302D30F2
:100B00003030302D303030302D30303030303030EB
:100B100030303030300A00507275736120693320F4
:100B20004F66662E005072757361206933207072B3
:100B30006970726176656E6100426564204F4B2E6C
:100B40000020423A0020453A00543A005A61687247
:100B50006976616E69206265642E2E2E005A616886
:100B6000726976616E69204F4B2E0020573A002043
:100B7000453A00543A005A6168726976616E692E8E
:100B80002E2E002042403A0020403A00202F003A0A
:100B900000205400202F0020423A00202F006F6BCD
:100BA00020543A002569206D696E2C202569207338
:100BB000656300456E642066696C65206C697374BA
:100BC00000426567696E2066696C65206C697374A4
:100BD000004E6F206D6F76652E0050727573612028
:100BE00069332070726970726176656E61004F6260
:100BF0006E6F76656E69207469736B7500576169F5
:100C00007420666F7220757365722E2E2E00536CE1
:100C10006565702E2E2E00256920686F7572732011
:100C20002569206D696E7574657300446F6E65206B
:100C30007072696E74696E672066696C65005354E2
:100C40004F505045442E20005072696E74657220DA
:100C500073746F707065642064756520746F2065AF
:100C600072726F72732E20466978207468652065F1
:100C700072726F7220616E6420757365204D393910
:100C80003920746F20726573746172742E20285439
:100C9000656D706572617475726520697320726527
:100CA0007365742E205365742069742061667465C1
:100CB000722072657374617274696E6729004E6F79
:100CC000204C696E65204E756D626572207769747F
:100CD0006820636865636B73756D2C204C61737459
:100CE000204C696E653A20004E6F20436865636B47
:100CF00073756D2077697468206C696E65206E75F8
:100D00006D6265722C204C617374204C696E653A7B
:100D10002000636865636B73756D206D69736D6129
:100D20007463682C204C617374204C696E653A20A2
:100D3000004C696E65204E756D6265722069732086
:100D40006E6F74204C617374204C696E65204E7513
:100D50006D6265722B312C204C617374204C696E6E
:100D6000653A20004D31313000446F6E652073616B
:100D700076696E672066696C652E006F6B004D3278
:100D800039002020506C616E6E6572427566666532
:100D90007242797465733A20002046726565204D71
:100DA000656D6F72793A20004665622020332032EB
:100DB00030313600436F6D70696C65643A200028ED
:100DC0006E6F6E652C2064656661756C7420636F50
:100DD0006E6669672900207C20417574686F723ADD
:100DE00020004665622020332032303136203039F1
:100DF0003A35353A353100204C61737420557064B2
:100E0000617465643A2000312E302E32004D6172DB
:100E10006C696E0020536F6674776172652052654D
:100E200073657400205761746368646F672052654E
:100E3000736574002042726F776E206F7574205254
:100E400065736574002045787465726E616C20521C
:100E50006573657400506F776572557000737461C7
:100E60007274002200656E717565696E67202200DC
:100E70002200656E717565696E67202200FFFFFFB5
:100E80000000A0400000A0400000004000005643C9
:100E9000000046431FC5484300000000000000005A
:100EA0001F856B3E00005643000046430000494347
:100EB00000000000000000001F856B3E6563686F46
:100EC0003A004572726F723A004B6172746120761B
:100ED000796A6D757461004B6172746120766C6F14
:100EE0007A656E610047312045343020463130301C
:100EF000004731204537302046343030004D3833FC
:100F000000473120452D38302046343030004D38F0
:100F100033002D2D3A2D2D002D2D2D005344000191
:100F20002000012000446F737461766F76616E69F2
:100F3000205A004D6F64202020202020205B7469FF
:100F40006368795D004D6F6420205B7679732E2095
:100F500076796B6F6E5D00446F6C6164656E6920BD
:100F60006F7379205A004D3630300056796D656EBA
:100F700069742066696C616D656E74005072757479
:100F80006F6B00507275746F6B00527963686C6F91
:100F900073742076656E742E00527963686C6F737B
:100FA000742076656E742E004265640042656400AC
:100FB000547279736B6100547279736B610052796A
:100FC00063686C6F737400527963686C6F7374003C
:100FD000486C61766E69206E616269646B61005A6B
:100FE00063686C6164697400464C4558202D20206C
:100FF0003233302F35300050502020202D20203229
:1010000035342F3130300048495053202D202032C4
:1010100032302F3130300050455420202D202032E6
:1010200034302F393000504C4120202D20203231D7
:10103000302F35300041425320202D2020323535CD
:101040002F31303000486C61766E69206E616269C4
:10105000646B61004D3834004D38342058205920DD
:101060005A2045004D3234004D323320257300059F
:101070002E2E00486C61766E69206E616269646B29
:101080006100527963686C6F73742076656E742E9C
:1010900000527963686C6F73742076656E742E00ED
:1010A0004265640042656400547279736B61005458
:1010B0007279736B61004E6173746176656E69005D
:1010C000580059005A00457874727564657200457D
:1010D0007874727564657200506F73756E6F757495
:1010E000205A00506F73756E6F7574205900506FE1
:1010F00073756E6F75742058004E617374617665F8
:101100006E69004D6F64202020202020205B7469D0
:101110006368795D004D6F6420205B7679732E20C3
:1011200076796B6F6E5D00473238004175746F20C1
:10113000686F6D65004D3834005679706E6F757448
:10114000206D6F746F727900473238205A004B61FE
:101150006C6962726F766174205A00506F73756E9D
:101160006F7574206F7375005465706C6F746100D7
:10117000486C61766E69206E616269646B610052D1
:1011800065763A203137352D316200686F77746F9C
:101190002E707275736133642E636F6D00666F72AB
:1011A000756D2E707275736133642E636F6D007090
:1011B0007275736133642E636F6D004669726D776B
:1011C000617265202D20322E322E336200486C6110
:1011D000766E69206E616269646B6100506F647045
:1011E0006F7261004E6173746176656E6900567945
:1011F0006A6D6F75742066696C616D656E74005AF6
:1012000061766573742066696C616D656E74005AF1
:1012100061646E61205344206B6172746100546993
:10122000736B207A205344005A6173746176697439
:10123000207469736B00506F6B7261636F766174B9
:1012400000506F7A61737461766974207469736B8E
:1012500000507265646568726576004C61646974FB
:1012600000496E666F726D61636500486172646308
:101270006F6465642044656661756C7420536574A1
:1012800074696E6773204C6F616465640046696CB5
:10129000616D656E742073657474696E67733A204E
:1012A00044697361626C6564002020204D323030E7
:1012B00020440046696C616D656E742073657474BA
:1012C000696E67733A002020204D32303920530078
:1012D0004175746F2D526574726163743A20533D89
:1012E0003020746F2064697361626C652C2031203A
:1012F000746F20696E74657270726574206578749D
:10130000727564652D6F6E6C79206D6F76657320D4
:101310006173207265747261637473206F722072DE
:1013200065636F7665726965730020460020202032
:101330004D3230382053005265636F7665723A2023
:10134000533D4578747261206C656E67746820281F
:101350006D6D2920463A537065656420286D6D2FA8
:101360006D2900205A002046002020204D323037C1
:10137000205300526574726163743A20533D4C658A
:101380006E67746820286D6D2920463A5370656534
:101390006420286D6D2F6D29205A3A205A4C6966B9
:1013A0007420286D6D290020440020490020202051
:1013B0004D333031205000504944207365747469B6
:1013C0006E67733A00205A0020590020204D3230B9
:1013D00036205800486F6D65206F6666736574200F
:1013E000286D6D293A00204500205A002058002021
:1013F000420020540020204D3230352053004164FB
:1014000076616E636564207661726961626C657392
:101410003A20533D4D696E2066656564726174655E
:1014200020286D6D2F73292C20543D4D696E20743A
:10143000726176656C2066656564726174652028EA
:101440006D6D2F73292C20423D6D696E696D756D30
:10145000207365676D656E742074696D6520286DF5
:1014600073292C20583D6D6178696D756D20585930
:10147000206A65726B20286D6D2F73292C20205AED
:101480003D6D6178696D756D205A206A65726B20BB
:10149000286D6D2F73292C2020453D6D6178696D75
:1014A000756D2045206A65726B20286D6D2F73293C
:1014B0000020540020204D3230342053004163631B
:1014C000656C65726174696F6E3A20533D61636348
:1014D000656C65726174696F6E2C20543D72657421
:1014E0007261637420616363656C65726174696FB6
:1014F0006E00204500205A0020590020204D323037
:10150000312058004D6178696D756D2041636365C8
:101510006C65726174696F6E20286D6D2F7332294E
:101520003A00204500205A0020590020204D32303A
:10153000332058004D6178696D756D20666565646E
:10154000726174657320286D6D2F73293A002045F0
:1015500000205A0020590020204D393220580053D5
:10156000746570732070657220756E69743A0045F9
:10157000303A20005A3A2000593A2000583A2000C8
:101580004D53312C4D53322050696E730A00656EF5
:101590006473746F7073206869743A205A00205A1B
:1015A0003A00656E6473746F7073206869743A20D2
:1015B000590020593A00656E6473746F7073206827
:1015C00069743A20580020583A00656E6473746F4D
:1015D0007073206869743A200024F4D43050C38EAC
:1015E00020C2A24017828B7011127A910D816CD9A2
:1015F0000AA861E108C7586607615143061E4B5DA2
:1016000005C145A7041A411104093D9803713931F8
:10161000034036DB0265339102D4305402802E1D24
:1016200002632CEE01752AC501B028A001102781A4
:10163000018F2564012B244B01E0223401AC211FD2
:10164000018D200D01801FFC00841EED00971DDF21
:1016500000B81CD200E61BC600201BBC00641AB2F6
:1016600000B219A8000A19A0006A189900D11791B0
:101670000040178B00B516840031167E00B3157933
:10168000003A157300C7146F0058146A00EE136611
:10169000008813630025135E00C7125B006C1257AD
:1016A0000015125400C111510070114F0021114B4F
:1016B00000D61049008D1047004610440002104229
:1016C00000C00F4000800F3E00420F3C00060F3B61
:1016D00000CB0E3800930E37005C0E3500270E3419
:1016E00000F30D3200C10D3100900D3000600D2E61
:1016F00000320D2D00050D2C00D90C2B00AE0C294D
:1017000000850C29005C0C2700350C27000E0C26E8
:1017100000E80B2400C40B2400A00B23007D0B2346
:10172000005A0B2100390B2100180B2000F80A1F6A
:1017300000D90A1E00BB0A1E009D0A1D00800A1D5A
:1017400000630A1C00470A1B002C0A1B00110A1A1E
:1017500000F7091A00DD091900C4091900AB0919BD
:1017600000920917007B091800630917004C09163D
:101770000036091600200916000A091500F508159B
:1017800000E0081400CC081400B8081400A40814E1
:1017900000900813007D0812006B0813005808120F
:1017A0000046081200340811002308110012081125
:1017B0000001081100F0071000E0071000D007102A
:1017C00000C0071000B0070F00A107100091070E1E
:1017D0000083070F0074070F0065070E0057070E00
:1017E0000049070E003B070D002E070E0020070DD5
:1017F0000013070D0006070D00F9060C00ED060D9D
:1018000000E0060C00D4060C00C8060C00BC060C58
:1018100000B0060C00A4060B0099060C008D060B08
:101820000082060B0077060B006C060B0061060AAF
:101830000057060B004C060A0042060A0038060A4A
:10184000002E060A0024060A001A060A00100609DD
:101850000007060A00FD050900F4050900EB05096B
:1018600000E2050900D9050900D0050900C70509EE
:1018700000BE050900B5050800AD050800A505096D
:10188000009C050800940508008C050800840508E4
:10189000007C050800740508006C05070065050854
:1018A000005D050700560508004E050700470507BF
:1018B000004005080038050700310507002A050724
:1018C00000230507001C050600160507000F050785
:1018D000000805060002050700FB040600F50407E2
:1018E00000EE040600E8040600E2040700DB04063C
:1018F00000D5040600CF040600C9040600C3040690
:1019000000BD040600B7040600B1040500AC0406DF
:1019100000A6040600A00405009B0406009504052B
:1019200000900406008A0405008504050080040672
:10193000007A04050075040500700405006B0405B9
:101940000066040500610405005C040500570405F9
:1019500000520405004D0405004804050043040539
:10196000003E0404003A0405003504050030040478
:10197000002C04050027040400230405001E0404B1
:10198000001A04040016040500110404000D0404E8
:1019900000090405000404040000040400FC03041E
:1019A00000F8030400F4030400F0030400EC030453
:1019B00000E8030400E4030400E0030400DC030483
:1019C00000D8030400D4030400D0030400CC0304B3
:1019D00000C8030300C503030024F404D9201BC47A
:1019E0000C5C0E9804C4095F0265077101F405F9E7
:1019F00000FB04B30048048700C103690058035585
:101A00000003034500BE023A008402310053022A5B
:101A1000002902250004022000E4011C00C801196D
:101A200000AF011700980114008401130071011028
:101A3000006101100051010E0043010D0036010B41
:101A4000002B010B0020010B00150109000C0109FE
:101A50000003010800FB000800F3000800EB00078A
:101A600000E4000600DE000600D8000600D20006F2
:101A700000CC000500C7000500C2000500BD000441
:101A800000B9000400B5000400B1000400AD00047A
:101A900000A9000400A5000300A20003009F0004A9
:101AA000009B0003009800030095000200930003D0
:101AB00000900003008D0002008B000300880002EC
:101AC000008600020084000300810002007F000203
:101AD000007D0002007B0002007900020077000117
:101AE0000076000200740002007200010071000222
:101AF000006F0002006D0001006C0002006A00012E
:101B00000069000200670001006600010065000135
:101B10000064000200620001006100010060000139
:101B2000005F0002005D0001005C0001005B00013D
:101B3000005A00010059000100580001005700013F
:101B40000056000100550001005400010053000040
:101B5000005300010052000100510001005000013B
:101B6000004F0001004E0000004E0001004D00013A
:101B7000004C0001004B0000004B0001004A000136
:101B80000049000100480000004800010047000132
:101B9000004600000046000100450000004500012D
:101BA0000044000100430000004300010042000027
:101BB000004200010041000000410001004000011E
:101BC000003F0000003F0001003E0000003E000119
:101BD000003D0000003D0001003C0000003C000012
:101BE000003C0001003B0000003B0001003A000007
:101BF000003A0001003900000039000100380000FF
:101C000000380000003800010037000000370001F4
:101C100000360000003600000036000100350000EC
:101C200000350000003500010034000000340000E1
:101C300000340001003300000033000000330001D5
:101C400000320000003200000032000100310000CC
:101C500000310000003100010030000000300000C1
:101C600000300001002F0000002F0000002F0000B6
:101C7000002F0001002E0000002E0000002E0001A9
:101C8000002D0000002D0000002D0000002D00019F
:101C9000002C0000002C0000002C0000002C000193
:101CA000002B0000002B0000002B0000002B000187
:101CB000002A0000002A0000002A0000002A00017B
:101CC0000029000000290000002900000029000070
:101CD0000029000100280000002800000028000062
:101CE0000028000000280001002700000027000055
:101CF0000027000000270000002700010026000048
:101D0000002600000026000000260000002600013A
:101D1000002500000025000000250000002500002F
:101D20000025000000250001002400000024000020
:101D30000024000000240000002400010023000013
:101D40000023000000230000002300000023000007
:101D500000230000002300010022000000220000F8
:101D600000220000002200000022000000220001EA
:101D700000210000002100000021000000210000DF
:101D800000210000002100000021000100200000CF
:101D900000200000002000000020000000200000C3
:101DA000002000000020000000200001001F0000B3
:101DB000001F0000001F0000001F0000001F0000A7
:101DC000001F0000001F0001001E0000001E000098
:101DD000001E0000001E00000020746F6F206C6F5A
:101DE0006E6720657874727573696F6E20707265A6
:101DF00076656E7465640020636F6C64206578742A
:101E0000727573696F6E2070726576656E74656445
:101E1000000000090A02080B0C0D0706030401006C
:101E200000000000000000000000000000000000B2
:101E30000000000000000000000000000011100F72
:101E40000000000000000000000000000000000092
:101E50000000000000000000000000000000000082
:101E600000000000000000010210202008081020DF
:101E70004010204080020102010804020101020416
:101E800008102040808040201008040201800402D5
:101E9000018040201008040201080402010102042C
:101EA000081020408001020408102040801008041F
:101EB0000880102040044080102040048005050563
:101EC00005070508080808020202020A0A080804B1
:101ED00004040401010101010101010303030303DF
:101EE000030303040707070C0C0C0C0C0C0C0C026E
:101EF00002020206060606060606060B0B0B0B0B75
:101F00000B0B0B07070A0A0A0A0A0A05050504044F
:101F1000040808000020002300260029002C002FC0
:101F20000032000001000003010601090100002247
:101F300000250028002B002E003100340002010093
:101F400000050108010B0100002100240027002AE0
:101F5000002D003000330001010000040107010AD8
:101F600001024E414E494E495459494E46CDCCCCC2
:101F70003D0AD7233C17B7D13877CC2B329595E65D
:101F8000241FB14F0A000020410000C84200401C3D
:101F90004620BCBE4CCA1B0E5AAEC59D7400EA64F6
:101FA0001A8106AAEE6411241FBECFEFD1E2DEBF74
:101FB000CDBF00E00CBF16E0A0E0B2E0E0ECFAE735
:101FC00001E00BBF02C007900D92A030B107D9F716
:101FD00024E1A0E0B6E001C01D92A93EB207E1F7FE
:101FE0001FE1C4EADFE100E006C022970109FE011B
:101FF0000BBF0E94F1B6CE39D10780E00807A9F7E0
:102000000E940AAE0C944FBD0C940000CF93DF9356
:10201000EC019C012C5F3F4F41E050E060E070E03C
:10202000898D9A8D0E94A81A882399F04D895E891E
:102030006F89788D452B462B472B59F44C815D8158
:102040006E817F814D8B5E8B6F8B788F99819068CD
:102050009983DF91CF910895CF92DF92EF92FF9213
:102060000F931F93CF93DF93EC0189899A89AB89F2
:10207000BC89803E9F4FAF41B10510F080E06BC03E
:10208000CE01C4DF8823D1F30E94BC18182F882307
:10209000A9F3E98DFA8DCC80DD80EE80FF8032E0FF
:1020A000C31AD108E108F108058404C0CC0CDD1C7A
:1020B000EE1CFF1C0A94D2F786859785A089B1890A
:1020C000C80ED91EEA1EFB1E81E080930606C09250
:1020D0000908D0920A08E0920B08F0920C0880E000
:1020E00092E0E9E0F6E0DF019C011D9221503040D2
:1020F000E1F701E0E98DFA8D8481081790F429E079
:1021000036E0B701A601400F511D611D711D809180
:102110000706909108060E94423D8823E1F00F5F78
:10212000E9CFC12C82E0D82EE12CF12C058404C02B
:10213000CC0CDD1CEE1CFF1C0A94D2F749895A898D
:102140006B897C894C0D5D1D6E1D7F1D498B5A8BE3
:102150006B8B7C8B812FDF91CF911F910F91FF9023
:10216000EF90DF90CF900895CF93DF93EC0141E0A3
:10217000611101C040E06C857D858E859F850E9440
:10218000FC18882341F0888920E2829FC001112435
:10219000875F994F02C080E090E0DF91CF91089572
:1021A00030E020E04EE2DC015C91503271F03830DA
:1021B00029F4FB01E20FF11D40832F5FFB01E20FC9
:1021C000F11DDC015C9150832F5F3F5F01963B3036
:1021D00051F7FB01E20FF11D10820895CF93DF93B9
:1021E000EB01FC012381211102C080E00EC02250CE
:1021F000223020F48FE28883198206C060E0B4DFC9
:10220000009799F3BE01CCDF81E0DF91CF91089573
:10221000FB012BE030E231932150E9F7DC0190E043
:1022200027E03A2FEB2F8D9181110AC0DA013C9300
:102230001196EC9381E0FB019081903239F525C035
:102240008F32A1F38E3219F0EAE8F1E008C02A30AB
:10225000E1F098E02AE0E5CF31963817B1F03491FB
:102260003111FACF291788F03FED380F3E3568F469
:1022700031E0390FFB01E90FF11D9FE9980F9A3109
:1022800008F480528083932FCCCF80E008950F9381
:102290001F93CF93DF93EC018B018B81882311F087
:1022A00080E042C0FB018789803139F18032C1F77B
:1022B00083E08B83F801428D538D648D758D4D8B3A
:1022C0005E8B6F8B788F9E012F5E3F4FC8010E94FF
:1022D000B319882329F31A8F098F81E089831C821F
:1022E0001D821E821F82188619861A861B861C86EE
:1022F0001D861E861F86188A17C082E08B831D8A62
:102300001E8A1F8A188EFB01408D518D60E070E09F
:1023100095E0440F551F661F771F9A95D1F7498B9B
:102320005A8B6B8B7C8BD7CFDF91CF911F910F9105
:1023300008952F923F924F925F926F927F928F9269
:102340009F92AF92BF92CF92DF92EF92FF920F9344
:102350001F93CF93DF93EC015B016A018B818111A5
:1023600003C08FEF9FEFC7C0898180FFFACF4989F3
:102370005A896B897C8988859985AA85BB852601C0
:10238000612C712C8A019B01081B190B2A0B3B0B3A
:10239000401651066206730618F06A01C81AD90A77
:1023A00076013E0124E0620E711CE114F10409F48F
:1023B00076C0488559856A857B854A0181E09822E7
:1023C0002B811A012B01E9E0569447943794279406
:1023D000EA95D1F7898D9A8DFC01223049F4628DFE
:1023E000738D848D958D620D731D841D951D3CC06C
:1023F00014811150122181149104C1F4111116C0DD
:10240000452B462B472B49F48D899E89AF89B88D82
:102410008C839D83AE83BF8309C04C815D816E81B7
:102420007F81930121D7882309F49BCFE98DFA8D11
:102430006C817D818E819F81625071098109910932
:10244000058404C0660F771F881F991F0A94D2F76E
:102450002685378540895189620F731F841F951F18
:10246000610F711D811D911D20E032E0281939098D
:1024700087012E153F0508F489010115F2E01F07B9
:1024800069F52091090830910A0840910B08509194
:102490000C08621773078407950719F41FC0C6015B
:1024A0002AC09501AB01BC018091070690910806F6
:1024B0000E94CD3C882309F454CFA00EB11E88851C
:1024C0009985AA85BB85800F911FA11DB11D8887A5
:1024D0009987AA87BB87E01AF10A67CF40E08CD6BC
:1024E000882309F43ECFB401675F794FA801C50185
:1024F0000E940EBAE2CFDF91CF911F910F91FF9012
:10250000EF90DF90CF90BF90AF909F908F907F9093
:102510006F905F904F903F902F900895CF93DF93EF
:102520001F92CDB7DEB741E050E0BE016F5F7F4F35
:1025300000DF019719F4898190E002C08FEF9FEFCF
:102540000F90DF91CF910895CF92DF92EF92FF929B
:102550000F931F93CF93DF936C01EB017A01FC0182
:102560008381823060F000851185228533850F716B
:10257000112722273327012B022B032B11F08FEF7A
:102580005CC04115510511F0F70110821DE040E2D9
:1025900050E0BE01C601CDDE8032910539F021E068
:1025A000892B09F420E0822F819547C028812223BE
:1025B000C1F0253E61F32E3251F33B853F733F302E
:1025C00061F4E114F10449F04A8D5B8D452B29F447
:1025D0002F713FEF320F343030F02B8523FDD7CFF2
:1025E0002CC080E02AC030E021503109129FC00188
:1025F000139F900D1124F701E80FF91F2981208303
:102600002B8121832D8122832F812383298524837C
:102610002E852583288926832A8927832C8920874C
:102620002E892187288D22872C8D23872E8D248724
:10263000288126FFD2CF1586D0CFDF91CF911F9171
:102640000F91FF90EF90DF90CF9008951F93CF935D
:10265000DF93EC018B81823018F480E090E023C09E
:10266000488559856A857B85A5E076956795579558
:102670004795AA95D1F7142F1F70CE014FDF97FD14
:10268000ECCF488559856A857B85415E5F4F6F4FEA
:102690007F4F488759876A877B8720E2129FC00156
:1026A0001124875F994FDF91CF911F9108954F9229
:1026B0005F926F927F92AF92BF92CF92DF92EF9232
:1026C000FF920F931F93CF93DF93EC016A017B017D
:1026D0002B81222349F089899A89AB89BC89841787
:1026E0009507A607B70710F480E06BC0223009F405
:1026F00063C0C114D104E104F10449F41C821D82B9
:102700001E821F82188619861A861B8659C08885E4
:102710009985AA85BB85E98DFA8DE585F0E0399626
:10272000AC01BD0141505109610971090E2E04C06F
:1027300076956795579547950A94D2F79701860144
:10274000015011092109310904C0369527951795C3
:102750000795EA95D2F7041715072607370720F0E3
:10276000892B8A2B8B2B49F48D899E89AF89B88D53
:102770008C839D83AE83BF8304C0041B150B260B83
:10278000370B280139015E0184E0A80EB11C411409
:1027900051046104710481F04C815D816E817F81FF
:1027A0009501898D9A8D60D591E0491A510861088B
:1027B00071088111ECCF05C0C886D986EA86FB86F0
:1027C00081E0DF91CF911F910F91FF90EF90DF900B
:1027D000CF90BF90AF907F906F905F904F90089593
:1027E0000F931F93CF93DF93EC018B818823D1F15B
:1027F000898187FF32C061E0CE01B6DC8C01009791
:1028000089F1FC018081853E69F18B81823040F441
:1028100049895A896B897C89448F558F668F778F58
:102820004D895E896F89788DF801538F428F758B42
:10283000648BE0910006F0910106309759F0B801E1
:102840006A5E7F4FC80148961995F801808D918D79
:10285000938B828B89818F778983DF91CF911F91B1
:102860000F918AC481E0888380E0DF91CF911F912E
:102870000F910895CF93DF93EC01B2DF1B82DF91BC
:10288000CF910895FC0123812111F4CF08954F9237
:102890005F926F927F92AF92BF92CF92DF92EF9250
:1028A000FF920F931F93CF93DF9300D01F92CDB76A
:1028B000DEB75C016A017B01FC0183818130E9F4B0
:1028C000818181FF1AC0F50181899289A389B48928
:1028D00084179507A607B70780F0892B8A2B8B2BC7
:1028E00009F472C0F5014084518462847384B70195
:1028F000A601C501DCDE811102C080E066C0F501E1
:10290000818D928DC114D104E104F10469F44589EB
:1029100056896789708D25D7882379F3F501158A43
:10292000168A178A108E37C0F50144815581668159
:1029300077819E012F5F3F4F97D48823F1F2498121
:102940005A816B817C81F501818D928DFC012789F3
:10295000203139F4483FFFEF5F0761057105D8F476
:1029600007C0483F2FEF520762072FE0720798F425
:10297000F8D6882309F4C1CFF501448155816681D9
:1029800077810FEF1FEF2FEF3FE0818D928D51D5B3
:10299000882309F4B2CFF501C18AD28AE38AF48A86
:1029A000818180688183C5011BDF882309F4A5CF5D
:1029B000B701A6014C145D046E047F0410F4B3014A
:1029C000A201C50174DE01C081E00F900F900F904D
:1029D0000F90DF91CF911F910F91FF90EF90DF90BB
:1029E000CF90BF90AF907F906F905F904F90089581
:1029F000FF920F931F93CF93DF93EC01F42E80E2AD
:102A0000689FF0011124E75FF94F8385817121F000
:102A1000842F827109F04EC08091090890910A08B4
:102A2000A0910B08B0910C088C879D87AE87BF875B
:102A3000688B4489558960E070E0BA0155274427C6
:102A4000028D138D20E030E0402B512B622B732B35
:102A50004D8B5E8B6F8B788F8385887151F4048DDD
:102A6000158D268D378D098B1A8B2B8B3C8B81E036
:102A70000BC08031F9F49E012F5E3F4F898D9A8DF6
:102A800072D48823B9F084E08B838F2D8F70898373
:102A90001C821D821E821F82188619861A861B863A
:102AA000F4FE0BC040E050E0BA01CE01F0DE81112F
:102AB00004C011C01B8280E00EC0F5FE0BC0498926
:102AC0005A896B897C89CE01DF91CF911F910F913B
:102AD000FF90EDCD81E0DF91CF911F910F91FF909D
:102AE0000895AF92BF92CF92DF92EF92FF920F9331
:102AF0001F93CF93DF937C01EB016A01B22E898D86
:102B00009A8DF701928F818F40E050E0BA01CE019B
:102B1000CEDDA12C088519852A853B8589899A896E
:102B2000AB89BC89081719072A073B07A0F585E080
:102B300036952795179507958A95D1F70F70CE0191
:102B400085DD009709F481C0FC012081222311F06A
:102B5000253EB9F4A1100EC04091090850910A0811
:102B600060910B0870910C08F701448755876687C0
:102B70007787008BFC018081AA24A3948111CACF9E
:102B80000AC04BE050E0BC01C6010E9401BA892B8B
:102B900009F0C0CF58C08B2D8274823409F055C023
:102BA000AA2049F0F701008961E0C701DDDAEC01F4
:102BB000009769F44AC08B81823009F446C0CE0187
:102BC0004BDA882309F441C0C9E0D6E000E080E296
:102BD000FE0111928A95E9F78BE0F601DE01019082
:102BE0000D928A95E1F7E0910006F0910106309789
:102BF00039F0BE01625F7F4FCE014096199508C043
:102C000081E298E2998B888B80E098E09F878E879D
:102C1000888999899B8B8A8B998F888F8E859F85D0
:102C20009F8B8E8BA9D2882381F04B2D602FC701FB
:102C3000DF91CF911F910F91FF90EF90DF90CF9098
:102C4000BF90AF90D5CEB7FEF0CF80E0DF91CF91AF
:102C50001F910F91FF90EF90DF90CF90BF90AF90BA
:102C600008953F924F925F926F927F928F929F92C0
:102C7000AF92BF92CF92DF92EF92FF920F931F938A
:102C8000CF93DF93CDB7DEB7C354D1090FB6F89415
:102C9000DEBF0FBECDBF5C016B0124965FAF4EAFB0
:102CA0002497522E1C8E1F8E19821C82611571056D
:102CB00011F410E073C0FC0183818111FACF2496D6
:102CC000EEADFFAD249780818F3211F076011DC0EB
:102CD0002496EEADFFAD249780818F3231F431968A
:102CE0002496FFAFEEAF2497F3CFF6018381825095
:102CF000823060F3F601618D728DCE010196C7DAE4
:102D00008823B9F2CE0101967C018E01045E1F4F2B
:102D10003801FE0131964F01402E312E19C0882313
:102D2000A9F121E0AE01495C5F4FB701C801D9DECE
:102D3000882309F4BECFEC14FD0411F0C7019ADD1D
:102D40000615170501F1942D832D7801092F182FF1
:102D5000AE014E5B5F4FBE01695C7F4F24968EAD26
:102D60009FAD249755DA882309F4A3CF2496EEADBE
:102D7000FFAD249780818F3291F631962496FFAF74
:102D8000EEAF2497F3CF982D892DDFCF252DAE01FF
:102D9000495C5F4FB701C501A4DE182FCE01019633
:102DA00071DDCE014C966EDD812FCD5BDF4F0FB60E
:102DB000F894DEBF0FBECDBFDF91CF911F910F9171
:102DC000FF90EF90DF90CF90BF90AF909F908F904B
:102DD0007F906F905F904F903F900895CF93DF93D7
:102DE000EC0140E050E0BA0152DD882361F061E07F
:102DF000CE01BAD9009739F025EEFC0120831B8261
:102E0000DF91CF91B9C180E0DF91CF9108951F93F9
:102E1000CF93DF93CDB7DEB76B970FB6F894DEBFD5
:102E20000FBECDBFAB0119821C8222E0BC01CE01D6
:102E3000019617DF182F882321F0CE010196CEDFEF
:102E4000182FCE0101961EDD812F6B960FB6F894D8
:102E5000DEBF0FBECDBFDF91CF911F9108952F929E
:102E60003F924F925F926F927F928F929F92AF921A
:102E7000BF92CF92DF92EF92FF920F931F93CF9367
:102E8000DF9300D01F921F92CDB7DEB78C015B019C
:102E90003A01DC0113968C9113978130C1F411969D
:102EA0008C9181FF14C082FF18C0F80141895289BA
:102EB0006389748980859185A285B3858417950778
:102EC000A607B70751F0C801F2DB811106C081E007
:102ED000F80180838FEF9FEF37C1630183C0D80172
:102EE00059968D919C915A97FC01F481F1501A01E9
:102EF0002B0169E056944794379427946A95D1F74B
:102F0000F221FD834A0121E09222FF2309F476C0D9
:102F100080E092E08819990976018C159D0508F4E6
:102F20007C01D8015996ED91FC915A9714962D90F9
:102F30003D904D905C901797B2E02B1A31084108F4
:102F40005108058404C0220C331C441C551C0A94EF
:102F5000D2F786859785A089B189280E391E4A1E29
:102F60005B1EED812E0E311C411C511CE114F2E060
:102F7000FF0609F089C08091090890910A08A09184
:102F80000B08B0910C0882159305A405B50569F4EA
:102F9000109206068FEF9FEFDC0180930908909353
:102FA0000A08A0930B08B0930C089501B201A10187
:102FB00080910706909108060E94423D882309F4FB
:102FC00086CFF80180859185A285B3858E0D9F1DE2
:102FD000A11DB11D80879187A287B387AE0CBF1C4E
:102FE000CE18DF08D80118964D915D916D917C91B6
:102FF0001B97C114D10409F072CF7AC081149104D7
:1030000009F086CF14964D915D916D917C91179743
:10301000411551056105710559F455968D919D91A4
:103020000D90BC91A02D0097A105B10539F520C0E8
:103030009E012F5F3F4F18D1882309F448CF898123
:103040009A81AB81BC81F801218D328DF9012789EC
:10305000203139F4883FFFEF9F07A105B10540F407
:103060000DC0883F2FEF9207A2072FE0B20730F084
:10307000C8010E94061081114BCF29CFF80184832B
:103080009583A683B78344CF8114910411F5D801A9
:1030900018964D915D916D917C911B9751968D91F4
:1030A0009D910D90BC91A02D481759076A077B0789
:1030B00080F062D0882309F40ACF81E0809306066D
:1030C0002092090830920A0840920B0850920C088E
:1030D00007C041E0C201B1018FD0882309F4F7CEC7
:1030E000A701B501C401875F994F0E940EBA69CF4D
:1030F00051968D919D910D90BC91A02DF80121814B
:1031000084179507A607B70738F4418B528B638B5A
:10311000748B206821830CC0809100069091010679
:10312000892B31F06114710419F02068F8012183B2
:10313000D80111968C9183FD02C0C30105C0C8015E
:103140004FDB8111FACFC3CE0F900F900F900F90ED
:103150000F90DF91CF911F910F91FF90EF90DF9033
:10316000CF90BF90AF909F908F907F906F905F9027
:103170004F903F902F900895CF938091060688231B
:10318000B9F14091090850910A0860910B087091BB
:103190000C0829E036E080910706909108060E940D
:1031A000423DC82F811102C0C0E023C040910206F9
:1031B0005091030660910406709105064115510572
:1031C0006105710591F029E036E080910706909144
:1031D00008060E94423D882339F31092020610929D
:1031E000030610920406109205061092060601C00E
:1031F000C1E08C2FCF910895CF92DF92EF92FF9292
:10320000CF936B017C01C42F8091090890910A082B
:10321000A0910B08B0910C088C159D05AE05BF055B
:10322000C9F0AADF811102C080E018C029E036E0B1
:10323000B701A60180910706909108060E94CD3C37
:10324000882391F3C0920908D0920A08E0920B08F3
:10325000F0920C0881E0C11180930606CF91FF9097
:10326000EF90DF90CF9008958F929F92AF92BF9290
:10327000CF92DF92EF92FF920F931F93CF93DF9342
:10328000EC016A017B01890189859A85AB85BC8542
:103290000196A11DB11D84179507A607B70710F465
:1032A00080E054C08F89803129F49927872F762FA9
:1032B000652F0BC08032A1F7CB01BA0127E09695AC
:1032C0008795779567952A95D1F78B889C88AD88E7
:1032D000BE88680D791D8A1D9B1D809009089090FD
:1032E0000A08A0900B08B0900C08681579058A05AB
:1032F0009B0581F48F89803191F4DD24EE24FF2435
:10330000F601EE0FFF1FE75FF94F80819181A0E08A
:10331000B0E016C040E070DF8111ECCFC1CFE8947F
:10332000C7F8DD24EE24FF24F601EE0FFF1FEE0F99
:10333000FF1FE75FF94F80819181A281B381BF7048
:10334000F80180839183A283B38381E0DF91CF91E1
:103350001F910F91FF90EF90DF90CF90BF90AF90B3
:103360009F908F9008954F925F926F927F92AF924D
:10337000BF92CF92DF92EF92FF920F931F93CF9362
:10338000DF9300D01F92CDB7DEB78C0149835A83FB
:103390006B837C835901C12CD12C7601412C42E0F6
:1033A000542E612C712C49815A816B817C819E0144
:1033B0002F5F3F4FC80158DF882341F1D301C2017D
:1033C000F801058404C0880F991FAA1FBB1F0A9427
:1033D000D2F7C80ED91EEA1EFB1E49815A816B81A5
:1033E0007C818789803139F481E0483F5F4F6105F6
:1033F000710538F4D8CF81E0483F5F4F6F4F7F4071
:1034000090F2F501C082D182E282F3820F900F9098
:103410000F900F90DF91CF911F910F91FF90EF9040
:10342000DF90CF90BF90AF907F906F905F904F9064
:1034300008954F925F926F927F928F929F92AF9278
:10344000BF92CF92DF92EF92FF920F931F93CF9391
:10345000DF93EC014A015B0128013901423051053B
:103460006105710508F462C049855A856B857C85C4
:103470004F5F5F4F6F4F7F4F481559056A057B05BA
:1034800008F454C08F89803129F4FF24EB2CDA2C06
:10349000C92C0CC0803209F049C07501640177E085
:1034A000F694E794D794C7947A95D1F74B895C89C1
:1034B0006D897E89C40ED51EE61EF71E41E0C70148
:1034C000B6019ADE882391F19F89903159F49924AD
:1034D000AA24BB24F401EE0FFF1FE75FF94F5182CE
:1034E000408210C0E89487F89924AA24BB24F401F0
:1034F000EE0FFF1FEE0FFF1FE75FF94F4082518273
:10350000628273829A89923090F04D815E816F81E0
:1035100078854C0D5D1D6E1D7F1D409302065093F6
:103520000306609304067093050601C080E0DF91F6
:10353000CF911F910F91FF90EF90DF90CF90BF90B0
:10354000AF909F908F907F906F905F904F90089575
:103550002F923F924F925F926F927F928F929F92A3
:10356000AF92BF92CF92DF92EF92FF920F931F9391
:10357000CF93DF93CDB7DEB72F970FB6F894DEBFAA
:103580000FBECDBF1C014C875D876E877F873B8751
:103590002A87DC0119960D911D912D913C911C9764
:1035A0000F5F1F4F2F4F3F4F0D831E832F83388791
:1035B000EA85FB8580809180A280B380811491048C
:1035C000A104B10431F0FFEF8F1A9F0AAF0ABF0ABE
:1035D00010C0DC018D909D90AD90BC90B1E0B9879A
:1035E0000C851D852E853F8501301105210531058E
:1035F00009F0198675016401412C512C3201F10149
:1036000081859285A385B485481659066A067B068E
:1036100008F04EC00D811E812F8138850C151D05C7
:103620002E053F0550F4F2E0CF2ED12CE12CF12CE9
:10363000A2E08A2E912CA12CB12C9E012F5F3F4F2E
:10364000B701A601C10110DE882391F149815A8199
:103650006B817C81D701C6010196A11DB11D452B4F
:10366000462B472B19F04C015D010FC0AC01BD0189
:10367000481959096A097B090C851D852E853F85E6
:10368000401751076207730741F01FEF411A510AB3
:10369000610A710A6C017D01B2CF0FEF1FEF2FEFAE
:1036A0003FE0B701A601C101C4DE8D83811113C0C3
:1036B0001D823DC02601370121E0421A51086108F0
:1036C000710897018601B301A201C101B2DE88230E
:1036D00079F3730162018C149D04AE04BF0450F3AE
:1036E000AA85BB854D915D916D917C9141155105E8
:1036F00061057105A9F4EA85FB8580829182A28229
:10370000B382F985FF2399F00FEF801A900AA00A7F
:10371000B00AD1018D929D92AD92BC92139707C0D1
:1037200095018401C10185DE8111E5CFC1CF8D8175
:103730002F960FB6F894DEBF0FBECDBFDF91CF91AD
:103740001F910F91FF90EF90DF90CF90BF90AF90BF
:103750009F908F907F906F905F904F903F902F90B1
:103760000895AF92BF92CF92DF92EF92FF920F93A4
:103770001F93CF93DF9300D01F92CDB7DEB75C01CC
:103780006A017B0182E090E0A0E0B0E0F501808377
:103790009183A283B3839E012F5F3F4FB701A601A0
:1037A000C50162DD811102C080E023C000E010E0AD
:1037B0009801B701A601C5013CDE8823A9F3C980A1
:1037C000DA80EB80FC80F5018789803149F481E063
:1037D000F8EFCF16FFEFDF06E104F10450F4DBCF82
:1037E00081E098EFC9169FEFD906E9069FE0F90638
:1037F00090F20F900F900F900F90DF91CF911F914B
:103800000F91FF90EF90DF90CF90BF90AF90089511
:103810007F928F929F92AF92BF92CF92DF92EF9260
:10382000FF920F931F93CF93DF93EC01142F7093AC
:103830000806609307061F8A82E090E0A0E0B0E0EF
:1038400088839983AA83BB8310920606109202068E
:103850001092030610920406109205068FEF9FEF58
:10386000DC018093090890930A08A0930B08B09399
:103870000C08442349F1453008F0DEC040E060E028
:1038800070E0CB01B9DC882309F4D6C020E1129F97
:10389000F0011124E954F84F80818F7709F0CCC0F2
:1038A00084859585A685B78584369105A105B105E2
:1038B00008F4C2C0C084D184E284F384C114D1046A
:1038C000E104F10421F4B8C0C12CD12C760140E010
:1038D000C701B60191DC782E882309F4ADC0809130
:1038E0001406909115068115924009F0A5C03091FB
:1038F0001906332309F4A0C0809117069091180689
:10390000892B09F499C020911606222309F494C04A
:103910003A8B2C831D8630E041E050E06D85062F08
:10392000CA01062E02C0880F991F0A94E2F72817D1
:10393000390731F081E0860F8D87683078F37CC0DD
:1039400020911F06309120062115310519F040E025
:1039500050E008C020912D0630912E0640912F0690
:10396000509130062D833E834F83588780911706F0
:103970009091180646015701880E991EA11CB11C92
:103980008B8A9C8AAD8ABE8AE0911A06F0911B064A
:10399000F98FE88FA0911906B0E00E94E1B6680D9A
:1039A000791D8A1D9B1D6A8F7B8F8C8F9D8FB5E043
:1039B000EE0FFF1FBA95E1F7E150FE4FEF2FFF2703
:1039C000E695DC01CB018E0F9F1FA11DB11D8E87D7
:1039D0009F87A88BB98B80901C0690901D06811440
:1039E000910419F0A12CB12C08C080902906909068
:1039F0002A06A0902B06B0902C06A7019601281B42
:103A0000390B4A0B5B0BDA01C901880D991DAA1D00
:103A1000BB1D04C0B695A795979587950A95D2F7D3
:103A200089879A87AB87BC87853F3FE09307A105CD
:103A3000B10520F48CE08F8B712C15C0853F9F4F12
:103A4000A105B10510F480E10DC08091350690917B
:103A50003606A0913706B09138068A8F9B8FAC8FBF
:103A6000BD8F80E28F8B872DDF91CF911F910F91BA
:103A7000FF90EF90DF90CF90BF90AF909F908F908E
:103A80007F9008954F925F926F927F928F929F9254
:103A9000AF92BF92CF92DF92EF92FF920F931F935C
:103AA000CF93DF932C0124EF33E081E090E0F90124
:103AB00045915491441655060CF062C0AC0141503A
:103AC0005109DA01AA0FBB1FAA0FBB1FAE50BC4F92
:103AD000FD0165917491440F551F440F551F4051CE
:103AE0005C4FFA0165907490FC01EE0FFF1FEE0F22
:103AF000FF1FEE50FC4FA590B490FD01059114916D
:103B0000F901C591D491FA0185909490882777FDA9
:103B10008095982F0E945BB36B017C01B2016619FE
:103B20007709882777FD8095982F0E945BB32B013A
:103B30003C01B501601B710B882777FD8095982F9C
:103B40000E945BB39B01AC01C301B2010E948EB520
:103B50002B013C01BE0168197909882777FD809502
:103B6000982F0E945BB39B01AC01C301B2010E947C
:103B7000C0B29B01AC01C701B6010E94E0B111C007
:103B800001962C5F3F4F8D33910509F090CFE2EE07
:103B9000F4E065917491882777FD8095982F0E94B5
:103BA0005BB3DF91CF911F910F91FF90EF90DF906A
:103BB000CF90BF90AF909F908F907F906F905F90CD
:103BC0004F9008954F925F926F927F928F929F9243
:103BD000AF92BF92CF92DF92EF92FF920F931F931B
:103BE000CF93DF932C01662371F1E2ECFEE0849128
:103BF000882341F09091C00095FFFCCF8093C600D0
:103C00003196F5CF70E04AE050E087EC9DE00E94ED
:103C10001A8EE9E5F2E08491882341F09091C0008A
:103C200095FFFCCF8093C6003196F5CF8091C00000
:103C300085FFFCCF8AE08093C6000E947D4660E04D
:103C400070E0CB017EC024E733E081E090E0F90131
:103C500045915491441655060CF062C0AC01415098
:103C60005109DA01AA0FBB1FAA0FBB1FAE58BC4FE8
:103C7000FD0165917491440F551F440F551F405924
:103C80005C4FFA0165907490FC01EE0FFF1FEE0F80
:103C9000FF1FEE58FC4FA590B490FD0105911491C3
:103CA000F901C591D491FA0185909490882777FD08
:103CB0008095982F0E945BB36B017C01B20166195D
:103CC0007709882777FD8095982F0E945BB32B0199
:103CD0003C01B501601B710B882777FD8095982FFB
:103CE0000E945BB39B01AC01C301B2010E948EB57F
:103CF0002B013C01BE0168197909882777FD809561
:103D0000982F0E945BB39B01AC01C301B2010E94DA
:103D1000C0B29B01AC01C701B6010E94E0B111C065
:103D200001962C5F3F4F8032910509F090CFEEEE67
:103D3000F3E065917491882777FD8095982F0E9414
:103D40005BB3DF91CF911F910F91FF90EF90DF90C8
:103D5000CF90BF90AF909F908F907F906F905F902B
:103D60004F90089560E080916208909163082ADF87
:103D700060935E0870935F08809360089093610879
:103D800080915C0890915D087DDE60935808709387
:103D9000590880935A0890935B088FB7F894109253
:103DA00050088FBF08952091140230911502409160
:103DB00016025091170260E070E08FE793E40E94D2
:103DC000C0B26093300870933108809332089093AA
:103DD0003308089597FF03C08091570804C0FC0181
:103DE000E65DF74F808190E00895CF93DF93D82F61
:103DF000C62FC19561E00E946AAC6C2F8D2F0E9486
:103E0000A3AC6C2F70E08D2FDF91CF910C9460AB41
:103E1000CF93C1E020E030E048E452E460915E08D6
:103E200070915F0880916008909161080E94BCB415
:103E300018160CF0C0E06C2F88E090E0CF91D5CF41
:103E40002F923F924F925F926F927F928F929F92AA
:103E5000AF92BF92CF92DF92EF92FF920F931F9398
:103E6000CF93DF93CDB7DEB728970FB6F894DEBFB8
:103E70000FBECDBF80915008882309F4F8C172DFCE
:103E800080905E0890905F08A0906008B0906108F4
:103E90000091660810916708B801882777FD809522
:103EA000982F0E945BB3A50194010E94DFB16B01C2
:103EB0007C01609338087093390880933A08909396
:103EC0003B0820E030E040E251E40E94BCB4181608
:103ED00024F481E080932F08F7C020E030E040E236
:103EE00051ECC701B6010E94B9B287FD02C0012B97
:103EF00021F481E080932F080CC180912F08882342
:103F000051F010924C0810924D0810924E081092E9
:103F10004F0810922F0820911802309119024091F9
:103F20001A0250911B02C701B6010E948EB5698327
:103F30007A838B839C8360934408709345088093B5
:103F400046089093470820914C0830914D084091C5
:103F50004E0850914F08C701B6010E94E0B12B01F5
:103F60003C012090340830903508109136080091BB
:103F700037089101412F502F0E94B9B287FD14C01C
:103F800020903008309031081091320800913308A9
:103F90009101412F502FB201C3010E94BCB41816E9
:103FA0001CF01201162D072DC101A12FB02F8093F7
:103FB0004C0890934D08A0934E08B0934F08209161
:103FC0001402309115024091160250911702B1016E
:103FD000812F902F0E948EB56D837E838F8398876B
:103FE000609340087093410880934208909343087F
:103FF000209148083091490840914A0850914B0857
:10400000C501B4010E94DFB120911002309111026C
:1040100040911202509113020E948EB520ED3CECAB
:104020004CE45DE30E948EB52B013C0123E333E3B6
:1040300043E75FE360913C0870913D0880913E0842
:1040400090913F080E948EB59B01AC01C301B20163
:104050000E94E0B12B013C0160933C0870933D0845
:1040600080933E0890933F082D813E814F81588573
:1040700069817A818B819C810E94E0B1A3019201C8
:104080000E94DFB12B013C0120E030E04FE753E418
:104090000E94BCB420E030E0A9011816E4F4C70186
:1040A000B6010E94BCB418167CF4A7019601B101B8
:1040B000812F902F0E94DFB160934C0870934D08C0
:1040C00080934E0890934F08412C512C9FE7692E06
:1040D00093E4792E21C0C301B2010E94B9B287FFD7
:1040E0001BC020E030E0A901C701B6010E94B9B2AF
:1040F00087FF0FC0A7019601B101812F902F0E9469
:10410000DFB160934C0870934D0880934E089093F4
:104110004F08412C512C3201809248089092490856
:10412000A0924A08B0924B0860912208709123082F
:10413000882777FD8095982F0E945BB39B01AC0187
:10414000C501B4010E94BCB41816DCF460910802E9
:1041500070910902882777FD8095982F0E945BB3A4
:104160009B01AC01C501B4010E94B9B287FF09C02F
:10417000C301B2010E9428B37595679560932A0820
:1041800002C010922A080E944AAD009126081091A0
:1041900027082091280830912908601B710B820B99
:1041A000930B653C79408105910558F031DE0E9402
:1041B0004AAD60932608709327088093280890934F
:1041C00029080E944AAD00912B0810912C082091DB
:1041D0002D0830912E08601B710B820B930B6838F1
:1041E00073418105910508F442C00E944AAD609375
:1041F0002B0870932C0880932D0890932E08C09064
:104200005808D0905908E0905A08F0905B0820E0D8
:1042100030E040E751E4C701B6010E94BCB4181673
:104220001CF520E030E046E153E4C701B6010E94EE
:10423000B9B287FF19C0609164087091650888273A
:1042400077FD8095982F0E945BB39B01AC01C7015D
:10425000B6010E94BCB487FD03C01092570807C086
:104260008FE78093570803C010925708A5982896A7
:104270000FB6F894DEBF0FBECDBFDF91CF911F9177
:104280000F91FF90EF90DF90CF90BF90AF909F90F5
:104290008F907F906F905F904F903F902F900895F8
:1042A000CF93DF931092340810923508109236089D
:1042B0001092370820911402309115024091160295
:1042C0005091170260E070E08FE793E40E94C0B263
:1042D00060933008709331088093320890933308CC
:1042E0006D9A809101018061809301019D9A809176
:1042F000010188608093010187ED80937A0010921C
:104300007E0010927D0080917E00816080937E000F
:1043100080917E00826080937E0080917E00846028
:1043200080937E0080E888BD80916E0084608093D9
:104330006E006AEF70E080E090E00E9479AD8FE05F
:1043400090E0909323088093220860E080910A0215
:1043500090910B0237DC20E030E040E751E40E940E
:10436000B9B287FF0AC080910A0290910B02409770
:1043700090930B0280930A02E8CF86E391E090933A
:1043800009028093080260E080912408909125083A
:1043900019DC20E030E04BE953E40E94BCB418166D
:1043A00054F4809124089091250840969093250814
:1043B00080932408E8CFC0912008D0912108CE0135
:1043C00061DB20E030E046E153E40E94BCB4181603
:1043D00034F46096D0932108C0932008ECCFDF918D
:1043E000CF91089508951092670810926608109270
:1043F00065081092640810922A0875981092650852
:104400001092640810925708A59808952F923F9231
:104410004F925F926F927F928F929F92AF92BF92D4
:10442000CF92DF92EF92FF920F931F93CF93DF9380
:10443000CDB7DEB7AE970FB6F894DEBF0FBECDBFD7
:104440006B8F7C8F8D8F292E5A8749873CA72BA78E
:104450000E944AAD6F8F78A389A39AA30E944AADA8
:104460006FA378A789A79AA729853A8512161306FC
:104470001CF0E0E3F3E017C0E3E4F3E0819188236C
:1044800039F09091C00095FFFCCF8093C600F6CF25
:104490008091C00085FFFCCF1BC29091C00095FFAA
:1044A000FCCF8093C60081918111F7CF8091C0002D
:1044B00085FFFCCF8AE08093C60095DF49855A8549
:1044C0008FE7452B99F1809357088F8D98A1A9A16B
:1044D000BAA1898B9A8BAB8BBC8B8D879E87AF875C
:1044E000B88B1D8290E4988FACE1A98FB6E4BA8FA7
:1044F0001DA61D8A1E8A1F8A2FE730E040E050E08B
:1045000029833A834B835C83EFE74E2E512C612C39
:10451000712C1BA21CA21DA21EA231E03E8F1C8684
:104520001B86312C00E010E01EA605C080932A08EF
:10453000CCCF0E94DB7780915008882309F4F6C025
:1045400011DC49855A85452B51F03090580800916F
:10455000590810915A0850915B085EA709C0309025
:104560005E0800915F0810916008809161088EA735
:10457000232D302F412F5EA56DA57D898E899F89C2
:104580000E94BCB418162CF03DA60D8B1E8B9EA568
:104590009F8B232D302F412F5EA56D81788D898DC6
:1045A0009A8D0E94B9B287FD05C03D82088F198F90
:1045B000AEA5AA8F0E944AAD2FA138A549A55AA53C
:1045C000621B730B840B950B653C7940810591054B
:1045D00038F01EDC0E944AAD6FA378A789A79AA77E
:1045E0004E8D442309F44FC02B8D3C8D4D8D522DA3
:1045F000632D702F812F9EA50E94BCB418160CF05D
:1046000095C00E944AAD29893A894B895C89621B11
:10461000730B840B950B693873418105910508F480
:1046200085C0D301C20129813A814B815C81821B03
:10463000930BA40BB50B49855A85B595A79597950E
:104640008795452B19F08093570802C080932A085C
:104650000E944AAD6D877E878F87988BDC01CB01E6
:1046600029893A894B895C89821B930BA40BB50B72
:104670008BA39CA3ADA3BEA33B8D3DA74C8D4D8BBF
:104680005D8D5E8B2F8A2B8D3C8D4D8D522D632D34
:10469000702F812F9EA50E94B9B287FFEEC20E94A3
:1046A0004AAD2D853E854F855889621B730B840B5F
:1046B000950B693873418105910508F4DEC20E94AB
:1046C0004AAD698B7A8B8B8B9C8BDC01CB012D8562
:1046D0003E854F855889821B930BA40BB50B4B85E8
:1046E0005C85452B09F010C189819A81AB81BC8121
:1046F000840D951DA61DB71D29853A85B595A795ED
:1047000097958795232B09F4B5C2809357084B855D
:104710005C854F5F5F4F5C874B875B8D5D838C8DC6
:10472000888F9D8D998F2A8EA1E0AE8F20E030E09A
:1047300040EA51E46B8D7C8D8D8D922D0E94E0B10D
:104740009B01AC01632D702F812F9EA50E94BCB4EC
:10475000181694F4EFEFF2E08491882341F09091E1
:10476000C00095FFFCCF8093C6003196F5CF8091B5
:10477000C00085FFFCCFACC00E944AAD2F8D38A190
:1047800049A15AA1621B730B840B950B613D7740C5
:104790008105910508F44FC049855A85452B81F064
:1047A000E0905708F12CE9EFF2E084918823C1F002
:1047B0009091C00095FFFCCF8093C6003196F5CF55
:1047C000E0902A08F12CE3EFF2E08491882341F095
:1047D0009091C00095FFFCCF8093C6003196F5CF35
:1047E00022E030E0432D502F612F7EA587EC9DE025
:1047F0000E94F08EEFEEF2E08491882341F09091D8
:10480000C00095FFFCCF8093C6003196F5CF4AE0FB
:1048100050E0B70187EC9DE00E941A8E8091C000A5
:1048200085FFFCCF8AE08093C6000E944AAD6F8F5F
:1048300078A389A39AA30E944AAD6B017C010E94D0
:104840004AAD89889A88AB88BC882D853E854F857E
:104850005889820E931EA41EB51EC818D908EA08EE
:10486000FB08C60ED71EE81EF91E31E8C3163FE44A
:10487000D30632E1E306F10490F0E2EDF2E0849138
:10488000882341F09091C00095FFFCCF8093C60033
:104890003196F5CF8091C00085FFFCCF19C04B85C4
:1048A0005C858BA59CA5841795070CF042CEE6E7A6
:1048B000F2E08491882341F09091C00095FFFCCFF5
:1048C0008093C6003196F5CF8091C00085FFFCCF64
:1048D0008AE08093C600AE960FB6F894DEBF0FBE96
:1048E000CDBFDF91CF911F910F91FF90EF90DF909F
:1048F000CF90BF90AF909F908F907F906F905F9080
:104900004F903F902F9008958BA09CA0ADA0BEA08B
:10491000880E991EAA1EBB1E2BA13CA14DA15EA113
:10492000281B390B4A0B5B0BCA01B90129813A815B
:104930004B815C810E9454B6A50194010E94B9B6D6
:10494000240D351D461D571D2431310541055105E6
:1049500004F129013A013CEE43165104610471044B
:104960002CF06BEE462E512C612C712C40E8441635
:10497000510461047104DCF08EEF90E0A0E0B0E03F
:1049800084199509A609B70989839A83AB83BC83E7
:1049900012C054E1452E512C612C712C24E130E0E1
:1049A00040E050E029833A834B835C8304C0498212
:1049B0005A826B827C82E8E6F3E08491882341F09E
:1049C0009091C00095FFFCCF8093C6003196F5CF43
:1049D0002AE030E0B301A20187EC9DE00E94EF8D58
:1049E000E3E6F3E08491882341F09091C00095FFC5
:1049F000FCCF8093C6003196F5CF2AE030E04981A4
:104A00005A816B817C8187EC9DE00E94EF8DECE503
:104A1000F3E08491882341F09091C00095FFFCCF92
:104A20008093C6003196F5CF22E030E04D81588D5D
:104A3000698D7A8D87EC9DE00E94F08EE5E5F3E0CC
:104A40008491882341F09091C00095FFFCCF809322
:104A5000C6003196F5CF22E030E04DA55D896E8924
:104A60007F8987EC9DE00E94F08E8091C00085FFD9
:104A7000FCCF8AE08093C6002B853C85233031052E
:104A80000CF432CE69817A818B819C810E945BB368
:104A900020E030E040E850E40E948EB56B017C01DC
:104AA0002D81388D498D5A8D6DA57D898E899F897F
:104AB0000E94DFB120ED3FE049E450E40E948EB552
:104AC00020E030E040E05FE30E948EB59B01AC0146
:104AD000C701B6010E94C0B26B017C01C501B401DF
:104AE0000E945BB320E030E04AE754E40E94C0B289
:104AF0004B015C01EFE4F3E08491882341F0909155
:104B0000C00095FFFCCF8093C6003196F5CF22E020
:104B100030E0B701A60187EC9DE00E94F08EE9E449
:104B2000F3E08491882341F09091C00095FFFCCF81
:104B30008093C6003196F5CF22E030E0B501A401A4
:104B400087EC9DE00E94F08E8091C00085FFFCCF35
:104B50008AE08093C6002AE939E949E15FE3C701A9
:104B6000B6010E948EB56B017C019B01AC010E94D5
:104B7000E0B1A50194010E94C0B26D837E838F8352
:104B80009887A5019401C701B6010E948EB520E067
:104B900030E040E05EE30E948EB54B015C01EBE348
:104BA000F3E08491882341F09091C00095FFFCCF01
:104BB0008093C6003196F5CF8091C00085FFFCCF71
:104BC0008AE08093C600E5E3F3E08491882341F016
:104BD0009091C00095FFFCCF8093C6003196F5CF31
:104BE00022E030E0B701A60187EC9DE00E94F08E44
:104BF0008091C00085FFFCCF8AE08093C600EFE281
:104C0000F3E08491882341F09091C00095FFFCCFA0
:104C10008093C6003196F5CF22E030E04D815E8171
:104C20006F81788587EC9DE00E94F08E8091C000B6
:104C300085FFFCCF8AE08093C600E9E2F3E084912F
:104C4000882341F09091C00095FFFCCF8093C6006F
:104C50003196F5CF22E030E0B501A40187EC9DE06C
:104C60000E94F08E8091C00085FFFCCF8AE0809387
:104C7000C6003ACD80932A084ACD1E8E57CDCF93D9
:104C8000C82FB1DB0E94444B811134C0E2ECFEE03E
:104C90009491992341F08091C00085FFFCCF9093BF
:104CA000C6003196F5CF6C2F70E04AE050E087ECFB
:104CB0009DE00E941A8E8091C00085FFFCCF8AE0A3
:104CC0008093C600ECE2F2E08491882341F0909159
:104CD000C00095FFFCCF8093C6003196F5CF809140
:104CE000C00085FFFCCF8AE08093C6008FE192E090
:104CF0000E944C77CF910C94054BCF93C82F73DB58
:104D00000E94444B811134C0E2ECFEE0949199235F
:104D100041F08091C00085FFFCCF9093C600319692
:104D2000F5CF6C2F70E04AE050E087EC9DE00E94E8
:104D30001A8E8091C00085FFFCCF8AE08093C60068
:104D4000E2EFF1E08491882341F09091C00095FF5B
:104D5000FCCF8093C6003196F5CF8091C00085FFCF
:104D6000FCCF8AE08093C60085EE91E00E944C77EC
:104D7000CF910C94054BA5980E94444B811125C0FE
:104D8000E2ECFEE08491882341F09091C00095FF11
:104D9000FCCF8093C6003196F5CFEBEAF1E0849129
:104DA000882341F09091C00095FFFCCF8093C6000E
:104DB0003196F5CF8091C00085FFFCCF8AE08093CB
:104DC000C6008AE991E00E944C770C94054B1F9233
:104DD0000F920FB60F9211240BB60F920F931F93E1
:104DE0002F933F934F935F936F937F938F939F93F3
:104DF000AF93BF93CF93DF93EF93FF93809107021D
:104E0000811112C080912A0880931F08882311F015
:104E1000759A01C075988091570880931E08882361
:104E200011F0A59A01C0A59890911F0880910702E2
:104E3000981708F4759890911E08809107029817AA
:104E400008F4A598809107028F5F8F7780930702FF
:104E50008091060290E08B30910508F093C0FC0130
:104E6000EE58FF4F0C94D5B610927B0080E48093EF
:104E70007C0080917A00806480937A000E9455774C
:104E800081E019C0209178003091790080911A0852
:104E900090911B08A0911C08B0911D08820F931FD0
:104EA000A11DB11D80931A0890931B08A0931C08A4
:104EB000B0931D0882E08093060264C010927B00CC
:104EC00082E480937C0080917A00806480937A00F1
:104ED0000E94557783E0EFCF2091780030917900E0
:104EE0008091160890911708A0911808B0911908A0
:104EF000820F931FA11DB11D809316089093170870
:104F0000A0931808B093190884E0D5CF10927B00C5
:104F100081E480937C0080917A00806480937A00A1
:104F20000E94557785E0C7CF2091780030917900B5
:104F30008091120890911308A0911408B09115085F
:104F4000820F931FA11DB11D809312089093130827
:104F5000A0931408B093150886E0ADCF0E94557752
:104F600087E0A9CF88E0A7CF0E94557789E0A3CF3B
:104F700010920602809111088F5F8093110802C081
:104F80001092060280911108803108F463C080916C
:104F90005008811110C080911A0890911B089093BD
:104FA0006308809362088091160890911708909387
:104FB0005D0880935C0881E080935008109211088E
:104FC00010921A0810921B0810921C0810921D08CB
:104FD00010921208109213081092140810921508DB
:104FE00010920D0810920E0810920F0810921008DF
:104FF00010921608109217081092180810921908AB
:1050000020916208309163088091240890912508CE
:105010008217930714F080E032DE2091620830910D
:10502000630880910A0290910B022817390714F047
:1050300080E063DE20915C0830915D08809120085B
:1050400090912108821793072CF010926508109216
:10505000640891DE00E010E0E801CC0FDD1FCF5ABC
:10506000D74F888199811816190644F461E0802F82
:105070000E94959788819981019709C0892B49F0F1
:1050800060E0802F0E94959788819981019699838D
:1050900088830F5F1F4F03301105F1F6FF91EF91E9
:1050A000DF91CF91BF91AF919F918F917F916F9140
:1050B0005F914F913F912F911F910F910F900BBED8
:1050C0000F900FBE0F901F9018952CEA35EC47E219
:1050D0005EE30C948EB52CEA35EC47E25EE30C946B
:1050E000C0B22CEA35EC47E25EE30C94C0B22CEA85
:1050F00035EC47E25EE30C948EB5CF93DF93EC0181
:1051000060E08E810E94A3AC81E090E00E949DADA2
:1051100061E08E810E94A3AC81E090E00E949DAD91
:1051200060E08E810E94A3AC84E690E0DF91CF9195
:105130000C949DADCF92DF92EF92FF920F931F934D
:10514000CF93DF937C01C0E0D0E0C62ED12C870145
:105150000C0F1D1F61E0F80187810E946AACB60147
:105160000C2E02C0759567950A94E2F76170F801FC
:1051700087810E94A3AC2196C430D10541F7C701B5
:10518000DF91CF911F910F91FF90EF90DF90CF9023
:10519000B4CFCF92DF92EF92FF920F931F93CF93F2
:1051A000DF937C01C0E0D0E0C62ED12C87010C0F2C
:1051B0001D1F61E0F80187810E946AACB6010C2EC8
:1051C00002C0759567950A94E2F76170F8018781CE
:1051D0000E94A3AC2196C830D10541F7C701DF91E9
:1051E000CF911F910F91FF90EF90DF90CF9085CFDF
:1051F0001F93CF93DF93EC01162F642F8C810E94B5
:10520000A3AC8D818F3F19F060E00E94A3AC8F8525
:10521000612F84FF05C0CE01DF91CF911F91B9CFDF
:1052200070E084E0759567958A95E1F7CE0182DF9D
:10523000612FCE01DF91CF911F917CCF40E0D8CF7D
:1052400061E0FCDF80E496E00C949DAD62E0F6DF67
:1052500080E496E00C949DADCF93DF93CDB7DEB79D
:1052600028970FB6F894DEBF0FBECDBF28E0E3EB62
:10527000F2E0DE01119601900D922A95E1F7FC0112
:105280002389421710F04FEF420FFE013196E40FD1
:10529000F11DE40FF11D2081260F2068622F289652
:1052A0000FB6F894DEBF0FBECDBFDF91CF91C6CF52
:1052B000FC016089262F2460208B6C60BFCFCF93C8
:1052C000DF93EC01423018F08F8588608F874B8B1D
:1052D0001C8A222329F0413019F48F8584608F873E
:1052E00080E593EC0E949DAD60E08C810E94A3ACB0
:1052F00060E08E810E94A3AC8D818F3F19F060E049
:105300000E94A3AC6F8564FD19C063E0CE0112DF7B
:1053100084E991E10E949DAD63E0CE010BDF84E959
:1053200091E10E949DAD63E0CE0104DF86E990E04B
:105330000E949DAD62E0CE01FDDE13C06062CE0131
:105340007DDF84E991E10E949DAD6F856062CE01B1
:1053500075DF86E990E00E949DAD6F856062CE01A9
:105360006DDF6F856062CE0169DF8CE390E00E94A3
:105370009DAD84E0888BCE019BDF8CE390E00E94A2
:105380009DADCE015DDF88EB9BE00E949DAD82E08C
:10539000898B66E0CE0152DF8CE390E0DF91CF9104
:1053A0000C949DAD6F927F928F92AF92CF92EF92BD
:1053B0000F931F93CF93DF93CDB7DEB73C01162F2A
:1053C000842F5E854F8538899989F30184832583ED
:1053D0000683E782C086A186828653874487358705
:1053E000968761E00E946AACF30185818F3F19F0D6
:1053F00061E00E946AAC61E0F30186810E946AACC0
:10540000112319F0F301178603C080E1F3018787A8
:1054100020E041E060E1C301DF91CF911F910F9146
:10542000EF90CF90AF908F907F906F9048CF8F92FA
:10543000AF92CF92EF920F93DC0113961C921E92C3
:105440001297E1E7F3E0ED93FC931F921F921F92F6
:105450001F928C2CAE2CC02EE22E042F2FEF462F45
:1054600061E0A0DF0F900F900F900F900F91EF90E1
:10547000CF90AF908F900895CF93DF93EC0142309F
:1054800018F08F8588608F874B8B1C8A222329F028
:10549000413019F48F8584608F8780E593EC0E94FA
:1054A0009DAD60E08C810E94A3AC60E08E810E9483
:1054B000A3AC8D818F3F19F060E00E94A3AC6F8593
:1054C00064FD19C063E0CE0135DE84E991E10E94FC
:1054D0009DAD63E0CE012EDE84E991E10E949DAD99
:1054E00063E0CE0127DE86E990E00E949DAD62E098
:1054F000CE0120DE13C06062CE01A0DE84E991E11E
:105500000E949DAD6F856062CE0198DE86E990E0D5
:105510000E949DAD6F856062CE0190DE6F856062F6
:10552000CE018CDE8CE390E00E949DAD84E0888B00
:10553000CE01BEDE8CE390E00E949DADCE0186DE02
:1055400080E496E00E949DAD82E0898B66E0CE010A
:1055500075DE8CE390E00E949DAD40E068E0CE01F6
:105560007BDE6AE973E0CE010E94D7B141E068E0DA
:10557000CE0172DE6AE973E0CE010E94D7B142E04B
:1055800066E0CE0169DE68E973E0CE01DF91CF917C
:105590000C94D7B1CF92DF92EF92FF920F931F93AB
:1055A000CF93DF931F921F92CDB7DEB78C01677048
:1055B00088E0689FB00111246064C80149835A8360
:1055C0003DDE4981C42E5A81D52EE12CF12CD60125
:1055D0006D916D01D801ED91FC910190F081E02D6C
:1055E000C8011995BFEFEB1AFB0AE8E0EE16F104CB
:1055F00071F70F900F90DF91CF911F910F91FF9056
:10560000EF90DF90CF90089541E0F2DD81E090E0EF
:1056100008952F923F924F925F926F927F928F9256
:105620009F92AF92BF92CF92DF92EF92FF920F9331
:105630001F93CF93DF93CDB7DEB7CF54D1090FB609
:10564000F894DEBF0FBECDBF1C017E8F6D8F4A0167
:105650002FAB09AF2896EFAE28972C96ACAEBDAE17
:10566000CEAEDFAE2C9734E0239F50011124FC0115
:10567000EA0DFB1D80819181A281B381898F9A8F70
:10568000AB8FBC8FDA01AA0DBB1DBCAFABAF4D9089
:105690005D906D907C90A3019201698D7A8D8B8DC8
:1056A0009C8D0E94E0B121966CAF7DAF8EAF9FAF15
:1056B0002197B4E00B9F80011124F101E00FF11F4D
:1056C00020813181428153812F8F38A349A35AA36E
:1056D000A401400F511F23965FAF4EAF2397DA010D
:1056E000CD90DD90ED90FC90A70196016F8D78A193
:1056F00089A19AA10E94E0B127966CAF7DAF8EAFD1
:105700009FAF27972896EFAD2897B4E0EB9FC00195
:105710001124F101E80FF91F208131814281538169
:105720002BA33CA34DA35EA3ED8DFE8DE80FF91FC7
:1057300060817181828193810E94DFB16FA378A71C
:1057400089A79AA7AD8DBE8D1C968D919D910D90C8
:10575000BC91A02D60968CAF9DAFAEAFBFAF6097F0
:10576000D1011C962D913D914D915C911F972BA7D6
:105770003CA74DA75EA7A301920150582D8B3E8BED
:105780004F8B588FD701C601B058898B9A8BAB8B42
:10579000BC8BED8DFE8DEA0DFB1D20813181428198
:1057A00053812FA738AB49AB5AAB21962CAD3DADF9
:1057B0004EAD5FAD21976FA578A989A99AA90E94DE
:1057C000DFB16B017C01ED8DFE8DE00FF11F80815B
:1057D0009181A281B3818BAB9CABADABBEAB279665
:1057E0002CAD3DAD4EAD5FAD2797BC01CD010E9404
:1057F000DFB14B015C01A70196016D897E898F891C
:10580000988D0E948EB52B013C01A50194016989F8
:105810007A898B899C890E948EB59B01AC01C3015A
:10582000B2010E94E0B12B013C01A50194016D89F8
:105830007E898F89988D0E948EB54B015C01A701EE
:10584000960169897A898B899C890E948EB59B0112
:10585000AC01C501B4010E94DFB1A30192010E9415
:1058600053B26B017C0120E030E0A9010E94B9B283
:1058700087FF0AC02BED3FE049EC50E4C701B601B9
:105880000E94E0B16B017C01AA968FADAA97882394
:1058900051F02BED3FE049EC50E4C701B6010E9406
:1058A000DFB16B017C012FA538A949A95AA9698DDF
:1058B0007A8D8B8D9C8D0E94B9B281111FC02BA94E
:1058C0003CA94DA95EA96F8D78A189A19AA10E94DA
:1058D000B9B2811113C020E030E0A901C701B601BF
:1058E0000E94B9B281110AC02BED3FE049EC50E4AF
:1058F000C701B6010E94E0B16B017C01A9962CADF5
:105900003DAD4EAD5FADA997C701B6010E948EB502
:105910002FA138A549A55AA55F770E94C9B44B01AC
:105920005C012FE632E143E85AE30E94B9B287FDF9
:10593000C8C1C501B4010E9496B30E942DB37A8FED
:10594000698FDB01AB2B21F4E1E0F0E0FA8FE98F06
:10595000298D3A8DB90180E090E00E9459B34B0146
:105960005C019B01AC01C701B6010E94C0B22B01D2
:105970003C01A50194016FA178A589A59AA50E9473
:10598000C0B26FA778AB89AB9AAB2BA53CA54DA550
:105990005EA560966CAD7DAD8EAD9FAD60970E94AB
:1059A000DFB1A50194010E94C0B26BAB7CAB8DABA3
:1059B0009EAB20E030E040E05FE3C301B2010E9413
:1059C0008EB5A30192010E948EB59B01AC0160E0EF
:1059D00070E080E89FE30E94DFB16FA378A789A7FA
:1059E0009AA7CE010196FC0128964FAD289734E086
:1059F000439FE00DF11D11242BA13CA14DA15EA1FF
:105A000020833183428353832BA53CA54DA55EA5FE
:105A10002D873E874F87588BB12C41E050E058A32B
:105A20004F8F1C01BFA9A4E0BA9F800D911D1124C6
:105A300098AF8FAB910159AD44E0549F200D311DBB
:105A400011243AAF29AFFCA7EBA74F8D58A1898D40
:105A50009A8D4817590708F01AC188E18B150CF484
:105A600044C02FA138A549A55AA569897A898B898F
:105A70009C890E948EB56B017C01A30192016D8906
:105A80007E898F89988D0E948EB5A70196010E940C
:105A9000E0B1A62E172F982E892E2FA138A549A543
:105AA0005AA56D897E898F89988D0E948EB56B016C
:105AB0007C01A301920169897A898B899C890E9462
:105AC0008EB59B01AC01C701B6010E94DFB16D8BA1
:105AD0007E8B8F8B988FB3948A2D912FA92DB82D03
:105AE000898B9A8BAB8BBC8B6CC0AF8DB8A1BD0181
:105AF00080E090E00E9459B3A30192010E948EB50C
:105B00006B017C010E94BDB2698B7A8B8B8B9C8B65
:105B1000C701B6010E94F1B54B015C01EBADFCADD4
:105B2000C080D180E280F380F7FAF094F7F8F09427
:105B30002396AEADBFAD23972D913D914D915C91D4
:105B40002BA33CA34DA35EA329893A894B895C8989
:105B5000C701B6010E948EB56D8B7E8B8F8B988F9F
:105B6000A50194016BA17CA18DA19EA10E948EB57F
:105B70009B01AC016D897E898F89988D0E94E0B16F
:105B80006D8B7E8B8F8B988FA5019401C701B60119
:105B90000E948EB56B017C0129893A894B895C8909
:105BA0006BA17CA18DA19EA10E948EB59B01AC0131
:105BB000C701B6010E94DFB1698B7A8B8B8B9C8BFE
:105BC000B12C2D893E894F89588D21966CAD7DADC4
:105BD0008EAD9FAD21970E94E0B1EFA9F8AD608333
:105BE00071838283938329893A894B895C892796BB
:105BF0006CAD7DAD8EAD9FAD27970E94E0B1A9AD94
:105C0000BAAD6D937D938D939C9313972FA538A96F
:105C100049A95AA9EBA5FCA5608171818281938174
:105C20000E94E0B1ABA5BCA56D937D938D939C9331
:105C300013972BA93CA94DA95EA96D857E858F85FB
:105C400098890E94E0B16D877E878F87988BC1010C
:105C50000E94C542FE01E659FF4F6F012C96ECAC45
:105C6000FDAC0EAD1FAD2C979E01235F3F4FAE01E3
:105C7000475F5F4FBE016B5F7F4FC1010E94909EE7
:105C80002F8D38A12F5F3F4F38A32F8FDECE2D8D64
:105C90003E8D245F3F4F4D8D5E8D485F5F4F6D8D14
:105CA0007E8D6C5F7F4FDE01A659BF4F6D012C9634
:105CB000ECACFDAC0EAD1FAD2C978D8D9E8D0E9472
:105CC000909EC15BDF4F0FB6F894DEBF0FBECDBF15
:105CD000DF91CF911F910F91FF90EF90DF90CF90C8
:105CE000BF90AF909F908F907F906F905F904F90FC
:105CF0003F902F900895FC01148217821382128224
:105D000088ED95E091838083089528ED35E0FC01CE
:105D1000318320832781222319F004960C943A14AE
:105D20000895CF92DF92EF92FF920F931F93CF933C
:105D3000DF93EC01875B9F4FDEDFCE0186599F4FDB
:105D4000DADF7E0129E8E20EF11C87016E0131E401
:105D5000C31A3EEFD30AC801CEDF015E1F4F0C15F8
:105D60001D05C9F7FE01EF53FE4F89E181831482BF
:105D70003596178ACE018C519E4FBDDFFE01EB5642
:105D8000FD4F108211821282138238961082118286
:105D9000128213821A821B82188219826E0187E690
:105DA000C81A8DEFD80AF60110821182128213826E
:105DB000F80111821082FE01ED5FFD4F108286E333
:105DC00091E0F7019C01119221503040E1F7FE0172
:105DD000EF55FD4F81E08083C95BDF4F1982188248
:105DE0000E944AAD68577C4E8F4F9F4FF6016083EB
:105DF000718382839383DF91CF911F910F91FF90E5
:105E0000EF90DF90CF900895FC0120E03EE2DB01AF
:105E10004C91403241F0283011F430833196DB014F
:105E20004C91408331962F5F6F5F7F4F2B3079F716
:105E3000108208952F923F924F925F926F927F92BD
:105E40008F929F92AF92BF92CF92DF92EF92FF928A
:105E50000F931F93CF93DF93CDB7DEB7CA58D10905
:105E60000FB6F894DEBF0FBECDBF8C016B017A0177
:105E70004901CA57DF4F1882C658D04084E0E80E67
:105E8000F11C180191E1290E311CF801EA5BFF4F6A
:105E9000C957DF4FF983E883C758D0403801FEE582
:105EA0006F1AFDEF7F0A58018CE5A81A8DEFB80A2A
:105EB00080E4482E512C4C0E5D1E94E0490E511C7E
:105EC000A101BE016F5F7F4FC7010E94A412181687
:105ED0000CF03CC12C85322F3871303109F09EC056
:105EE000F301808191810197029708F497C0BE0168
:105EF0006F5F7F4FCE0187589F4F86DFA0961FAE02
:105F0000A097F6018081811107C065E773E0CE019B
:105F1000815A9F4F0E9431BAB601CE01815A9F4FDC
:105F20000E9431BABE0167587F4FCE01815A9F4F00
:105F30000E9431BA65E773E0CE01815A9F4F0E94FB
:105F400031BACE01805C9F4FD6DE21E0AE014758CA
:105F50005F4FB701C2010E943116811139C0F301B0
:105F600080819181892BA1F5ECEBFEE0849188235F
:105F700041F09091C00095FFFCCF8093C600319610
:105F8000F5CFE7E7F3E08191882339F09091C000E5
:105F900095FFFCCF8093C600F6CF8091C00085FFAF
:105FA000FCCF8AE08093C600FE01E758FF4F819145
:105FB000882339F09091C00095FFFCCF8093C600F4
:105FC000F6CF8091C00085FFFCCF8AE08093C600A9
:105FD0008BE1FE01EC5BFF4FDE01959601900D9287
:105FE0008A95E1F724968EAD9FAD24979CA38BA351
:105FF00088ED95E09AA389A320E030E0AE014F5DE3
:106000005F4FBE01615A7F4FC80114DFCE018196F8
:106010007CDECE01805C9F4F78DE52CF8981882361
:1060200009F494C08E3209F44BCF8F3509F448CF70
:10603000F80181898E3209F443CF8F3509F440CFBE
:1060400023FD3ECF81E0303109F080E0C957DF4FBA
:10605000E881F981C758D0408083811108C08985C3
:10606000873409F02DCF8A858E3709F429CF98011E
:106070002C5F3F4FBE016F5F7F4FC901C757DF4F96
:106080002883C958D040C657DF4F3883CA58D040FC
:10609000BBDEF30180819181C757DF4F2881C9584A
:1060A000D040C657DF4F3881CA58D0400097F1F42E
:1060B000F6018191882339F09091C00095FFFCCFC3
:1060C0008093C600F6CFF9018191882339F0909131
:1060D000C00095FFFCCF8093C600F6CF8091C00032
:1060E00085FFFCCF8AE08093C600EACE813091051F
:1060F00039F4F50180819181019691838083E0CE0E
:10610000029709F0DDCE8114910439F0B901C40180
:106110000E941EBA892B71F419C0CA57DF4FF8814B
:10612000C658D0402F2F30E0F5018081918128178B
:10613000390761F0CA57DF4FF881C658D040FF5F7A
:10614000CA57DF4FF883C658D040BACEC657DF4F84
:106150000FB6F894DEBF0FBECDBFDF91CF911F9178
:106160000F91FF90EF90DF90CF90BF90AF909F90F6
:106170008F907F906F905F904F903F902F900895F9
:106180000F931F93CF93DF93CDB7DEB76F970FB603
:10619000F894DEBF0FBECDBF8C01FC01EE55FD4F64
:1061A0001182108240E050E0BA01835B9F4F0E9451
:1061B0005713C801875B9F4F2BE1FC013496DE012A
:1061C000159601900D922A95E1F7FC018281938149
:1061D0009C838B8388ED95E09A83898320E030E06F
:1061E000AE014F5F5F4F6EE973E0C80123DECE0161
:1061F00001968BDD6F960FB6F894DEBF0FBECDBF54
:10620000DF91CF911F910F9108952BE1FB013496FF
:10621000DC01149601900D922A95E1F7FB01228191
:106220003381FC01338322830895EF92FF920F9311
:106230001F93CF93DF93EC011B82FC01E05BFF4FC8
:106240008081882329F0CE01835B9F4F0E943A14FE
:106250007E018FE3E81A8EEFF80A45E360E0C7019C
:106260000E941A3C81111FC0ECEBFEE08491882350
:1062700041F09091C00095FFFCCF8093C60031960D
:10628000F5CFE8ECF6E08491882341F09091C000CE
:1062900095FFFCCF8093C6003196F5CF8091C0006A
:1062A00085FFFCCF77C08E010A531E4F41E0B70136
:1062B000C8010E94081C811126C040E0B701C80136
:1062C0000E94081C81111FC0E2ECFEE0849188232B
:1062D00041F09091C00095FFFCCF8093C6003196AD
:1062E000F5CFE5EBF6E08491882341F09091C00072
:1062F00095FFFCCF8093C6003196F5CF8091C0000A
:1063000085FFFCCF47C0B801CE01835B9F4F0E9441
:10631000471181111FC0E2ECFEE08491882341F017
:106320009091C00095FFFCCF8093C6003196F5CFC9
:10633000E5EAF6E08491882341F09091C00095FF52
:10634000FCCF8093C6003196F5CF8091C00085FFC9
:10635000FCCF20C081E08B83ECEBFEE084918823AE
:1063600041F09091C00095FFFCCF8093C60031961C
:10637000F5CFEAE9F6E08491882341F09091C000DE
:1063800095FFFCCF8093C6003196F5CF8091C00079
:1063900085FFFCCF8AE08093C6008E01075B1F4F0C
:1063A000B801CE0186599F4F30DFC859DF4F19839E
:1063B0000883DF91CF911F910F91FF90EF90089587
:1063C000FC01128213820895FC012381222311F023
:1063D00021E022830895FC01228121111282089577
:1063E000AF92BF92CF92DF92EF92FF920F931F93E3
:1063F000CF93DF931F92CDB7DEB78C018FE2FB0105
:1064000081935F01D12C41E07801F1E4EF1AFEEFB6
:10641000FF0A9FE1C92E2D2D30E0F7018081918187
:1064200028173907D8F4C29EC001C39E900D1124CD
:1064300083579F4FB501800F911F49830E94EE1033
:10644000C50149815C010196F5012081222321F0DB
:106450004D3810F44F5FF6CFD394DDCF47FD11C018
:10646000B501C80188519E4F0F90DF91CF911F91C8
:106470000F91FF90EF90DF90CF90BF90AF900C9472
:10648000EE10F50110820F90DF91CF911F910F91C7
:10649000FF90EF90DF90CF90BF90AF9008953F9224
:1064A0004F925F926F927F928F929F92AF92BF9224
:1064B000CF92DF92EF92FF920F931F93CF93DF93D0
:1064C000CDB7DEB7AC970FB6F894DEBF0FBECDBF29
:1064D0007C015B01FC018381882309F408C1C701A9
:1064E00088519E4F0E943A14F7011282CE01019604
:1064F0006C0101DC270198E6490E511CC701875B3E
:106500009F4FF20191838083F50180818F3209F0E2
:1065100084C06FE270E0C5010E943CBA8C010F5F3D
:106520001F4F2AE0322E0115110509F47CC06FE2DD
:1065300070E0C8010E943CBA4C01009709F474C095
:106540000817190708F070C03C01601A710AA3010E
:10655000B801CE0180960E9465BAE0E2F0E0EC0F4F
:10656000FD1FE60DF71D1082FE01B0968191882374
:1065700039F09091C00095FFFCCF8093C600F6CF14
:106580008091C00085FFFCCF3092C600F20160818F
:1065900071816115710519F06C5F7F4F02C060E079
:1065A00070E021E0AE01405E5F4FCE0105960E9493
:1065B000311681112BC0EFE7F5E08491882341F07B
:1065C0009091C00095FFFCCF8093C6003196F5CF27
:1065D000FE01B0968191882339F09091C00095FF1B
:1065E000FCCF8093C600F6CFEDE7F5E084918823D9
:1065F00041F09091C00095FFFCCF8093C60031968A
:10660000F5CF8091C00085FFFCCF6CC0F201D18234
:10661000C08284010F5F1F4F86CFC70186599F4FED
:10662000F201918380838501F2018081918100973D
:1066300011F0049602C080E090E0B8010E940717B4
:10664000882339F1EFE6F5E08491882341F09091B9
:10665000C00095FFFCCF8093C6003196F5CFF801BE
:106660008191882339F09091C00095FFFCCF8093F1
:10667000C600F6CF8091C00085FFFCCF8AE08093F2
:10668000C600F701E356FD4F108211821282138279
:106690002CC0E7E5F5E08491882341F09091C0009B
:1066A00095FFFCCF8093C6003196F5CFF80181911C
:1066B000882339F09091C00095FFFCCF8093C600ED
:1066C000F6CFE5E5F5E08491882341F09091C00094
:1066D00095FFFCCF8093C6003196F5CF8091C00026
:1066E00085FFFCCF8AE08093C600C6010EDBAC9626
:1066F0000FB6F894DEBF0FBECDBFDF91CF911F91D3
:106700000F91FF90EF90DF90CF90BF90AF909F9050
:106710008F907F906F905F904F903F9008958F92F1
:106720009F92AF92BF92CF92DF92EF92FF92CF9360
:10673000DF931F92CDB7DEB77C01FC0182818823F5
:1067400009F4AFC071968191882339F09091C0000F
:1067500095FFFCCF8093C600F6CFE3E5F5E084918A
:10676000882341F09091C00095FFFCCF8093C60034
:106770003196F5CFE1E4F5E08491882341F09091E2
:10678000C00095FFFCCF8093C6003196F5CFF7018E
:10679000E356FD4F40815181628173812AE030E0F0
:1067A00087EC9DE00E94468EEFE3F5E0849188231C
:1067B00041F09091C00095FFFCCF8093C6003196C8
:1067C000F5CFF701EB56FD4F408151816281738116
:1067D0002AE030E087EC9DE00E94468E8091C00068
:1067E00085FFFCCF8AE08093C6000E944AAD30E668
:1067F000C32E3AEED32EE12CF12CA70196010E9474
:1068000097B649015A0160917008709171088091A2
:10681000720890917308A70196010E9497B6821A98
:10682000930AC4016CE370E00E9470B66983CE01E4
:1068300001960E945E7AFC012191CF01222339F05A
:106840003091C00035FFFCCF2093C600F4CF40E06C
:1068500050E06AE387EC9DE00E94FE8DC4016CE38A
:1068600070E00E9470B68983CE0101960E945E7A24
:10687000FC012191CF01222339F03091C00035FF76
:10688000FCCF2093C600F4CFEDE3F5E0849188239C
:10689000E1F09091C00095FFFCCF8093C600319647
:1068A000F5CFE0E3F5E08491882341F09091C000BA
:1068B00095FFFCCF8093C6003196F5CF8091C00044
:1068C00085FFFCCF8AE08093C6000F90DF91CF91C7
:1068D000FF90EF90DF90CF90BF90AF909F908F9000
:1068E0000895AF92BF92CF92DF92EF92FF920F93F3
:1068F0001F93CF93DF935C01EB01FB01019000201C
:10690000E9F78F0101501109061B170B6C01F8E123
:10691000CF1AFEEFDF0AF60110826EE470E0CE01BE
:106920000E943CBA7C01009729F4F8013197EC0FE2
:10693000FD1F0DC060E270E00E943CBAEC012196A0
:106940006AE270E0C7010E943CBAFC0131978DE019
:1069500081838AE082831382BE01C5018C519E4FE0
:106960000E94038FF6018081882309F1E2ECFEE0AA
:106970008491882341F09091C00095FFFCCF8093D3
:10698000C6003196F5CFEAE1F5E08491882341F025
:106990009091C00095FFFCCF8093C6003196F5CF53
:1069A0008091C00085FFFCCF8AE08093C600DF9114
:1069B000CF911F910F91FF90EF90DF90CF90BF90FC
:1069C000AF9008952F923F924F925F926F927F9275
:1069D0008F929F92AF92BF92CF92DF92EF92FF92EF
:1069E0000F931F93CF93DF93CDB7DEB7CC55D1096B
:1069F0000FB6F894DEBF0FBECDBF4C018C010F5512
:106A00001D4F662339F0F8011082F4018381811152
:106A10001DC015C0F8018081882309F4AFC0F401BE
:106A2000E756FD4FC080D180E280F3800E944AADDE
:106A3000C616D706E806F90608F4A0C0E4CFC401DC
:106A4000F4DBF4018381882309F498C07401F7E42E
:106A5000EF0EF11CF70181818F9380818F9381E18B
:106A600095E09F938F938E01015C1F4F1F930F93AF
:106A70000E9474BA0F900F900F900F900F900F908C
:106A8000B12CF80101900020E9F73197E01BF10BE0
:106A9000BE1684F46801CB0CD11CB7FCDA94F60165
:106AA0008081992787FD90950E94B1B9F601808376
:106AB000B394E7CFFDE48F0E911C40E050E0BA01A3
:106AC000C4010E945713512CCE0101966C014AE07B
:106AD000642E45E0742E5E0191E2A90EB11C40E0E7
:106AE00050E0B601C4010E94A4121816DCF5412C36
:106AF000F60101900020E9F73197EC19FD094E16D7
:106B000074F41601240C311C47FC3A94F101808185
:106B100090E00E94B1B9F10180834394E9CF8A8566
:106B20008E37E9F245E050E0B801C6010E9457BA3D
:106B3000892BA9F61F930F937F926F92BF92AF920A
:106B40000E9474BAC5010E941B3F86E095E00E9436
:106B50008E3F0F900F900F900F900F900F90552435
:106B60005394BDCF511004C08FEF9FEFF70104C0C5
:106B7000F70180819181019691838083C45ADF4F10
:106B80000FB6F894DEBF0FBECDBFDF91CF911F913E
:106B90000F91FF90EF90DF90CF90BF90AF909F90BC
:106BA0008F907F906F905F904F903F902F900895BF
:106BB0000F931F93CF93DF93EC018C0108511E4F6D
:106BC000C8010E94F013C8010E943A141882198269
:106BD000DF91CF911F910F910895CF92DF92EF92A5
:106BE000FF920F931F93CF93DF93CDB7DEB76F97CD
:106BF0000FB6F894DEBF0FBECDBF8C016A017C01D9
:106C000088E6E80EF11CC80186599F4FF701918371
:106C10008083E65CFD4F22E030E0318320833296B2
:106C20007183608340E050E0BA0104960E945713DC
:106C3000F701808191812BE1FC013496DE011596EC
:106C400001900D922A95E1F7FC01828193819C834A
:106C50008B8388ED95E09A8389839601AE014F5F1F
:106C60005F4F6EE973E0C801E5D8CE0101964DD8BB
:106C70006F960FB6F894DEBF0FBECDBFDF91CF91F8
:106C80001F910F91FF90EF90DF90CF9008952F927A
:106C90003F924F925F926F927F928F929F92AF92AC
:106CA000BF92CF92DF92EF92FF920F931F93CF93F9
:106CB000DF93CDB7DEB7AC970FB6F894DEBF0FBE4B
:106CC000CDBF8C016B01342EDC0113968C9188238F
:106CD00009F4EEC2F801E551FE4F8081882309F4E2
:106CE000F5C02111C1C07801BDEFEB1AFB0AF70115
:106CF0008081882361F1E2ECFEE08491882341F0F9
:106D00009091C00095FFFCCF8093C6003196F5CFDF
:106D1000E7E5F6E08491882341F09091C00095FF6B
:106D2000FCCF8093C6003196F5CF4AE050E061E099
:106D300070E087EC9DE00E941A8E8091C00085FF74
:106D4000FCCF8AE08093C6000E947D46B1C2ECEB86
:106D5000FEE08491882341F09091C00095FFFCCF24
:106D60008093C6003196F5CFEEE3F6E08491882358
:106D700041F09091C00095FFFCCF8093C600319602
:106D8000F5CFF6018191882339F09091C00095FFED
:106D9000FCCF8093C600F6CFE3E3F6E0849188232E
:106DA00041F09091C00095FFFCCF8093C6003196D2
:106DB000F5CFD7018C916DE8B62EB801B89E600D65
:106DC000711D1124685F7D4FC8010ADBF7018081C6
:106DD000F801B89EE00DF11D1124E85FFD4F81918F
:106DE000882339F09091C00095FFFCCF8093C600B6
:106DF000F6CFEDE2F6E08491882341F09091C00057
:106E000095FFFCCF8093C6003196F5CF5801F3E68D
:106E1000AF1AFDEFBF0AD5014D915D916D917C9147
:106E20002AE030E087EC9DE00E94468E8091C00011
:106E300085FFFCCF8AE08093C600F7012081F8012E
:106E400084E0289FE00DF11D1124EC5FFD4FD5017A
:106E50004D915D916D917C914083518362837383E9
:106E60002F5FF70120832CC0ECEBFEE08491882398
:106E700041F09091C00095FFFCCF8093C600319601
:106E8000F5CFECE1F6E08491882341F09091C000C9
:106E900095FFFCCF8093C6003196F5CFF601819126
:106EA000882339F09091C00095FFFCCF8093C600F5
:106EB000F6CF8091C00085FFFCCF8AE08093C600AA
:106EC000C80188519E4F0E943A1430C0F801ED5F0E
:106ED000FD4F1082ECEBFEE08491882341F090910D
:106EE000C00095FFFCCF8093C6003196F5CFEBE054
:106EF000F6E08491882341F09091C00095FFFCCF8B
:106F00008093C6003196F5CFF6018191882339F040
:106F10009091C00095FFFCCF8093C600F6CF809182
:106F2000C00085FFFCCF8AE08093C600D80112968E
:106F30001C92FE0131965F01CF010E947B2E280139
:106F4000F8E64F0E511CC801875B9F4FD2018D930D
:106F50009C93F60180818F3209F084C06FE270E06B
:106F6000C6010E943CBA01967C015AE0252EE1142C
:106F7000F10409F47DC06FE270E0C7010E943CBAE1
:106F80004C01009709F475C0E816F90608F071C0C5
:106F90003C016E187F08A301B701CE0180960E94C4
:106FA00065BAE0E2F0E0EC0FFD1FE60DF71D108280
:106FB000FE01B0968191882339F09091C00095FF31
:106FC000FCCF8093C600F6CF8091C00085FFFCCF38
:106FD0002092C600D2016D917C916115710519F066
:106FE0006C5F7F4F02C060E070E021E0AE01405E68
:106FF0005F4FCE0105960E94311681112BC0E7EF3D
:10700000F5E08491882341F09091C00095FFFCCF7A
:107010008093C6003196F5CFFE01B096819188230A
:1070200039F09091C00095FFFCCF8093C600F6CF59
:10703000E5EFF5E08491882341F09091C00095FF41
:10704000FCCF8093C6003196F5CF8091C00085FFBC
:10705000FCCF02C1F201B182A0827401FFEFEF1AEE
:10706000FF0A85CFC80186599F4FD2018D939C930B
:107070007601F801E851FE4F4F01332009F4B1C009
:10708000D2016D917C916115710519F06C5F7F4F94
:1070900002C060E070E021E0A701C4010E94311647
:1070A000882309F474C0F40181899289A389B48981
:1070B000F801EB56FD4F80839183A283B383E7EE03
:1070C000F5E08491D801AB56BD4F882349F09091EB
:1070D000C00095FFFCCF8093C60031968491F5CF18
:1070E000F7018191882339F09091C00095FFFCCF82
:1070F0008093C600F6CFEFEDF5E08491882341F050
:107100009091C00095FFFCCF8093C6003196F5CFDB
:107110004D915D916D917C912AE030E087EC9DE08E
:107120000E94468E8091C00085FFFCCF8AE080934C
:10713000C600F801E356FD4F1082118212821382BD
:10714000E1EDF5E08491882341F09091C00095FF36
:10715000FCCF8093C6003196F5CF8091C00085FFAB
:10716000FCCF8AE08093C600A70160E070E0C80110
:1071700034DDD80151968C91882319F0C8014196CD
:1071800001C0C7010E949A738AE893E08CC0EDEBBE
:10719000F5E08491882341F09091C00095FFFCCFE9
:1071A0008093C6003196F5CFF7018191882339F09D
:1071B0009091C00095FFFCCF8093C600F6CFEBEB1B
:1071C000F5E08491882341F09091C00095FFFCCFB9
:1071D0008093C6003196F5CF8091C00085FFFCCF2B
:1071E0003BC0F201608171816115710519F06C5F1E
:1071F0007F4F02C060E070E026E5A701C4010E9455
:10720000311681112DC0E7EAF5E08491882341F021
:107210009091C00095FFFCCF8093C6003196F5CFCA
:10722000F7018191882339F09091C00095FFFCCF40
:107230008093C600F6CFE5EAF5E08491882341F01B
:107240009091C00095FFFCCF8093C6003196F5CF9A
:107250008091C00085FFFCCF8AE08093C60025C0E6
:1072600081E0D8018C93E3E9F5E08491882341F033
:107270009091C00095FFFCCF8093C6003196F5CF6A
:10728000F6018191882339F09091C00095FFFCCFE1
:107290008093C600F6CF8091C00085FFFCCF8AE0C6
:1072A0008093C600C7010E949A73C5010E94852E73
:1072B000AC960FB6F894DEBF0FBECDBFDF91CF9175
:1072C0001F910F91FF90EF90DF90CF90BF90AF9004
:1072D0009F908F907F906F905F904F903F902F90F6
:1072E000089521E0FC01218340E0D1CCCF92DF92D0
:1072F000EF92FF920F931F93CF93DF93CDB7DEB73B
:107300006F970FB6F894DEBF0FBECDBF8C016C0136
:1073100028E6C20ED11C86599F4FF60191838083C7
:10732000E65CFD4F21E030E0318320837801FCE50D
:10733000EF1AFDEFFF0AF7011182108240E050E0E2
:10734000BA0104960E945713F601808191812BE1C6
:10735000FC013496DE01159601900D922A95E1F715
:10736000FC01828193819C838B8388ED95E09A83D5
:10737000898320E030E0AE014F5F5F4F6EE973E03C
:10738000C8010E941A2FCE0101960E94852EF70196
:10739000808191816F960FB6F894DEBF0FBECDBF8E
:1073A000DF91CF911F910F91FF90EF90DF90CF90E1
:1073B0000895AF92BF92CF92DF92EF92FF920F9318
:1073C0001F93CF93DF93CDB7DEB76F970FB6F894C7
:1073D000DEBF0FBECDBF8C017B01CE0101960E94A6
:1073E0007B2EF801EF58FF4F80816801811104C0A6
:1073F00029E4C20ED11C03C08AE6C80ED11C21E0CC
:10740000A701B6016C5F7F4FCE0105960E94311631
:1074100081112DC0ECEBFEE08491882341F0909126
:10742000C00095FFFCCF8093C6003196F5CFE0EF0A
:10743000F4E08491882341F09091C00095FFFCCF47
:107440008093C6003196F5CFF7018191882339F0FA
:107450009091C00095FFFCCF8093C600F6CF80913D
:10746000C00085FFFCCF8AE08093C60036C0F801DB
:10747000E154FE4F808191818A30910530F59C0165
:107480002F5F3F4F318320832FE1289F7001299F79
:10749000F00C112429E8E20EF11CE00EF11E5C0153
:1074A000B701C7014F960E94053181E0A81AB108C3
:1074B0002FE1E21AF1088FEFA816B80689F7B60196
:1074C000C80187579F4F0E940531BE016F5F7F4FF4
:1074D000C80186599F4F0E940531CE0101960E9436
:1074E000852E6F960FB6F894DEBF0FBECDBFDF912D
:1074F000CF911F910F91FF90EF90DF90CF90BF90B1
:10750000AF900895EF92FF920F931F93CF93DF9365
:10751000EC01C154DE4F2881398121153105F9F084
:1075200021503109398328838C0107571F4FB80137
:1075300086599F4F0E940531C80100E010E07C0190
:107540002FE1E20EF11C288139810217130738F46C
:107550000F5F1F4FB7010E940531C701F0CFDF91C8
:10756000CF911F910F91FF90EF900895EF92FF92AE
:107570000F931F93CF93DF93EC010E94FD968E0132
:107580000D5F1D4FF80180819E0128513E4F79010A
:107590008823A1F1C9010E943A14F8018081815029
:1075A0008083BE01FDE88F9F600D711D1124685F0F
:1075B0007D4F21E041E0CE016ADBF8018081FE01D0
:1075C00024E0829FE00DF11D1124EC5FFD4F40810E
:1075D000518162817381FE01E356FD4F40835183E7
:1075E00062837383C7010E945713CE01DF91CF914D
:1075F0001F910F91FF90EF900C94E4310E947397CC
:10760000C7010E943A141A8284EE94E0DF91CF9170
:107610001F910F91FF90EF9081C48FEF8EBD0DB43D
:1076200007FEFDCF8EB508958EBD0DB407FEFDCFCC
:10763000089561E0FC0180810C94A3ACFC012281DF
:10764000322F306A36953CBD20FD06C031E0263031
:1076500009F430E0232F01C020E02DBD60E0FC01E3
:1076600080810C94A3ACCF92DF92EF92FF920F93A4
:107670001F93CF93DF93EC018B017A010E944AADF7
:107680006B01CBDF8B838F3F49F40E944AAD6C19AD
:107690007D096D327140A8F381E144C08E3F11F045
:1076A0008FE040C0E114F104D9F0C70101972FEF3A
:1076B0002EBDF8014FEF9F01201B310B2817390712
:1076C00038F40DB407FEFDCF2EB521934EBDF3CF98
:1076D0000DB407FEFDCF2EB5F801E80FF91F20838A
:1076E000D801E00EF11EC12CD12CAE15BF0579F0EA
:1076F0008D91ED2DFF27E827EE0FFF1FEB52F94F7D
:1077000085919491DC2CCC24C826D926EECF85DF38
:10771000082F10E0102F002780DF082BC016D1069D
:1077200031F080E28983CE0184DF80E003C0CE01A6
:1077300080DF81E0DF91CF911F910F91FF90EF905B
:10774000DF90CF9008950F931F93CF93DF93EB01BA
:107750000E944AAD8B0161DF8F3F49F00E944AAD24
:10776000601B710B6C177D07B0F380E001C081E0F6
:10777000DF91CF911F910F910895CF92DF92FF92E9
:107780000F931F93CF93DF9300D01F92CDB7DEB737
:107790006C01F62E29833A834B835C834FDF6CE2C6
:1077A00071E0C601D0DF8F2D80643EDF08E110E07C
:1077B0005C814B813A812981DA01C901002E04C024
:1077C000B695A795979587950A94D2F729833A831A
:1077D0004B835C8329DF0850110929813A814B8151
:1077E0005C81083F8FEF180739F7FF2029F0E8E0A8
:1077F000FE1621F08FEF03C085E901C087E814DF92
:10780000FCE0FF1201C009DF10E007DFF60183830F
:1078100087FF04C01F3F11F01F5FF7CF0F900F903D
:107820000F900F90DF91CF911F910F91FF90DF90FC
:10783000CF900895BF92CF92DF92EF92FF920F9375
:107840001F93CF93DF93EC01B62E1C8219824883DD
:107850000E944AAD8B0161E088810E946AACCE0132
:10786000E8DE60E082E30E946AAC61E083E30E94AC
:107870006AAC61E084E30E946AAC61E085E30E9447
:107880006AAC61E085E30E94A3AC85E08A8382E56F
:107890008CBD1DBC6AE0F62E8FEFC6DEFA94E1F7D0
:1078A00020E030E0A90160E0CE0167DFF82E8B8395
:1078B00081E0F81649F00E944AAD601B710B613DF2
:1078C000774070F381E046C02AEA31E040E050E0C2
:1078D00068E0CE0152DF82FF02C0FC820CC054E09F
:1078E000F52E9BDE8B83FA94E1F78A3A11F082E061
:1078F00031C082E08C838C81823031F4C12CD12C58
:10790000E12C40E4F42E03C0C12CD12C760120E000
:1079100030E0A90167E3CE0130DFA701960169E2FB
:10792000CE012BDF8B83882349F00E944AAD601B78
:10793000710B613D774058F38AE00CC08C81823036
:10794000B1F420E030E0A9016AE3CE0116DF88231C
:1079500029F088E08983CE016CDE14C05EDE807C75
:10796000803C11F483E08C8358DE57DE56DECE0176
:1079700060DE86E08B1518F488E1898303C0BA8243
:1079800081E001C080E0DF91CF911F910F91FF90C6
:10799000EF90DF90CF90BF900895AF92BF92CF92BB
:1079A000DF92EF92FF920F931F93CF93DF93EC013F
:1079B0006A017B0189018C81833039F0F9E0CC0CBC
:1079C000DD1CEE1CFF1CFA95D1F773E0B72EE4E046
:1079D000AE2EBA94A701960161E1CE01CEDE8823D6
:1079E00011F0A98207C040E052E0B801CE013BDEB1
:1079F00081110EC0CE01BB2049F01BDE20E030E03B
:107A0000A9016CE0CE01B9DE1982E3CF12DE80E07D
:107A1000DF91CF911F910F91FF90EF90DF90CF906A
:107A2000BF90AF900895CF93DF93EC016EBD20E03F
:107A300030E00DB407FEFDCFFA01E20FF31F8081A5
:107A40008EBD0DB407FEFDCF81818EBD2E5F3F4FF1
:107A5000211582E0380769F70DB407FEFDCF8FEFDF
:107A6000E3DD8FEFE1DDD9DD8B838F71853031F080
:107A700083E18983CE01DDDD80E001C081E0DF911B
:107A8000CF9108950F931F93CF93DF93EC0189015A
:107A90008C81833039F0B9E0440F551F661F771F82
:107AA000BA95D1F79A01AB0168E1CE0166DE882371
:107AB00011F086E01EC0A8016EEFCE01B4DF88236E
:107AC000C9F068E572E0CE013EDE182F811102C0D8
:107AD00087E10FC020E030E0A9016DE0CE014DDE6E
:107AE000811106C09ADD811103C0CE01A2DD05C05F
:107AF00086E18983CE019DDD10E0812FDF91CF915A
:107B00001F910F910895FC01659175918591949154
:107B100008952F923F924F925F926F927F928F9231
:107B20009F92AF92BF92CF92DF92EF92FF920F930C
:107B30001F93CF93DF9300D000D0CDB7DEB71C01E9
:107B4000FC01E358F14F14919C01220F331F220FC7
:107B5000331F3E832D832E59354F4901F901108281
:107B60001182128213822EE63AE04AE65AE066E675
:107B70007AE082E69AE00E9457A88D819E81845720
:107B8000914FC1DF6B017C01612F772767FD7095F5
:107B9000872F972F0E945BB32B013C012D813E81E3
:107BA000235D354F590120E030E040EC5FE3C70131
:107BB000B6010E948EB5A30192010E948EB5F50117
:107BC00060837183828393832D813E81215A3D4F4F
:107BD0003C832B83F9016081718182819381609361
:107BE000210270932202809323029093240220E0CA
:107BF00030E040E752E40E94C0B22EE4C22E2AE0F8
:107C0000D22E7B018C0129E33AE045E35AE061E39F
:107C10007AE08DE29AE00E94909E0E94FD96F40127
:107C200010821182128213822EE63AE04AE65AE06E
:107C300066E67AE082E69AE00E9457A82D813E81AE
:107C40002058314F3A832983C9015DDF9058A30141
:107C500092010E948EB5F5016083718382839383C4
:107C600020E030E040E752E460912102709122026E
:107C700080912302909124020E94C0B27B018C016A
:107C800029E33AE045E35AE061E37AE08DE29AE0E5
:107C90000E94909E0E94FD9689819A8134DF9B010B
:107CA000AC010E94E0B1A30192010E948EB5F501E2
:107CB000608371838283938320E030E040E05FE360
:107CC000EB81FC8160817181828193810E948EB5FC
:107CD00060932102709322028093230290932402E6
:107CE00020E030E040E752E40E94C0B27B018C010A
:107CF00029E33AE045E35AE061E37AE08DE29AE075
:107D00000E94909E0E94FD968D819E818856914F83
:107D1000FADE0D811E810A5A154FF801208131814A
:107D2000428153810E94E0B1F401608371838283B8
:107D300093838D819E818055914FE5DE2D813E811B
:107D40002D5B3D4F7901F8012081318142815381C2
:107D50000E94E0B1F70160837183828393838D81F8
:107D60009E818C55914FCFDE2D813E81295C3D4F08
:107D70007901F80120813181428153810E94E0B173
:107D8000F7016083718382839383F4018081918101
:107D9000A281B381F50180839183A283B383109282
:107DA00021021092220210922302109224020E94B9
:107DB000AA8FF101ED5AF54F81E0808326960FB628
:107DC000F894DEBF0FBECDBFDF91CF911F910F9111
:107DD000FF90EF90DF90CF90BF90AF909F908F90EB
:107DE0007F906F905F904F903F902F900895FC018F
:107DF0002491222341F03091C00035FFFCCF209325
:107E0000C6000196F4CF22E030E087EC9DE00C94B0
:107E1000F08EFC012491222341F03091C00035FF07
:107E2000FCCF2093C6000196F4CF2AE030E087EC27
:107E30009DE00C94468E2091820830918308243076
:107E400031050CF06AC0409184085091850860E6C5
:107E5000649F9001659F300D1124BC01C9018457B6
:107E6000974F0E9450BAECEBFEE08491882341F0DA
:107E70009091C00095FFFCCF8093C6003196F5CF5E
:107E8000E2E7FEE08491882341F09091C00095FFE5
:107E9000FCCF8093C6003196F5CF809184089091F5
:107EA000850820E6289FF001299FF00D1124E45752
:107EB000F74F8191882339F09091C00095FFFCCF56
:107EC0008093C600F6CFE0E7FEE08491882341F07E
:107ED0009091C00095FFFCCF8093C6003196F5CFFE
:107EE0008091C00085FFFCCF8AE08093C60080911E
:107EF000840890918508019664E070E00E9484B641
:107F000090938508809384088091820890918308DB
:107F100001969093830880938208089520918208A7
:107F200030918308243031050CF06AC040918408F8
:107F30005091850860E6649F9001659F300D112483
:107F4000BC01C9018457974F0E94B9B9ECEBFEE020
:107F50008491882341F09091C00095FFFCCF8093DD
:107F6000C6003196F5CFE5E6FEE08491882341F026
:107F70009091C00095FFFCCF8093C6003196F5CF5D
:107F8000809184089091850820E6289FF001299F20
:107F9000F00D1124E457F74F8191882339F0909127
:107FA000C00095FFFCCF8093C600F6CFE3E6FEE06D
:107FB0008491882341F09091C00095FFFCCF80937D
:107FC000C6003196F5CF8091C00085FFFCCF8AE0D6
:107FD0008093C6008091840890918508019664E0A2
:107FE00070E00E9484B69093850880938408809105
:107FF0008208909183080196909383088093820869
:1080000008959B9AA3980895FCDF40E052EC61E04C
:1080100070E087EC9DE00E94FE8CEDE5FEE084912F
:10802000882341F09091C00095FFFCCF8093C6005B
:108030003196F5CF8091C00085FFFCCF8AE0809318
:10804000C6008CEB9EE0FC012491222341F030918C
:10805000C00035FFFCCF2093C6003196F5CF24B782
:1080600020FF14C0E5E5FEE03491332341F0409158
:10807000C00045FFFCCF3093C6003196F5CF30915C
:10808000C00035FFFCCF3AE03093C60021FF14C09A
:10809000E5E4FEE03491332341F04091C00045FF18
:1080A000FCCF3093C6003196F5CF3091C00035FF3C
:1080B000FCCF3AE03093C60022FF14C0E4E3FEE0B8
:1080C0003491332341F04091C00045FFFCCF309301
:1080D000C6003196F5CF3091C00035FFFCCF3AE0B5
:1080E0003093C60023FF14C0E4E2FEE03491332352
:1080F00041F04091C00045FFFCCF3093C60031965F
:10810000F5CF3091C00035FFFCCF3AE03093C60088
:1081100025FF14C0E4E1FEE02491222341F03091D8
:10812000C00035FFFCCF2093C6003196F5CF2091DB
:10813000C00025FFFCCF2AE02093C60014BEEDE06E
:10814000FEE02491222341F03091C00035FFFCCFA6
:108150002093C6003196F5CFE7E0FEE0249122237C
:1081600041F03091C00035FFFCCF2093C60031961E
:10817000F5CF2091C00025FFFCCF2AE02093C60058
:10818000FC012491ECEBFEE0222349F03091C00089
:1081900035FFFCCF2093C60031962491F5CFE7EF51
:1081A000FDE02491222341F03091C00035FFFCCF47
:1081B0002093C6003196F5CFE2EEFDE02491222314
:1081C00041F03091C00035FFFCCF2093C6003196BE
:1081D000F5CFE6EDFDE02491222341F03091C0007F
:1081E00035FFFCCF2093C6003196F5CFEFEBFDE0D5
:1081F0002491222341F03091C00035FFFCCF209321
:10820000C6003196F5CF2091C00025FFFCCF2AE0B3
:108210002093C600E4EBFDE02491222341F030914D
:10822000C00035FFFCCF2093C6003196F5CFE8EAB9
:10823000FDE02491222341F03091C00035FFFCCFB6
:108240002093C6003196F5CF2091C00025FFFCCFCA
:108250002AE02093C600FC018491ECEBFEE0882329
:1082600049F09091C00095FFFCCF8093C6003196F5
:108270008491F5CFE9E9FDE08491882341F0909164
:10828000C00095FFFCCF8093C6003196F5CF0E94C9
:10829000719A4AE050E0BC0187EC9DE00E941A8E82
:1082A000E2E8FDE08491882341F09091C00095FFC1
:1082B000FCCF8093C6003196F5CF4AE050E060EDE8
:1082C00074E087EC9DE00E941A8E8091C00085FFCB
:1082D000FCCF8AE08093C60010928808109289082B
:1082E00010928A0810928B080E94218B0E94F386BC
:1082F0000E9450210E94409E0E945F990E94AF7789
:10830000FFEF23ED80E3F15020408040E1F700C013
:108310000000089580917C0890917D0860E070E0F5
:1083200001960C9410B780917C0890917D084AE0EA
:1083300050E060E070E001960C9478B8682F7727E1
:1083400067FD7095209186083091870840E6429F2E
:10835000C001439F900D11248457974F0E943CBA4F
:1083600090937D0880937C0821E0892B09F420E01C
:10837000822F08950E944AAD60937808709379081F
:1083800080937A0890937B0808950E944AAD609389
:1083900078087093790880937A0890937B08E0912D
:1083A0008608F0918708E857F74F8081811114C043
:1083B000EDE7F9E08491882341F09091C00095FFAA
:1083C000FCCF8093C6003196F5CF8091C00085FF29
:1083D000FCCF8AE08093C600089587EC9DE00E9460
:1083E000508DE0E8F9E08491882341F09091C0003D
:1083F00095FFFCCF8093C6003196F5CF4091110ACE
:108400005091120A6091130A7091140A4F5F5F4FE6
:108410006F4F7F4F2AE030E087EC9DE00E94EF8DA8
:108420008091C00085FFFCCF8AE08093C600ADCF6D
:108430008F929F92AF92BF92CF92DF92EF92FF9274
:108440000F931F93CF93DF9334EDE32E34E0F32E9D
:1084500002E61AE0CDE2DAE047E7C42E4AE0D42E85
:10846000F70181917F016ADF882311F153DF4B010E
:108470005C01F6018081811103C060910C0A01C08A
:1084800061E070E080E090E00E945BB3F801208141
:108490003181428153810E948EB59B01AC01C5019F
:1084A000B4010E94E0B1688379838A839B8309C009
:1084B000F80180819181A281B38188839983AA8305
:1084C000BB830C5F1F4F2496FFEFCF1ADF0A88EDA6
:1084D000E81684E0F80621F686E430DF8823D1F040
:1084E00019DF6B017C0160931D0A70931E0A809353
:1084F0001F0A9093200A20E030E0A9010E94BCB43A
:10850000181644F4C0922102D0922202E092230273
:10851000F0922402DF91CF911F910F91FF90EF9085
:10852000DF90CF90BF90AF909F908F90089580DFA5
:1085300089E404DF882351F0EDDE6093210A709313
:10854000220A8093230A9093240A08C01092210AD9
:108550001092220A1092230A1092240A8AE4EEDE74
:10856000882351F0D7DE6093250A7093260A809302
:10857000270A9093280A08951092250A1092260A35
:108580001092270A1092280A0895CF92DF92EF9254
:10859000FF92CF93DF93EC01C0904302D09044024E
:1085A000E0904502F0904602A7019601688179812A
:1085B0008A819B810E94B9B287FF04C0C882D98298
:1085C000EA82FB82C0904702D0904802E0904902C4
:1085D000F0904A02A70196016C817D818E819F8176
:1085E0000E94B9B287FF04C0CC82DD82EE82FF8296
:1085F00020E030E0A90160914B0270914C02809123
:108600004D0290914E020E94E0B16B017C019B01F2
:10861000AC01688579858A859B850E94B9B287FF00
:1086200004C0C886D986EA86FB86C0903702D090FF
:108630003802E0903902F0903A02A7019601688171
:1086400079818A819B810E94BCB4181624F4C88267
:10865000D982EA82FB82C0903B02D0903C02E0903B
:108660003D02F0903E02A70196016C817D818E81D2
:108670009F810E94BCB4181624F4CC82DD82EE8265
:10868000FF82C0903F02D0904002E0904102F09003
:108690004202A7019601688579858A859B850E949B
:1086A000BCB4181624F4C886D986EA86FB86DF9106
:1086B000CF91FF90EF90DF90CF900895CF92DF920F
:1086C000EF92FF920F931F938DE29AE05EDF0E947C
:1086D0004AAD609378087093790880937A089093F4
:1086E0007B0820912D0A30912E0A40912F0A50913B
:1086F000300A6091620A7091630A8091640A9091D5
:10870000650A0E94B9B2811179C02091310A309175
:10871000320A4091330A5091340A6091660A70918E
:10872000670A8091680A9091690A0E94B9B2811122
:1087300065C020E030E040E752E460912102709192
:10874000220280912302909124020E94C0B25EE432
:10875000C52E5AE0D52E7B018C0129E33AE045E392
:108760005AE061E37AE08DE29AE00E94909E809167
:108770002D0A90912E0AA0912F0AB091300A809371
:10878000620A9093630AA093640AB093650A809189
:10879000310A9091320AA091330AB091340A809341
:1087A000660A9093670AA093680AB093690A809159
:1087B000350A9091360AA091370AB091380A809311
:1087C0006A0A90936B0AA0936C0AB0936D0A809129
:1087D000390A90913A0AA0913B0AB0913C0A8093E1
:1087E0006E0A90936F0AA093700AB093710A1F915A
:1087F0000F91FF90EF90DF90CF90089560915D0210
:1088000070915E02882777FD8095982F0E945BB358
:1088100020912102309122024091230250912402A2
:108820000E948EB520E030E040E752E40E94C0B2E2
:1088300020E030E048EC52E488CFCF92DF92EF9214
:10884000FF92CF93C62FE0914E0AF0E0882309F4FF
:10885000C2C0DF01A65BB54F8C91811196C180919A
:10886000620A9091630AA091640AB091650A8093AC
:108870002D0A90932E0AA0932F0AB093300A80916C
:10888000660A9091670AA091680AB091690A80937C
:10889000310A9093320AA093330AB093340A80913C
:1088A0006A0A90916B0AA0916C0AB0916D0A80934C
:1088B000350A9093360AA093370AB093380AC090CD
:1088C0006E0AD0906F0AE090700AF090710AC09220
:1088D000390AD0923A0AE0923B0AF0923C0AEE0F33
:1088E000FF1FEE0FFF1FE15BFD4F208131814281B1
:1088F0005381CC2349F060912F0270913002809116
:1089000031029091320208C06091330270913402BA
:1089100080913502909136020E94C0B29B01AC0159
:10892000C701B6010E94E0B160936E0A70936F0AAE
:108930008093700A9093710A8EE69AE00E94FCA8D8
:10894000C0902102D0902202E0902302F0902402F5
:1089500020E030E040E752E460912B0270912C025D
:1089600080912D0290912E020E948EB5609321027B
:10897000709322028093230290932402E0914E0A86
:10898000F0E0E65BF54F81E0808398DE2091460AB7
:108990003091470A4091480A5091490A60916A0A09
:1089A00070916B0A80916C0A90916D0A0E94DFB100
:1089B00060936A0A70936B0A80936C0A90936D0AB5
:1089C0002EE63AE04AE65AE066E67AE082E69AE087
:1089D0000E9457A8D1C0E65BF54F8081882309F437
:1089E000D4C08091620A9091630AA091640AB09108
:1089F000650A80932D0A90932E0AA0932F0AB093B4
:108A0000300A8091660A9091670AA091680AB09135
:108A1000690A8093310A9093320AA093330AB09383
:108A2000340A60916A0A70916B0A80916C0A909185
:108A30006D0A6093350A7093360A8093370A9093D3
:108A4000380AC0906E0AD0906F0AE090700AF090D9
:108A5000710AC092390AD0923A0AE0923B0AF09227
:108A60003C0A2091460A3091470A4091480A5091A9
:108A7000490A0E94E0B160936A0A70936B0A80937E
:108A80006C0A90936D0A2EE63AE04AE65AE066E6F2
:108A90007AE082E69AE00E9457A8F0904E0ACC2332
:108AA00089F020913E0A30913F0A4091400A50914E
:108AB000410A60912F0270913002809131029091B1
:108AC000320210C02091420A3091430A4091440A78
:108AD0005091450A609133027091340280913502C1
:108AE000909136020E94E0B124E0F29EF001112440
:108AF000E15BFD4F20813181428153810E94C0B2F0
:108B00009B01AC0160916E0A70916F0A8091700AAE
:108B10009091710A0E94DFB160936E0A70936F0AA0
:108B20008093700A9093710A8EE69AE00E94FCA8E6
:108B3000C0902102D0902202E0902302F090240203
:108B400020E030E040E752E4609127027091280273
:108B50008091290290912A020E948EB56093210291
:108B6000709322028093230290932402E0914E0A94
:108B7000F0E0E65BF54F1082A1DDC0922102D092B9
:108B80002202E0922302F0922402CF91FF90EF9014
:108B9000DF90CF900895AF92BF92CF92DF92EF9285
:108BA000FF920F931F93CF93DF93D82F2091250A25
:108BB0003091260A4091270A5091280A6091210A93
:108BC0007091220A8091230A9091240A0E94C9B4CC
:108BD000C62F172F082FF92E60915D0270915E024B
:108BE000882777FD8095982F0E945BB32091210202
:108BF0003091220240912302509124020E948EB5AE
:108C000020E030E040E752E40E94C0B220E030E0D3
:108C100048EC52E40E94C0B220914E0A2F93DF9399
:108C2000FF920F931F93CF935B016C0172E0E72ECD
:108C300001E020E041E25AE06DE27AE082E69AE06B
:108C40000E94092B80912D0A90912E0AA0912F0A43
:108C5000B091300A8093620A9093630AA093640AE9
:108C6000B093650A8091310A9091320AA091330A3B
:108C7000B091340A8093660A9093670AA093680AB9
:108C8000B093690A8091350A9091360AA091370A0B
:108C9000B091380A80936A0A90936B0AA0936C0A89
:108CA000B0936D0A8091390A90913A0AA0913B0ADB
:108CB000B0913C0A80936E0A90936F0AA093700A59
:108CC000B093710A0E944AAD609378087093790856
:108CD00080937A0890937B080F900F900F900F90DD
:108CE0000F900F90DF91CF911F910F91FF90EF9018
:108CF000DF90CF90BF90AF900895F8940E94F32139
:108D0000179A1092530A169A1092540A159A1092B2
:108D1000550A149A60E087E40E946AACE2ECFEE037
:108D20008491882341F09091C00095FFFCCF8093FF
:108D3000C6003196F5CFEEE5F9E08491882341F045
:108D40009091C00095FFFCCF8093C6003196F5CF7F
:108D50008091C00085FFFCCF8AE08093C60085E546
:108D600099E00E944C777894C6E0D0E02197209754
:108D700049F068EC70E080E090E00E9479AD0E94DC
:108D8000DB77F4CFF894FFCF2F923F924F925F9210
:108D90006F927F928F929F92AF92BF92CF92DF920B
:108DA000EF92FF920F931F93CF93DF93CDB7DEB770
:108DB0006E970FB6F894DEBF0FBECDBFB0E6BB2EE8
:108DC00014E0E12EF12C08E4C02E0CE0D02E8AE055
:108DD000A82E992493948091480E9091490E209149
:108DE0004A0E30914B0E821B930B8F779927892B5C
:108DF00009F41AC2809182089091830804970CF0BC
:108E000013C287EC9DE00E94348D809381082091ED
:108E10007F08309180088A3061F08D3051F08A33BC
:108E200021F490917E08992321F02F3531050CF41F
:108E30001DC12115310509F437C180918408909135
:108E40008508B89E3001B99E700C1124F301E20F21
:108E5000F31FE457F74F108220917E08211101C1C2
:108E600010927E08FC01E857F74F108283010457E7
:108E7000174F6EE470E0C8010E943CBA0097F1F110
:108E800090937D0880937C08801B910B860D971D25
:108E90004AE050E060E070E08357974F0E9478B856
:108EA0006093150A7093160A8093170A9093180A14
:108EB0004090110A5090120A6090130A7090140AA0
:108EC0002FEF421A520A620A720A00918408109126
:108ED0008508641575058605970509F4E8C0B09EF8
:108EE000C001B19E900D112464E67DE08457974F38
:108EF0000E94E7B9892B09F0DAC069C16AE270E023
:108F0000C8010E943CBA892B09F444C0E2ECFEE09F
:108F10008491882341F09091C00095FFFCCF80930D
:108F2000C6003196F5CFEEEBFCE08491882341F04A
:108F30009091C00095FFFCCF8093C6003196F5CF8D
:108F40004091110A5091120A6091130A7091140A0B
:108F50002AE030E087EC9DE00E94EF8D8091C00018
:108F600085FFFCCF8AE08093C600109280081092A3
:108F70007F08C0C28091150A9091160AA091170A25
:108F8000B091180A8093110A9093120AA093130AC1
:108F9000B093140A8091840890918508B89E80014E
:108FA000B99E100D1124C8018457974F3C0167E406
:108FB00070E00E943CBA009781F190937D08809305
:108FC0007C0886199709800F911F60E070E0835735
:108FD000974F0E9410B70E9428B364307105E8F4DF
:108FE00080916A088823C9F0F6018491E8E4FCE0E6
:108FF000882349F09091C00095FFFCCF8093C60074
:1090000031968491F5CF8091C00085FFFCCFA0926E
:10901000C6008EE39CE00E943F7700918408109187
:109020008508B09EC001B19E900D11246FE973E0D8
:109030008457974F0E9447BA892B09F45EDEC80116
:109040000196B7010E9484B69093850880938408A6
:109050008091820890918308019690938308809371
:1090600082081092800810927F08B5CE8B3311F4DD
:1090700090927E0890917E089111ADCE4091840827
:1090800050918508B9016F5F7F4F7093800860939E
:109090007F08B49EF001B59EF00D1124E20FF31F7E
:1090A000E457F74F808397CE10927E0823C2B09E7C
:1090B0003001B19E700C1124C3018457974F1C01DD
:1090C0006AE270E00E943CBA009789F5E2ECFEE0AB
:1090D0008491882341F09091C00095FFFCCF80934C
:1090E000C6003196F5CFE8EEFCE08491882341F08C
:1090F0009091C00095FFFCCF8093C6003196F5CFCC
:109100004091110A5091120A6091130A7091140A49
:109110002AE030E087EC9DE00E94EF8D8091C00056
:1091200085FFFCCF8AE08093C60057D91ECF20E090
:1091300010E0F301E20FF11DE457F74F30813A32AE
:1091400019F02F5F1327F5CF90937D0880937C084B
:1091500082199309860D971D60E070E08357974F41
:109160000E9410B70E9428B3212F30E0261737073E
:1091700009F400CFE2ECFEE08491882341F0909165
:10918000C00095FFFCCF8093C6003196F5CFE2E199
:10919000FDE08491882341F09091C00095FFFCCFC1
:1091A0008093C6003196F5CF4091110A5091120A72
:1091B0006091130A7091140A2AE030E087EC9DE078
:1091C0000E94EF8D8091C00085FFFCCFABCFE2EC19
:1091D000FEE08491882341F09091C00095FFFCCF80
:1091E0008093C6003196F5CFE1E3FDE084918823BA
:1091F00041F09091C00095FFFCCF8093C60031965E
:10920000F5CF4091110A5091120A6091130A7091A2
:10921000140A2AE030E087EC9DE00E94EF8D8091F7
:10922000C00085FFFCCF7ECF8091830A882309F49C
:1092300061C180917F0890918008892B09F05AC103
:109240008091820890918308892B11F4109268080C
:10925000F8EE2F2EF3E03F2E412C512CACE3CA2E1A
:10926000D12CE12CF12C8E010F5F1F4FE0E66E2E0A
:109270007724739440911E0D50911F0D6091200D25
:109280007091210D8091160D9091170DA091180DE0
:10929000B091190D481759076A077B0708F02AC1D2
:1092A000809182089091830804970CF023C18091EB
:1092B000680881111FC18091710C9091720CA0916E
:1092C000730CB091740C80931E0D90931F0DA0939E
:1092D000200DB093210D89E69CE00E948E12482F4C
:1092E000809381088A30B9F04D30A9F0433229F4D7
:1092F00020917E08222379F002C04A33C9F32091DD
:109300007F08309180082F3531052CF48F3FFFEF17
:109310009F0709F0D1C040911E0D50911F0D609123
:10932000200D7091210D8091160D9091170DA09137
:10933000180DB091190D481759076A077B0708F4F3
:1093400081C0EBE2FCE08491882341F09091C00061
:1093500095FFFCCF8093C6003196F5CF8091C00079
:1093600085FFFCCFFAE0F093C6000E944AAD6093FF
:109370006C0870936D0880936E0890936F088090CE
:10938000700890907108A0907208B09073086819E6
:1093900079098A099B09A20191010E9497B64901A6
:1093A0005A01CA01B901A70196010E9497B6CA01E4
:1093B000B901A70196010E9497B67F936F93C501EB
:1093C000B40120E13EE040E050E00E9497B63F93B8
:1093D0002F93A7E1BCE0BF93AF931F930F930E941D
:1093E00074BAECEBFEE084910FB6F894DEBF0FBECA
:1093F000CDBF882349F09091C00095FFFCCF8093AA
:10940000C60031968491F5CFF8018191882339F017
:109410009091C00095FFFCCF8093C600F6CF80915D
:10942000C00085FFFCCF3AE03093C600C8010E941F
:109430009A7381E89AE00E94B63A61E081E89AE086
:109440000E94E23480918108833211F4709268089E
:1094500020917F08309180082115310509F424CE30
:109460008091840890918508689EF001699EF00DB6
:109470001124E20FF31FE457F74F1082FC01E85765
:10948000F74F708220918208309183082F5F3F4F01
:109490003093830820938208019664E070E00E9474
:1094A00084B6909385088093840810927E08109269
:1094B000800810927F08DECE4B3311F470927E0844
:1094C00040917E084111D2CE409184085091850888
:1094D000B9016F5F7F4F7093800860937F08649E2F
:1094E000F001659EF00D1124E20FF31FE457F74FD2
:1094F0008083C0CE6E960FB6F894DEBF0FBECDBF90
:10950000DF91CF911F910F91FF90EF90DF90CF905F
:10951000BF90AF909F908F907F906F905F904F9093
:109520003F902F900895CF92DF92EF92FF920F938A
:109530001F93CF93C82F809182089091830803973F
:109540000CF422DC0E944AAD009174081091750859
:109550002091760830917708C0907808D0907908EB
:10956000E0907A08F0907B086C197D098E099F09BC
:10957000061717072807390728F4012B022B032B9E
:1095800009F0BBDB40911D0250911E0260911F0249
:1095900070912002452B462B472B19F10E944AADB2
:1095A000009178081091790820917A0830917B0811
:1095B000601B710B820B930B00911D0210911E0218
:1095C00020911F023091200206171707280739073C
:1095D00040F49091990E8091980E981302C0CC237C
:1095E00049F0CF911F910F91FF90EF90DF90CF90B6
:1095F0000C94749E179A1092530A169A1092540A59
:10960000159A1092550A149AECCF0E94F32180917A
:109610006A08811138C081E080936A088091110A3C
:109620009091120AA091130AB091140A80930D0A26
:1096300090930E0AA0930F0AB093100AE2ECFEE09A
:109640008491882341F09091C00095FFFCCF8093D6
:10965000C6003196F5CFEFEDF8E08491882341F014
:109660009091C00095FFFCCF8093C6003196F5CF56
:109670008091C00085FFFCCF8AE08093C60085ED15
:1096800098E00C943F77089580916A080895CF93ED
:10969000DF93EC0180914E0A80936B0884E50E9471
:1096A0009E41811102C080E075C00E948A410E94E3
:1096B0002DB360936B086623B1F3ECEBFEE084916D
:1096C000882341F09091C00095FFFCCF8093C600A5
:1096D0003196F5CFCD36D105B9F054F4C836D10561
:1096E000B1F0C936D10509F045C0E9EEF3E021C07B
:1096F000CA3DD10531F0CD3DD105E1F5E4EAF3E015
:1097000036C0EBEBF3E029C0E2EDF3E01CC0E0E093
:10971000F4E08191882371F19091C00095FFFCCF16
:109720008093C600F6CF9091C00095FFFCCF809348
:10973000C60081918111F7CF1DC09091C00095FFA7
:10974000FCCF8093C60081918111F7CF13C0909117
:10975000C00095FFFCCF8093C60081918111F7CFA7
:1097600009C09091C00095FFFCCF8093C600819105
:109770008111F7CF40E050E060916B0887EC9DE0ED
:109780000E94518E8091C00085FFFCCF8AE08093BB
:10979000C60081E0DF91CF910895CF92DF92EF92E2
:1097A000FF922091720A2223F1F020E030E040E0A5
:1097B0005FE30E948EB56B017C0120E030E0A901DF
:1097C0000E94B9B2882379F0A7019601C701B601BA
:1097D0000E948EB52BED3FE049E450E40E948EB527
:1097E0009B01AC0104C020E030E040E85FE360E0B2
:1097F00070E080E89FE30E94C0B2FF90EF90DF909E
:10980000CF90089560915302709154028091550257
:1098100090915602C2DF60934F0270935002809382
:1098200051029093520208953F924F925F926F922D
:109830007F928F929F92AF92BF92CF92DF92EF92E0
:10984000FF920F931F93CF93DF93CDB7DEB7E997C6
:109850000FB6F894DEBF0FBECDBF81E40E949E41DB
:109860008823B1F182E70E949E418823A9F0E6E2B5
:10987000F4E08191882339F09091C00095FFFCCFEE
:109880008093C600F6CF8091C00085FFFCCF8AE0B0
:109890008093C6000C94416286E70E949E41882313
:1098A00011F40C944162EDE2F4E08191882339F0E7
:1098B0009091C00095FFFCCF8093C600F6CF8091B9
:1098C000C00085FFFCCF8AE08093C6000C94416203
:1098D00087E40E949E41882309F462C20E948A4163
:1098E0000E9428B36A30710509F4AFC09CF462305D
:1098F000710509F44CC024F477FF25C00C94416233
:109900006330710509F44EC06430710509F455C027
:109910000C9441626A35710509F4EEC154F46B3060
:10992000710509F498C06C31710509F49AC00C9462
:1099300041626B35710509F4E3C16C35710509F4B9
:10994000E4C10C94416280916A0881110C944162D7
:109950000E94184280914B0A8823A9F088E50E9452
:109960009E41811110C089E50E949E4181110BC06A
:109970008AE50E949E41811106C085E40E949E41B5
:1099800081110C9444620E945E430C944162809168
:109990006A0881110C9441620E94974281E0FBD8D1
:1099A0000C94416280916A0881110C9441620E947A
:1099B000974280E0F0D80C9441628EE09CE00E94D7
:1099C0003F7780E50E949E41882339F00E948A41BA
:1099D0000E942DB34B015C0103C0812C912C5401DA
:1099E00083E50E949E41882361F00E948A4120E025
:1099F00030E04AE754E40E948EB50E942DB34B013B
:109A00005C010E94FD960E944AAD6B017C01C80C6E
:109A1000D91CEA1CFB1C0E944AAD60937808709325
:109A2000790880937A0890937B080E944AAD6C1560
:109A30007D058E059F0510F00C9441620E94201F49
:109A400080E071DD0E94DB77F0CF60E081E00E9472
:109A50001D440C94416260E080E00E941D440C941F
:109A600041628091210290912202A0912302B09143
:109A700024028093190A90931A0AA0931B0AB093A8
:109A80001C0A80915D0290915E029093760A809309
:109A9000750A84E690E090935E0280935D020E94D6
:109AA0004AAD609378087093790880937A08909310
:109AB0007B0881E00E94B18F8091620A9091630AD5
:109AC000A091640AB091650A80932D0A90932E0AA2
:109AD000A0932F0AB093300A8091660A9091670A8A
:109AE000A091680AB091690A8093310A9093320A72
:109AF000A093330AB093340A80916A0A90916B0A5A
:109B0000A0916C0AB0916D0A8093350A9093360A41
:109B1000A093370AB093380A80916E0A90916F0A29
:109B2000A091700AB091710A8093390A90933A0A11
:109B3000A0933B0AB0933C0A109221021092220299
:109B4000109223021092240288E50E949E418823ED
:109B500011F090E00AC089E50E949E418111F9CF81
:109B60008AE50E949E4191E09827909325029111E9
:109B70000C94736288E50E949E4181110C9473627B
:109B80008091250281110C94796289E50E949E41A1
:109B900081110C94796288E50E949E418823D1F05E
:109BA0000E949341672B682B692BA1F00E948A4188
:109BB0002091560A3091570A4091580A5091590AFB
:109BC0000E94E0B16093620A7093630A8093640A12
:109BD0009093650A89E50E949E418823D1F00E94F6
:109BE0009341672B682B692BA1F00E948A41209139
:109BF0005A0A30915B0A40915C0A50915D0A0E94BA
:109C0000E0B16093660A7093670A8093680A909344
:109C1000690A8091250281110C947F628AE50E9475
:109C20009E4181110C947F628AE50E949E418823A7
:109C3000D1F00E949341672B682B692BA1F00E9401
:109C40008A4120915E0A30915F0A4091600A5091EA
:109C5000610A0E94E0B160936A0A70936B0A809374
:109C60006C0A90936D0A2EE63AE04AE65AE066E600
:109C70007AE082E69AE00E9457A880E00E94B18FC5
:109C80008091190A90911A0AA0911B0AB0911C0A9E
:109C90008093210290932202A0932302B093240286
:109CA0008091750A9091760A90935E0280935D028E
:109CB0000E944AAD609378087093790880937A087F
:109CC00090937B080E94AA8F8091830A882311F4C5
:109CD0000C9441626FE77AE089EF9FE00E94D370B5
:109CE00080917F0A9091800A892B11F40C94416233
:109CF0000E947E790C94416210920C0A0C9441628D
:109D000081E080930C0A0C94416285E40E949E419C
:109D1000811102C00E94FD9654EDC52E54E0D52E4F
:109D200066E5E62E6AE0F62E02E61AE0B12CF601B0
:109D300081916F010E949E41882339F1F3E0BF12A7
:109D40000CC00E948A41F8016083718382839383EF
:109D50008EE69AE00E94FCA818C00E948A41F70192
:109D600020813181428153810E94E0B1F8016083FA
:109D70007183828393832EE63AE04AE65AE066E6F0
:109D80007AE082E69AE00E9457A8B394F4E0EF0EDE
:109D9000F11C0C5F1F4F24E0B212C9CF0C9441623A
:109DA0008DE40E949E41882311F40C9470610E94FE
:109DB0008A410E9428B36537710511F40C943B5712
:109DC0000CF0A6C06032710509F4F0C20CF056C068
:109DD0006731710509F445C254F56231710509F422
:109DE00069C7BCF477FF02C00C9441626230710510
:109DF0000CF461C16131710511F00C94416281ED87
:109E00009BE00E943F7717981698159814980C9429
:109E100041626531710509F418C20CF01CC264314D
:109E2000710511F00C944162E1ECFBE0EAC16B3189
:109E3000710509F442C2B4F46931710509F429C20B
:109E40000CF02DC281E89AE00E94E4310E944AADF4
:109E500060937008709371088093720890937308F0
:109E60000C9441626E31710509F462C20CF03AC380
:109E70006C31710509F427C20C9441626C3571058F
:109E800009F46BC7ECF46235710509F40AC764F490
:109E90006035710509F4DBC60CF0E6C66A3271055F
:109EA00009F47EC30C9441626435710509F402C75C
:109EB0000CF4FBC66535710509F434C70C94416296
:109EC0006B36710509F4BDC664F46936710509F491
:109ED000DEC30CF086C66836710509F4A8C30C947D
:109EE00041626037710509F4BFC334F46D36710502
:109EF00009F4DAC40C9441626237710509F4CFC7E2
:109F00006337710511F00C944162EFE3FAE0AEC7DC
:109F10006D3D710511F40C94435B0CF04DC06B3C2E
:109F2000710511F40C94BF5944F56C38710509F4AE
:109F30009DC39CF46837710511F40C942F58693750
:109F4000710511F40C9434586737710511F00C94B5
:109F50004162E4E3F4E00C943F58683C710511F46D
:109F60000C942959693C710511F40C949E596E3B6F
:109F7000710511F00C94416221C56F3C710511F41B
:109F80000C94795A54F46D3C710511F40C94FE59FB
:109F900014F40C94DC590C945C5A613D710511F475
:109FA0000C94D45A14F40C94AE5A6C3D710511F40F
:109FB0000C94345B0C944162603931E0730711F406
:109FC0000C94065D54F56E3291E0790711F40C940F
:109FD000C05C84F46C32F1E07F0711F40C94C45B34
:109FE00014F00C94FA5B623E710511F40C94695BF9
:109FF0000C9441626E3531E0730711F40C94DD600E
:10A000006F3581E0780711F40C9414616F32714060
:10A0100011F00C9441620C94CE5C6835E2E07E074E
:10A0200011F40C94E45DBCF4663F21E0720711F476
:10A030000C94095D673F31E0730711F40C940C5DDB
:10A04000653F714011F00C9441620E94218B0E9487
:10A05000F3860C9441626B3893E0790711F40C9409
:10A06000B7603CF46335734011F40C940F5D0C94AD
:10A070004162603A23E0720709F401C2673E73400F
:10A0800011F00C94416210926A080E9452778091FC
:10A090000D0A90910E0AA0910F0AB091100A8093B8
:10A0A000110A9093120AA093130AB093140A0E9403
:10A0B000ED410C94416200917C0810917D080E5F87
:10A0C0001F4F80E50E949E41882379F00E948A41BB
:10A0D0000E942DB36B017C01BB24B3946115710503
:10A0E0008105910531F4B12C04C0B12CC12CD12CC7
:10A0F000760183E50E949E41882399F00E948A415F
:10A1000020E030E04AE754E40E948EB50E942DB36F
:10A110006B017C01AA24A394611571058105910549
:10A1200009F4A12C6AE270E0C8010E943CBA0097D1
:10A1300011F0FC011082F801CF0121912032E1F3EE
:10A14000B11007C0A11005C0222319F00E949A7314
:10A1500004C08DEF9BE00E943F7781E00E947A73FC
:10A160000E94FD960E944AAD60937808709379082A
:10A1700080937A0890937B08C114D104E104F10420
:10A18000A9F00E944AAD4B015C018C0C9D1CAE1CD9
:10A19000BF1C0E944AAD681579058A059B05B8F475
:10A1A0000E94AF78811113C00C9485620E94AD7833
:10A1B000882311F40C9441620E94AF7881110AC087
:10A1C0000E94201F80E0AFD90E94DB77F5CF80E0AE
:10A1D0000E947A738091830A882331F08EEE9BE08F
:10A1E0000E943F770C9441628AED9BE00E943F778A
:10A1F0000C9441629091C00095FFFCCF8093C60003
:10A20000319684918111F6CF8091C00085FFFCCFFB
:10A210008AE08093C60081E89AE00E94C030E3EBB8
:10A22000FBE08491882341F09091C00095FFFCCF22
:10A230008093C6003196F5CF8091C00085FFFCCF9A
:10A240008AE08093C6000C94416281E89AE00E9403
:10A2500015310C94416281E89AE00E94E0310C943F
:10A26000416200917C0810917D080C5F1F4F6AE2EB
:10A2700070E0C8010E943CBA009711F0FC01108206
:10A2800021E041E0B80181E89AE00E9447360C9451
:10A29000416281E89AE00E94EB310C944162809126
:10A2A000840A882311F40C94416283E50E949E4144
:10A2B00081110C948E620C94416281E89AE00E94B4
:10A2C0008F330C94416280917C0890917D086AE202
:10A2D00070E004960E943CBA8C010097D9F020915E
:10A2E00086083091870840E6429FC001439F900D49
:10A2F00011246EE470E08457974F0E943CBA60E2EC
:10A3000070E00E943CBA019690937D0880937C088F
:10A31000F801108260917C0870917D086C5F7F4F1E
:10A3200021E040E081E89AE00E9447360C944162C7
:10A330008091840A882311F40C94416260E081E8E2
:10A340009AE00E94D83580917C0890917D086AE25D
:10A3500070E004960E943CBA8C010097D9F02091DD
:10A3600086083091870840E6429FC001439F900DC8
:10A3700011246EE470E08457974F0E943CBA60E26B
:10A3800070E00E943CBA019690937D0880937C080F
:10A39000F801108260917C0870917D086C5F7F4F9E
:10A3A00081E89AE00E944F320C9441628091830AC6
:10A3B00081110E94FD9600917C0810917D080C5F30
:10A3C0001F4F6AE270E0C8010E943CBA7C0161E262
:10A3D00070E0C8010E943CBA009719F08C010F5F31
:10A3E0001F4FE114F10411F0F701108280E50E9483
:10A3F0009E41F82E20917C0830917D0802171307AA
:10A4000008F4F12C8091840A882311F40C944162A1
:10A4100021E02F2541E0B80181E89AE00E9447360B
:10A4200083E50E949E418823B9F020917C083091F9
:10A430007D082017310780F40E949341AB01BC01D5
:10A4400040931E0D50931F0D6093200D7093210DAE
:10A4500089E69CE00E94571381E89AE00E94E4316B
:10A46000F1100C9441620E944AAD609370087093A1
:10A47000710880937208909373080C9441628091E4
:10A480007C0890917D086AE270E005960E943CBAD3
:10A490008C010097D9F0209186083091870840E61A
:10A4A000429FC001439F900D11246EE470E08457D9
:10A4B000974F0E943CBA60E270E00E943CBA01965D
:10A4C00090937D0880937C08F801108260917C084D
:10A4D00070917D086B5F7F4F81E89AE00E9471392F
:10A4E0000C9441620E944AAD60936C0870936D08B1
:10A4F00080936E0890936F08009170081091710816
:10A500002091720830917308601B710B820B930BC2
:10A5100028EE33E040E050E00E9497B6CA01B9014E
:10A520002CE330E040E050E00E9497B67F936F93B9
:10A530003F932F9384EA9BE09F938F93CE010196E4
:10A540009F938F930E9474BAECEBFEE084910FB658
:10A55000F894DEBF0FBECDBF882349F09091C000B4
:10A5600095FFFCCF8093C60031968491F5CFFE0114
:10A5700031968191882339F09091C00095FFFCCFEE
:10A580008093C600F6CF8091C00085FFFCCF8AE0A3
:10A590008093C600CE0101960E949A730C9441628A
:10A5A00083E50E949E41882311F40C9441620E942D
:10A5B0008A410E9428B3F62EE72E862F9E2D8C010D
:10A5C00080E50E949E41882331F00F3F110509F07C
:10A5D00010F40C949F620DE010E0ECE9F4E081913E
:10A5E00091918017910711F40C94416234E0E43D9D
:10A5F000F307A9F70630110539F48F2D9E2D90939E
:10A600004D0A80934C0A04C017FF02C00C944162AB
:10A6100061E0802F0E946AAC6F2D802F0E94A3AC56
:10A620006F2D7E2D802F0E9460AB0C94416288E6D6
:10A6300090E02DD881110C94416283E50E949E41E7
:10A64000882371F000916B080E948A4110E0000F8E
:10A65000111F0A59174F0E9428B3F80171836083B4
:10A660000E94F2210C9441620E947D4683E50E9483
:10A670009E41882311F40C9441620E948A410E94F9
:10A6800028B370936508609364080C94416289E66E
:10A6900090E00E94474B81110C944162EEE9FBE08F
:10A6A0008491882341F09091C00095FFFCCF809366
:10A6B000C6003196F5CFE0916B0824E0E29FF001EF
:10A6C0001124E25AF74F408151816281738121E068
:10A6D00030E087EC9DE00E94F08EEBE9FBE0849196
:10A6E000882341F09091C00095FFFCCF8093C60075
:10A6F0003196F5CFE0916B08F0E0EE0FFF1FEA59BD
:10A70000F74F60817181882777FD8095982F0E948F
:10A710005BB3AB01BC0121E030E087EC9DE00E941F
:10A72000F08EE7E9FBE08491882341F09091C0002E
:10A7300095FFFCCF8093C6003196F5CF4091580825
:10A740005091590860915A0870915B0821E030E0FF
:10A7500087EC9DE00E94F08EE4E9FBE08491882381
:10A7600041F09091C00095FFFCCF8093C6003196D8
:10A77000F5CF6091640870916508882777FD809512
:10A78000982F0E945BB3AB01BC0121E030E087EC65
:10A790009DE00E94F08EE1E9FBE08491882341F086
:10A7A0009091C00095FFFCCF8093C6003196F5CF05
:10A7B0004AE050E060E070E087EC9DE00E941A8E75
:10A7C000EFE8FBE08491882341F09091C00095FF71
:10A7D000FCCF8093C6003196F5CF40915E08509132
:10A7E0005F08609160087091610821E030E087ECBB
:10A7F0009DE00E94F08EECE8FBE08491882341F01C
:10A800009091C00095FFFCCF8093C6003196F5CFA4
:10A810006091660870916708882777FD8095982F6A
:10A820000E945BB3AB01BC0121E030E087EC9DE00E
:10A830000E94F08EE8E8FBE08491882341F090913B
:10A84000C00095FFFCCF8093C6003196F5CF809174
:10A850006B0890E00E94EA1E4AE050E0BC0187ECE1
:10A860009DE00E941A8EE3E8FBE08491882341F08A
:10A870009091C00095FFFCCF8093C6003196F5CF34
:10A880008FEF9FEF0E94EA1E4AE050E0BC0187EC88
:10A890009DE00E941A8E8091C00085FFFCCF8AE067
:10A8A0008093C6000C94FD638DE690E00E94474BB8
:10A8B00081110C94416286E79BE00E943F7783E51B
:10A8C0000E949E41882391F000916B080E948A416A
:10A8D00010E0000F111F0A59174F0E9428B3F8010A
:10A8E0007183608381E080931C0215C082E50E9421
:10A8F0009E41882381F000916B080E948A4110E0FC
:10A90000000F111F0A59174F0E9428B3F8017183D5
:10A91000608310921C020E94F2210E944AAD4B01FA
:10A920005C0100916B0810E0F801EE0FFF1FEA597F
:10A93000F74F60817181882777FD8095982F0E945D
:10A940005BB3F801EE0FFF1FEE0FFF1FE25AF74F48
:10A9500011E020813181428153810E94BCB41816DC
:10A960000CF010E01093690810923D0ACC24CA94B0
:10A97000DC2C760148EE442E43E0542E612C712CE1
:10A980005AE0352E80913D0A81110C94BA63FFEF95
:10A99000CF16DF06EF06FF0611F40C94A662F7FE51
:10A9A00002C00C94BA630E944AAD6C197D09683BE1
:10A9B0007B4010F40C94A6620C94BA638CE49BE088
:10A9C0000E943F7783E50E949E41882361F00E94A8
:10A9D0008A410E9428B3709365086093640881E0FF
:10A9E00080931C020FC082E50E949E41882351F093
:10A9F0000E948A410E9428B370936508609364089E
:10AA000010921C020E944AAD4B015C0110923D0A5B
:10AA10006091640870916508882777FD8095982F6C
:10AA20000E945BB311E02091580830915908409181
:10AA30005A0850915B080E94BCB418160CF010E044
:10AA40001093690809E41BE0E5E4EE2EEBE0FE2E2E
:10AA5000F1E4CF2EFBE0DF2EAAE07A2E8091690888
:10AA60006091640870916508882309F48BC0809117
:10AA70003D0A811187C0882777FD8095982F0E9415
:10AA80005BB3209158083091590840915A08509171
:10AA90005B080E94BCB418160CF08BC00E944AAD33
:10AAA000681979098A099B09693E734081059105F6
:10AAB00008F460C0E0914E0A84E0E89FF0011124A0
:10AAC000E25AF74F4081518162817381F80184918C
:10AAD000E9E4FBE0882349F09091C00095FFFCCFAA
:10AAE0008093C60031968491F5CF22E030E087EC68
:10AAF0009DE00E94F08EF7018491E5E4FBE088235D
:10AB000049F09091C00095FFFCCF8093C60031962C
:10AB10008491F5CF60914E0A70E04AE050E087ECF6
:10AB20009DE00E941A8EF6018491E1E4FBE0882307
:10AB300049F09091C00095FFFCCF8093C6003196FC
:10AB40008491F5CF409158085091590860915A0866
:10AB500070915B0821E030E087EC9DE00E94F08E70
:10AB60008091C00085FFFCCF7092C6000E944AAD64
:10AB70004B015C010E94201F80E00E94934A0E94CA
:10AB8000DB776CCF882777FD8095982F0E945BB389
:10AB9000209158083091590840915A0850915B080B
:10ABA0000E94B9B287FF05C080911C02882309F476
:10ABB00075CF89E39BE00E943F778091830A8823C9
:10ABC00021F08AE893E00E949A730E944AAD609354
:10ABD00078087093790880937A0890937B080C9496
:10ABE000416283E50E949E41882319F10E948A41B7
:10ABF00020E030E0A9010E94B9B287FD0FC00E9499
:10AC00008A4120E030E04FE753E40E94BCB41816BC
:10AC100044F00E948A410E9428B305C060E070E0C1
:10AC200002C06FEF70E070934D0A60934C0A0C9471
:10AC300041628FEF90E090934D0A80934C0A0C9400
:10AC4000416210924D0A10924C0A0C9441629B9AF8
:10AC5000A39881E08093260285E29BE00E943F77E3
:10AC60000E94DB770C9441620E94F3210E94FD96C2
:10AC7000149A0E94679710924D0A10924C0A68EE3F
:10AC800073E080E090E00E9479AD9B9AA39A1092C5
:10AC9000260287E19BE00E943F770E94DB770C94BD
:10ACA000416210927A0A0C94416281E080937A0AA0
:10ACB0000C94416283E50E949E418823A1F00E948A
:10ACC0008A4120E030E04AE754E40E948EB50E94B9
:10ACD0002DB360931D0270931E0280931F02909308
:10ACE00020020C94416288E50E949E4181110C94DF
:10ACF000DB6389E50E949E4181110C94DB638AE548
:10AD00000E949E4181110C94DB6385E40E949E4168
:10AD100081110C94DB630E94FD96149A0E94679740
:10AD20000C94416283E50E949E41882311F40C94A7
:10AD300041620E948A4120E030E04AE754E40E94E8
:10AD40008EB50E942DB3609374087093750880933C
:10AD50007608909377080C94416224ED34E039AF83
:10AD600028AF0DEC13E16DED862E63E1962E71E9AF
:10AD7000A72E73E1B72E312CE8ADF9AD8191F9AF73
:10AD8000E8AF0E949E41882309F45BC0F3E03F12C4
:10AD900051C00E948A416B017C0120E030E040EA12
:10ADA00051E40E94B9B287FF3FC0A7019601F801A4
:10ADB00060817181828193810E94C0B22B013C012C
:10ADC0009B01AC016091A5137091A6138091A7130C
:10ADD0009091A8130E948EB56093A5137093A6134B
:10ADE0008093A7139093A813A3019201F4016081AB
:10ADF0007181828193810E948EB5F4016083718399
:10AE000082839383F50160817181828193810E94A5
:10AE100059B3A30192010E948EB50E942DB3F50192
:10AE20006083718382839383F801C082D182E2823E
:10AE3000F38207C00E948A41F80160837183828394
:10AE4000938333940C5F1F4FF4E08F0E911C24E02A
:10AE5000A20EB11C34E033128FCF0C94416290915A
:10AE6000C00095FFFCCF8093C6003196849181117C
:10AE7000F6CF0C94416200917C0810917D080B5F25
:10AE80001F4F6AE270E0C8010E943CBA009711F0BF
:10AE9000FC011082C8010E949A730C944162ECE399
:10AEA000FAE08491882341F09091C00095FFFCCF97
:10AEB0008093C6003196F5CF4091620A5091630AA3
:10AEC0006091640A7091650A22E030E087EC9DE0B1
:10AED0000E94F08EE8E3FAE08491882341F090919B
:10AEE000C00095FFFCCF8093C6003196F5CF40910E
:10AEF000660A5091670A6091680A7091690A22E0B7
:10AF000030E087EC9DE00E94F08EE4E3FAE084916B
:10AF1000882341F09091C00095FFFCCF8093C6003C
:10AF20003196F5CF40916A0A50916B0A60916C0A94
:10AF300070916D0A22E030E087EC9DE00E94F08E77
:10AF4000E0E3FAE08491882341F09091C00095FFFE
:10AF5000FCCF8093C6003196F5CF40916E0A509198
:10AF60006F0A6091700A7091710A22E030E087ECFC
:10AF70009DE00E94F08EE5E2FAE08491882341F0A2
:10AF80009091C00095FFFCCF8093C6003196F5CF1D
:10AF90000E9459970E945BB32091CD133091CE133C
:10AFA0004091CF135091D0130E94C0B2AB01BC01AD
:10AFB00022E030E087EC9DE00E94F08EE1E2FAE0D2
:10AFC0008491882341F09091C00095FFFCCF80933D
:10AFD000C6003196F5CF81E00E9459970E945BB37D
:10AFE0002091D1133091D2134091D3135091D413A7
:10AFF0000E94C0B2AB01BC0122E030E087EC9DE0D2
:10B000000E94F08EEDE1FAE08491882341F0909166
:10B01000C00095FFFCCF8093C6003196F5CF82E04B
:10B020000E9459970E945BB32091D5133091D6139B
:10B030004091D7135091D8130E94C0B2AB01BC010C
:10B0400022E030E087EC9DE00E94F08E8091C0000D
:10B0500085FFFCCF8AE08093C6000C94416280E0BB
:10B060000E94B18F0C94416281E00E94B18F0C94D8
:10B0700041629091C00095FFFCCF8093C600819102
:10B080008111F7CF8091C00085FFFCCF8AE08093CB
:10B09000C600E5E1FAE08491882341F09091C00078
:10B0A00095FFFCCF8093C6003196F5CF1E9B03C061
:10B0B000E7E1F4E009C0E1E2F4E006C09091C000ED
:10B0C00095FFFCCF8093C60081918111F7CF8091CD
:10B0D000C00085FFFCCF8AE08093C600EDE0FAE077
:10B0E0008491882341F09091C00095FFFCCF80931C
:10B0F000C6003196F5CF029903C0E7E1F4E009C03C
:10B10000E1E2F4E006C09091C00095FFFCCF80938F
:10B11000C60081918111F7CF8091C00085FFFCCFDF
:10B120008AE08093C600E5E0FAE08491882341F04C
:10B130009091C00095FFFCCF8093C6003196F5CF6B
:10B140001D9B03C0E7E1F4E009C0E1E2F4E006C0C2
:10B150009091C00095FFFCCF8093C6008191811132
:10B16000F7CF8091C00085FFFCCF8AE08093C600B6
:10B17000EDEFF9E08491882341F09091C00095FFB4
:10B18000FCCF8093C6003196F5CF019903C0E7E16B
:10B19000F4E009C0E1E2F4E006C09091C00095FF40
:10B1A000FCCF8093C60081918111F7CF8091C000C0
:10B1B00085FFFCCF8AE08093C600E5EFF9E084913B
:10B1C000882341F09091C00095FFFCCF8093C6008A
:10B1D0003196F5CF1C9B03C0E7E1F4E009C0E1E242
:10B1E000F4E006C09091C00095FFFCCF8093C600AC
:10B1F00081918111F7CF8091C00085FFFCCF8AE05B
:10B200008093C600EDEEF9E08491882341F090919F
:10B21000C00095FFFCCF8093C6003196F5CF3799DB
:10B2200003C0E7E1F4E009C0E1E2F4E006C0909178
:10B23000C00095FFFCCF8093C60081918111F7CFAC
:10B240008091C00085FFFCCF8AE08093C6000C94FB
:10B25000416280914E0A80936B0884E50E949E4172
:10B26000882319F10E948A410E942DB360936B08D4
:10B270006623D9F0ECEBFEE08491882341F09091B5
:10B28000C00095FFFCCF8093C6003196F5CFEDE46A
:10B29000F4E08191882311F40C9441629091C000F4
:10B2A00095FFFCCF8093C600F4CF84E40E949E41BA
:10B2B000882311F40C9441620E948A4120E030E01E
:10B2C000A9010E94B9B2811103C01092720A32C062
:10B2D00000916B0810E00E948A41F801EE0FFF1FF9
:10B2E000EE0FFF1FED5AFD4F6083718382839383BE
:10B2F000E0905302F09054020091550210915602D2
:10B3000020E030E0A901B701C8010E94B9B2811163
:10B3100004C0E12CF12C00E410E4C701D8018093B3
:10B32000530290935402A0935502B093560281E0C9
:10B330008093720A0E94024C0C94416204ED14E066
:10B340004DEBE42E43E1F42EF80181918F010E9430
:10B350009E41882349F00E948A410E942DB3F70143
:10B360006083718382839383F4E0EF0EF11C24E009
:10B37000083D120749F70E9429A90C94416204ED87
:10B3800014E03DEDE32E33E1F32EF80181918F01BE
:10B390000E949E41882339F00E948A41F701608310
:10B3A000718382839383F4E0EF0EF11C24E0083D67
:10B3B000120759F70C94416283E50E949E4188234D
:10B3C00051F00E948A416093B5137093B613809335
:10B3D000B7139093B81384E50E949E41882311F41B
:10B3E0000C9441620E948A416093B1137093B2132E
:10B3F0008093B3139093B4130C94416283E50E943D
:10B400009E41882351F00E948A416093B913709342
:10B41000BA138093BB139093BC1384E50E949E41A2
:10B42000882351F00E948A416093A1137093A21364
:10B430008093A3139093A41382E40E949E418823D7
:10B4400061F00E948A410E942DB36093ED137093C6
:10B45000EE138093EF139093F01388E50E949E41C2
:10B46000882351F00E948A416093AD137093AE130C
:10B470008093AF139093B0138AE50E949E41882376
:10B4800051F00E948A416093A9137093AA1380938C
:10B49000AB139093AC1385E40E949E41882309F47A
:10B4A000F0C70E948A416093A5137093A6138093FE
:10B4B000A7139093A813E5C704ED14E026E5E22E48
:10B4C0002AE0F22EF80181918F010E949E4188238B
:10B4D00039F00E948A41F7016083718382839383EC
:10B4E000F4E0EF0EF11C24E0073D120709F4C9C790
:10B4F000E9CF83E50E949E41882351F00E948A4152
:10B500006093330270933402809335029093360235
:10B5100086E40E949E41882381F00E948A4120E0B7
:10B5200030E040E752E40E94C0B260932B02709377
:10B530002C0280932D0290932E028AE50E949E4158
:10B54000882309F49EC70E948A416093460A70933B
:10B55000470A8093480A9093490A93C783E50E945B
:10B560009E41882351F00E948A416093420A709361
:10B57000430A8093440A9093450A86E40E949E41C0
:10B58000882309F47EC70E948A4120E030E040E72A
:10B5900052E40E94C0B26093270270932802809305
:10B5A000290290932A026DC783E50E949E41882359
:10B5B00009F467C70E948A410E9428B3611571058A
:10B5C00049F06130710559F481E080934B0A109283
:10B5D0004A0A57C710924B0A10924A0A52C7ECEB1C
:10B5E000FEE08491882341F09091C00095FFFCCF4C
:10B5F0008093C6003196F5CFEAEDF9E08491882377
:10B6000041F09091C00095FFFCCF8093C600319629
:10B61000F5CF809186089091870820E6289FF00159
:10B62000299FF00D1124E457F74F8191882339F0B9
:10B630009091C00095FFFCCF8093C600F6CFE8ED57
:10B64000F9E08491882341F09091C00095FFFCCFF0
:10B650008093C6003196F5CF8091C00085FFFCCF66
:10B660008AE08093C6000DC783E50E949E4188232F
:10B6700009F407C70E948A410E9428B370935E02B2
:10B6800060935D02FEC683E50E949E41882309F413
:10B69000F8C60E948A410E9428B36B017C0184E5B0
:10B6A0000E949E41882381F08DED90E00E94474BDF
:10B6B0008111E7C6E0916B08F0E0EE0FFF1FE75A3B
:10B6C000FD4FD182C082DDC6D0925C02C0925B0287
:10B6D000D8C680E50E949E41882309F4D2C60E9404
:10B6E0008A410E9428B3D62E062F172F83E50E9489
:10B6F0009E41882331F00E948A410E9428B37B0139
:10B7000003C0EE24EA94FE2CC7010196039708F0CB
:10B71000B8C6ECE9F4E0819191918017910709F4A2
:10B72000B0C634E0E43DF307B1F717FDAAC60E94A6
:10B73000FD96CD2C60E08D2D0E946AAC8FEFE8164F
:10B74000F80631F0EA94EF2871F000E010E00DC047
:10B750008D2D0E94D8AC31E020E0892B09F030E03B
:10B76000032F122F02C001E010E08C2D0E94D8ACF4
:10B770008017910709F485C60E94201F80E00E946F
:10B78000934A0E94DB77F1CF83E50E949E41882394
:10B7900031F00E948A410E9428B38B0102C00EE65C
:10B7A00010E080E50E949E41882331F00E948A418A
:10B7B0000E9428B3CB0102C088EE93E06C01EE2416
:10B7C000D7FCE094FE2C101611067CF420E030E04B
:10B7D000A901B8018EE40E9416AEC701B6010E940D
:10B7E00079AD8EE40E9427B14CC6C701B6010E9414
:10B7F00079AD47C680E50E949E41882351F00E94A2
:10B800008A41609318027093190280931A029093F0
:10B810001B0289E40E949E41882361F00E948A41B4
:10B820000E9465286093140270931502809316029B
:10B830009093170284E40E949E41882361F00E9445
:10B840008A410E94712860931002709311028093C4
:10B8500012029093130283E40E949E41882351F0C8
:10B860000E948A4160930C0270930D0280930E0235
:10B8700090930F020E94D31EE4E6F4E081918823A6
:10B8800039F09091C00095FFFCCF8093C600F6CFB1
:10B89000E7E6F4E08191882339F09091C00095FFAC
:10B8A000FCCF8093C600F6CF409118025091190248
:10B8B00060911A0270911B0222E030E087EC9DE05B
:10B8C0000E94F08EEBE6F4E08191882339F09091AC
:10B8D000C00095FFFCCF8093C600F6CF60911402A4
:10B8E0007091150280911602909117020E946B28A8
:10B8F000AB01BC0122E030E087EC9DE00E94F08EBD
:10B90000EFE6F4E08191882339F09091C00095FF33
:10B91000FCCF8093C600F6CF6091100270911102A7
:10B9200080911202909113020E947728AB01BC0112
:10B9300022E030E087EC9DE00E94F08EE3E7F4E047
:10B940008191882339F09091C00095FFFCCF8093BE
:10B95000C600F6CF40910C0250910D0260910E028C
:10B9600070910F0222E030E087EC9DE00E94F08EA3
:10B970008091C00085FFFCCF8AE08093C60081C51E
:10B9800083E50E949E41882319F00E948A4103C0EA
:10B9900060E070E0CB010E9420A973C585E40E949D
:10B9A0009E41882341F00E948A410E9428B38B0166
:10B9B00077FF03C009C000E010E0C12CD12CB6E134
:10B9C000EB2EB3E4FB2E06C0C12CD12CACE8EA2E42
:10B9D000A2E4FA2E83E50E949E41882321F00E9472
:10B9E0008A416B017C0183E40E949E41882331F0EF
:10B9F0000E948A410E9428B39B0102C025E030E0EA
:10BA0000A801C701B6010E9406223BC50E94FD960F
:10BA100038C50E94218B35C50E94F38632C58AE560
:10BA20000E949E41882309F497C00E948A416B01BD
:10BA30007C0120E030E040E751EC0E94BCB487FD7F
:10BA40003FC020E030E040EA50ECC701B6010E9460
:10BA5000B9B21816ACF1F7FAF094F7F8F094C09276
:10BA60004F0AD092500AE092510AF092520AECEB3F
:10BA7000FEE08491882341F09091C00095FFFCCFB7
:10BA80008093C6003196F5CFECECF9E084918823E1
:10BA900041F09091C00095FFFCCF8093C600319695
:10BAA000F5CF8091C00085FFFCCF8AE08093C6006F
:10BAB0008091C00085FFFCCF8AE08093C600E1C47E
:10BAC000ECEBFEE08491882341F09091C00095FF5B
:10BAD000FCCF8093C6003196F5CFE3ECF9E084917A
:10BAE000882341F09091C00095FFFCCF8093C60061
:10BAF0003196F5CFEBEBF9E08491882341F09091FA
:10BB0000C00095FFFCCF8093C6003196F5CF4AE088
:10BB100050E061EF7FEF87EC9DE00E941A8EE3EB2F
:10BB2000F9E08491882341F09091C00095FFFCCF0B
:10BB30008093C6003196F5CF4AE050E06BEF7FEF7F
:10BB400087EC9DE00E941A8E8091C00085FFFCCF9B
:10BB50008AE08093C60095C4ECEBFEE084918823D4
:10BB600041F09091C00095FFFCCF8093C6003196C4
:10BB7000F5CFE7EAF9E08491882341F09091C00085
:10BB800095FFFCCF8093C6003196F5CF8091C00021
:10BB900085FFFCCF8AE08093C60040914F0A509108
:10BBA000500A6091510A7091520A705822E030E0B8
:10BBB00087EC9DE00E94F08E8091C00085FFFCCF55
:10BBC0008AE08093C6005DC480915D0290915E0220
:10BBD0009093580280935702C090620AD090630AF3
:10BBE000E090640AF090650ACF8ED8A2E9A2FAA28A
:10BBF0000091660A1091670A2091680A3091690ADB
:10BC00000BA31CA32DA33EA340916A0A50916B0A7B
:10BC100060916C0A70916D0A4FA358A769A77AA723
:10BC200080916E0A90916F0AA091700AB091710A8A
:10BC30008BA79CA7ADA7BEA7C982DA82EB82FC8244
:10BC40000D831E832F83388749875A876B877C87AC
:10BC50008D879E87AF87B88B85E40E949E4188239D
:10BC600059F00E948A419B01AC016BA57CA58DA572
:10BC70009EA50E94E0B10AC020E030E040E050E420
:10BC80006BA57CA58DA59EA50E94DFB16BA77CA7A7
:10BC90008DA79EA7EEE4CE2EEAE0DE2EE12CF12C5D
:10BCA00008EC13E49E01255D3F4FAE01495D5F4FF7
:10BCB000BE016D5D7F4FCE014F960E94909E8AE53A
:10BCC0000E949E41882349F00E948A419B01AC0159
:10BCD0006FA178A589A59AA51EC020E030E040E0BC
:10BCE00050E46FA178A589A59AA50E94E0B16B01E7
:10BCF0007C016FA378A789A79AA720E030E040E2F3
:10BD000051E40E94B9B287FF0CC020E030E040E26D
:10BD100051E4C701B6010E94E0B16FA378A789A7DB
:10BD20009AA76EE4C62E6AE0D62EE12CF12C06E925
:10BD300013E49E01255D3F4FAE01495D5F4FBE019B
:10BD40006D5D7F4FCE014F960E94909E88E50E94C8
:10BD50009E41882379F00E948A419B01AC016F8D3E
:10BD600078A189A19AA10E94E0B16F8F78A389A3DD
:10BD70009AA308C080E090E0A3E5B3E48F8F98A376
:10BD8000A9A3BAA389E50E949E41882339F00E94A5
:10BD90008A416BA37CA38DA39EA304C01BA21CA2FB
:10BDA0001DA21EA24EE4C42E4AE0D42EE12CF12C9A
:10BDB0000CE812E49E01255D3F4FAE01495D5F4FE7
:10BDC000BE016D5D7F4FCE014F960E94909E8CE428
:10BDD0000E949E41882359F00E948A419B01AC0138
:10BDE0006BA57CA58DA59EA50E94E0B10AC020E0B0
:10BDF00030E040EA52E46BA57CA58DA59EA50E948B
:10BE0000DFB16BA77CA78DA79EA72EE4C22E2AE0E8
:10BE1000D22EE12CF12C08EC13E49E01255D3F4F5E
:10BE2000AE01495D5F4FBE016D5D7F4FCE014F9604
:10BE30000E94909E0E94FD96149A64E670E080E055
:10BE400090E00E9479AD0E941C7000E010E0F12C9F
:10BE50000E94AF7881111BC0F3940E94201F81E0E3
:10BE60000E94934AF110F4CF043FE1E01E0711F461
:10BE700000E010E06A9A0115110511F4729A04C0ED
:10BE80000431110509F472980F5F1F4FE1CF7298CA
:10BE900020E030E04CE852E46BA57CA58DA59EA582
:10BEA0000E94E0B16BA77CA78DA79EA71EE4C12EC0
:10BEB0001AE0D12EE12CF12C00EA11E49E01255D5F
:10BEC0003F4FAE01495D5F4FBE016D5D7F4FCE01BB
:10BED0004F960E94909E20E030E048E452E46BA52B
:10BEE0007CA58DA59EA50E94E0B16BA77CA78DA720
:10BEF0009EA7E12CF12C00E010E49E01255D3F4F50
:10BF0000AE01495D5F4FBE016D5D7F4FCE014F9623
:10BF10000E94909E1092740A1092730A0E9482707E
:10BF20008091730A9091740A019709F47CC0109271
:10BF3000740A1092730A0E94B5788091730A9091E6
:10BF4000740A8230910549F1039709F069C020E035
:10BF500030E048E452E46BA57CA58DA59EA50E9427
:10BF6000E0B16BA77CA78DA79EA77EE4C72E7AE0E1
:10BF7000D72EE12CF12C00E010E49E01255D3F4F0F
:10BF8000AE01495D5F4FBE016D5D7F4FCE014F96A3
:10BF90000E94909E0E944270C3CF20E030E04CE8A7
:10BFA00052E46BA57CA58DA59EA50E94E0B16BA770
:10BFB0007CA78DA79EA7FEE4CF2EFAE0DF2EE12C12
:10BFC000F12C00EA11E49E01255D3F4FAE01495D71
:10BFD0005F4FBE016D5D7F4FCE014F960E94909ED8
:10BFE00020E030E048E452E46BA57CA58DA59EA539
:10BFF0000E94E0B16BA77CA78DA79EA7E12CF12C36
:10C0000000E010E49E01255D3F4FAE01495D5F4FAA
:10C01000BE016D5D7F4FCE014F960E94909E7ECFF8
:10C020000E9435707DCF20E030E040EA50E46BA5FF
:10C030007CA58DA59EA50E94E0B16BA77CA78DA7CE
:10C040009EA79EE4C92E9AE0D92EE12CF12C00E0A7
:10C0500010E49E01255D3F4FAE01495D5F4FBE017B
:10C060006D5D7F4FCE014F960E94909EA801970173
:10C070006BA57CA58DA59EA50E94DFB16BA77CA7B3
:10C080008DA79EA7E12CF12C08EC13E49E01255D01
:10C090003F4FAE01495D5F4FBE016D5D7F4FCE01E9
:10C0A0004F960E94909EE12CF12C0CE812E49E0128
:10C0B000255D3F4FAE01495D5F4FBE016B5F7F4F16
:10C0C000CE0101960E94909EE12CF12C06E913E42A
:10C0D0009E01255D3F4FAE01475F5F4FBE016B5F25
:10C0E0007F4FCE0101960E94909E20E030E040E01C
:10C0F00050E46BA57CA58DA59EA50E94E0B16BA721
:10C100007CA78DA79EA7E12CF12C08EC13E49E01DF
:10C11000255D3F4FAE01475F5F4FBE016B5F7F4FB5
:10C12000CE0101960E94909ECE010D960E94FCA821
:10C13000809157029091580280935D0290935E0225
:10C140009F938F938EE999E09F938F938E01015D6A
:10C150001F4F1F930F930E9474BAC8010E941B3F88
:10C160000F900F900F900F900F900F908AC188E55D
:10C170000E949E41882339F00E948A410E9428B380
:10C1800080E00E9427988AE50E949E41882339F02A
:10C190000E948A410E9428B381E00E94279885E48A
:10C1A0000E949E41882309F46CC10E948A410E942A
:10C1B00028B382E00E94279864C183E50E949E41D3
:10C1C000811104C004ED14E0F12C10C010E00E94B5
:10C1D0008A410E942DB3812F0E94FD981F5F153068
:10C1E000B1F7F0CFF394F4E0FF1679F0F801819104
:10C1F0008F010E949E418823A9F30E948A410E94D8
:10C200002DB38F2D0E94FD98EDCF82E40E949E41B8
:10C21000882339F00E948A410E942DB384E00E9455
:10C22000FD980E94C3992DC183E50E949E418823F9
:10C2300009F453C00E948A410E9428B361307105FD
:10C2400041F06230710509F048C004ED14E0F12CB2
:10C2500025C004ED14E0F12CF80181918F010E94BA
:10C260009E41882341F00E948A410E9428B34FEFEB
:10C270008F2D0E94BF98F394F4E0FF12EDCF82E47B
:10C280000E949E41882349F10E948A410E9428B35E
:10C290004FEF20C0F394F4E0FF1689F0F80181918C
:10C2A0008F010E949E418823A9F30E948A410E9427
:10C2B00028B3462F6FEF8F2D0E94BF98EBCF82E4FB
:10C2C0000E949E41882349F00E948A410E9428B31F
:10C2D000462F6FEF84E00E94BF980E94C399D1C09F
:10C2E00084E50E949E41882309F487C00E948A4108
:10C2F0000E942DB360936B086623A9F1ECEBFEE07E
:10C300008491882341F09091C00095FFFCCF8093E9
:10C31000C6003196F5CFE7E7F4E08191882339F044
:10C320009091C00095FFFCCF8093C600F6CF40E00F
:10C3300050E060916B0887EC9DE00E94518EE9E728
:10C34000F4E08191882339F09091C00095FFFCCFF3
:10C350008093C600F6CF8091C00085FFFCCF8AE0B5
:10C360008093C6008EC086E40E949E418823D9F047
:10C370000E948A416B017C0160931D0A70931E0A22
:10C3800080931F0A9093200A20E030E0A9010E94C8
:10C39000BCB4181644F4C0922102D0922202E0925A
:10C3A0002302F0922402ECEBFEE08491882341F01A
:10C3B0009091C00095FFFCCF8093C6003196F5CFD9
:10C3C000EAE8F4E08191882339F09091C00095FF6C
:10C3D000FCCF8093C600F6CF60914E0A70E04AE031
:10C3E00050E087EC9DE00E941A8E8091C00085FF8E
:10C3F000FCCF8AE08093C60044C0ECEBFEE0849161
:10C40000882341F09091C00095FFFCCF8093C60037
:10C410003196F5CFEBE8F9E08491882341F09091D3
:10C42000C00095FFFCCF8093C6003196F5CF809178
:10C4300086089091870820E6289FF001299FF00D3B
:10C440001124E457F74F8191882339F09091C0006F
:10C4500095FFFCCF8093C600F6CFE9E8F9E0849120
:10C46000882341F09091C00095FFFCCF8093C600D7
:10C470003196F5CF8091C00085FFFCCF8AE0809394
:10C48000C6000E94C541B9C1C090390AD0903A0A8D
:10C49000E0903B0AF0903C0A20916E0A30916F0ABE
:10C4A0004091700A5091710AC701B6010E94DFB134
:10C4B0002DEC3CEC4CEC5DE30E94BCB4181614F07F
:10C4C0000C94C34CC0926E0AD0926F0AE092700A2C
:10C4D000F092710A8EE69AE00E94FCA860E080E08B
:10C4E0000E941D448AC180E090E00E94893D0C9426
:10C4F000C04D81E090E00E94893D0C94CB4D82E0DC
:10C5000090E00E94893D0C94144E0E94201F80E010
:10C510000E94934A0E94DB770C94C9500E94934179
:10C52000AB01BC0140931E0D50931F0D6093200D75
:10C530007093210D89E69CE00E945713A2CF0E94C0
:10C540008A410E9428B38B010C94ED520E944AAD9F
:10C55000681979098A099B09693E7340810591052B
:10C5600008F479C0E3E7FBE08491882341F09091DF
:10C57000C00095FFFCCF8093C6003196F5CFE091C7
:10C580006B0824E0E29FF0011124E25AF74F40814A
:10C5900051816281738121E030E087EC9DE00E944F
:10C5A000F08EEFE6FBE08491882341F09091C0008B
:10C5B00095FFFCCF8093C6003196F5CF60916B0854
:10C5C00070E04AE050E087EC9DE00E941A8EEBE6B6
:10C5D000FBE08491882341F09091C00095FFFCCF4F
:10C5E0008093C6003196F5CFF7FE03C0EBEBF5E084
:10C5F00025C00E944AAD8B019C01C701B601685459
:10C60000744F8F4F9F4F601B710B820B930BA301D5
:10C6100092010E9497B6BA01A9012AE030E087ECA6
:10C620009DE00E94468E8091C00085FFFCCF0DC02A
:10C630009091C00095FFFCCF8093C600819181113D
:10C64000F7CF8091C00085FFFCCF3092C6000E94DA
:10C650004AAD4B015C010E94201F80E00E94934A7A
:10C660000E94DB77FFEFCF16DF06EF06FF0609F02B
:10C6700046C080916908E0916B08F0E08F01000FDF
:10C68000111F000F111F025A174FEE0FFF1FEA591B
:10C69000F74F608171818823C9F0882777FD8095E5
:10C6A000982F0E945BB320E030E040E85FE30E94F7
:10C6B000DFB19B01AC01F8016081718182819381BE
:10C6C0000E94BCB487FF50C00C94C254882777FDE9
:10C6D0008095982F0E945BB320E030E040E85FE354
:10C6E0000E94E0B19B01AC01F801608171818281FF
:10C6F00093810E94B9B21816BCF50C94C254F7FE8F
:10C7000002C00C94C254E0916B08F0E08F01000F5E
:10C71000111F000F111F025A174FEE0FFF1FEA598A
:10C72000F74F60817181882777FD8095982F0E944F
:10C730005BB39B01AC01F8016081718182819381BF
:10C740000E94DFB10E9428B397FF07C090958095A3
:10C75000709561957F4F8F4F9F4F663071058105B2
:10C76000910514F40C94C2540E944AAD6B017C01F3
:10C770000C94C2548DE59BE00E943F778091830A20
:10C78000882321F08AE893E00E949A730E944AADC0
:10C790006093700870937108809372089093730887
:10C7A0000E944AAD609378087093790880937A0864
:10C7B00090937B0866CE0E94FD9688E50E949E417C
:10C7C000882319F0179A1092530A89E50E949E4116
:10C7D000882319F0169A1092540A8AE50E949E4105
:10C7E000882319F0159A1092550A85E40E949E41FB
:10C7F000882309F446CE149A44CEE9960FB6F894ED
:10C80000DEBF0FBECDBFDF91CF911F910F91FF9083
:10C81000EF90DF90CF90BF90AF909F908F907F90E0
:10C820006F905F904F903F900895CF93DF938091EA
:10C83000820890918308039714F40E94C44660E034
:10C8400081E89AE00E94E234809182089091830806
:10C85000892B09F464C08091810A8823E1F08091DA
:10C8600086089091870820E6289FE001299FD00D37
:10C870001124C457D74F6EE77DE0CE010E94E7B97F
:10C88000892BF1F4BE0181E89AE00E947134809115
:10C89000820A882319F00E94144C2BC0EBE7FDE0BC
:10C8A0008491882341F09091C00095FFFCCF809344
:10C8B000C6003196F5CF8091C00085FFFCCF16C031
:10C8C00060E081E89AE00E94D835E9E6FDE08491D5
:10C8D000882341F09091C00095FFFCCF8093C60063
:10C8E0003196F5CF8091C00085FFFCCF8AE0809320
:10C8F000C6008091820890918308019790938308E5
:10C90000809382088091860890918708019664E060
:10C9100070E00E9484B690938708809386080E94F6
:10C92000201F80E00E94934A0E940F8FDF91CF91D9
:10C930000C94DB778F929F92AF92BF92CF92DF924F
:10C94000EF92FF920F931F93CF93DF938C018C5143
:10C950009E4F0E94852E680189E8C80ED11C21F1E6
:10C96000780181E4E81A8EEFF80AE70157018FE1B8
:10C97000A81AB10878ED872E75E0972ECC15DD0545
:10C9800099F0FE01EE19FF09EA0DFB1D91828082EC
:10C99000FE0178978081811102C06F97EFCFCE01A1
:10C9A0004B970E943A14F9CFC80186599F4F0E94B5
:10C9B000852EC801875B9F4FDF91CF911F910F910B
:10C9C000FF90EF90DF90CF90BF90AF909F908F90AF
:10C9D0000C94852E81E89AE00C94912E81E89AE0DF
:10C9E000A9CFFB0160917002709171027093500D9C
:10C9F00060934F0D6091590D70915A0D70934E0DCB
:10CA000060934D0D62E060936F026FED71E870937B
:10CA100071026093700290934C0D80934B0DF093D4
:10CA20004A0DE093490D662757FD6095762F409398
:10CA3000450D5093460D6093470D7093480DC90105
:10CA4000AA2797FDA095BA2F841B950BA60BB70BB1
:10CA50008093410D9093420DA093430DB093440DEC
:10CA600080819181AA2797FDA095BA2F841B950BF1
:10CA7000A60BB70B8093590D90935A0DA0935B0DA5
:10CA8000B0935C0D08950F931F93CF93DF93EB0149
:10CA9000142F022F482F60E084E69DE00E942C298D
:10CAA000612F84E69DE00E94D8B111E1FE016491FE
:10CAB000662311F0111117C0112339F060E284E6EA
:10CAC0009DE00E94D8B11150F7CF602F84E69DE021
:10CAD0000E94D8B160E284E69DE0DF91CF911F9182
:10CAE0000F910C94D8B184E69DE00E94D8B12196B4
:10CAF0001150DCCFEF92FF920F931F93CF93DF93F0
:10CB0000EB01E42E8901F90101900020E9F7F22EF2
:10CB1000FE1A92E1F90E482F60E084E69DE00E9443
:10CB20002C296E2D84E69DE00E94D8B1FE0164910F
:10CB3000662311F0F11019C06AE384E69DE00E94BB
:10CB4000D8B1FF2039F060E284E69DE00E94D8B1C0
:10CB5000FA94F7CFB80184E69DE0DF91CF911F9161
:10CB60000F91FF90EF900C94D7B184E69DE00E9466
:10CB7000D8B12196FA94DACF1092BE0D81E89AE0EE
:10CB80000E94823A1092620D089581E89AE00C9416
:10CB9000E43181E89AE00C94EB31CF93DF93CDB789
:10CBA000DEB7C054D1090FB6F894DEBF0FBECDBFBB
:10CBB00088E0EBEBF2E0DE01D99601900D928A95C8
:10CBC000E1F788E0E3ECF2E0DE01D19601900D920E
:10CBD0008A95E1F788E0EBECF2E0DE0199960190AE
:10CBE0000D928A95E1F788E0E3EDF2E0DE0191969F
:10CBF00001900D928A95E1F788E0EBEDF2E0DE011D
:10CC0000599601900D928A95E1F788E0E3EEF2E003
:10CC1000DE01519601900D928A95E1F788E0EBEEE6
:10CC2000F2E0DE01199601900D928A95E1F788E015
:10CC3000E3EFF2E0DE01119601900D928A95E1F7A3
:10CC4000AE01475C5F4F60E084E69DE00E94CA2A27
:10CC5000AE014F5C5F4F61E084E69DE00E94CA2A0E
:10CC6000AE01475D5F4F62E084E69DE00E94CA2A04
:10CC7000AE014F5D5F4F63E084E69DE00E94CA2AEB
:10CC8000AE01475E5F4F64E084E69DE00E94CA2AE1
:10CC9000AE014F5E5F4F65E084E69DE00E94CA2AC8
:10CCA000AE01475F5F4F66E084E69DE00E94CA2ABE
:10CCB000AE014F5F5F4F67E084E69DE00E94CA2AA5
:10CCC000C05CDF4F0FB6F894DEBF0FBECDBFDF9163
:10CCD000CF910895CF9382E080936F020E944AAD76
:10CCE0006C507E4F8F4F9F4F60935E0D70935F0D22
:10CCF0008093600D9093610D6A9ACAE0729A84E6FF
:10CD000090E00E949DAD729884E690E00E949DADF7
:10CD1000C150A1F7CF910895E0917002F091710296
:10CD2000E817F90771F090937102809370024093B5
:10CD3000590D50935A0D60935B0D70935C0D21114A
:10CD4000C9CF089521E040E050E0BA01E5CF21E0ED
:10CD500040E050E0BA01E0CFCF92DF92EF92FF9235
:10CD60000F931F93CF93DF938091590D90915A0D9C
:10CD7000A0915B0DB0915C0D81309048A105B1058B
:10CD800040F01092590D10925A0D10925B0D1092B6
:10CD90005C0D8091590D90915A0DA0915B0DB09151
:10CDA0005C0DB695A795979587954091620D50E0DB
:10CDB00060E070E084179507A607B70710F480932A
:10CDC000620DD091620D1091630D12FB112710F9C5
:10CDD000C0E0FBE0CF2ED12CE12CF12C01E0409102
:10CDE000590D50915A0D60915B0D70915C0DD111F0
:10CDF0002DC080916F02882369F023E042305105F5
:10CE00006105710510F443E001C040E26DEC71E191
:10CE10008C2F39DE112309F4F1C08091590D9091C6
:10CE20005A0DA0915B0DB0915C0D0297A105B10563
:10CE300008F0E4C04FDF8EEB93E7DF91CF911F91B5
:10CE40000F91FF90EF90DF90CF907CCFD13051F5D4
:10CE500080916F02882389F076956795579547955D
:10CE600023E0413051056105710511F443E001C033
:10CE700040E26BEB71E18C2F06DE112309F4BEC09A
:10CE80008091590D90915A0DA0915B0DB0915C0D60
:10CE9000B695A795979587950197A105B10509F0D6
:10CEA000ADC0C8CFD23051F580916F02882389F090
:10CEB000769567955795479523E042305105610572
:10CEC000710511F443E001C040E26FEA71E18C2F7B
:10CED000DADD112309F492C08091590D90915A0D19
:10CEE000A0915B0DB0915C0DB695A7959795879530
:10CEF0000297A105B10509F081C09CCFD33051F54F
:10CF000080916F02882389F07695679557954795AC
:10CF100023E0433051056105710511F443E001C080
:10CF200040E26DE971E18C2FAEDD112309F466C09A
:10CF30008091590D90915A0DA0915B0DB0915C0DAF
:10CF4000B695A795979587950397A105B10509F023
:10CF500055C070CFD43041F580916F02882389F09D
:10CF6000769567955795479523E0443051056105BF
:10CF7000710511F443E001C040E26BE871E18C2FD0
:10CF800082DD1123D9F18091590D90915A0DA09114
:10CF90005B0DB0915C0DB695A79597958795049715
:10CFA000A105B10559F546CFD53041F580916F0205
:10CFB000882389F0769567955795479523E0453006
:10CFC00051056105710511F443E001C040E26FE7CE
:10CFD00071E18C2F58DD112389F08091590D9091CA
:10CFE0005A0DA0915B0DB0915C0DB695A7959795E4
:10CFF00087950597A105B10509F41CCF8091590DBE
:10D0000090915A0DA0915B0DB0915C0D0C97A1050C
:10D01000B10540F0C092590DD0925A0DE0925B0DCF
:10D02000F0925C0D4091590D50915A0D60915B0D3D
:10D0300070915C0D76956795579547958091620D37
:10D0400090E00396242F30E0821793074CF48DEF85
:10D05000840F8093620D00936F02DCEFD40FCFEF4B
:10D06000CF5FDF5FC43008F4BACEDF91CF911F915C
:10D070000F91FF90EF90DF90CF9008950F931F9343
:10D08000CF93DF938091590D90915A0DA0915B0D34
:10D09000B0915C0D81309048A105B10540F010922F
:10D0A000590D10925A0D10925B0D10925C0D8091EB
:10D0B000590D90915A0DA0915B0DB0915C0DB695F4
:10D0C000A795979587954091620D50E060E070E0DC
:10D0D00084179507A607B70710F48093620DD091C7
:10D0E000620D1091630D12FB112710F9C0E001E0F1
:10D0F0008091590D90915A0DA0915B0DB0915C0DEE
:10D10000D11128C020916F02222361F023E0029701
:10D11000A105B10510F443E001C040E269EF70E100
:10D120008C2FB1DC112309F46EC08091590D9091C0
:10D130005A0DA0915B0DB0915C0D0297A105B10550
:10D1400008F061C0C7DD8DE591E7DF91CF911F91B8
:10D150000F91F8CDD13059F520916F02222381F043
:10D16000B695A795979587952EE70197A105B105E7
:10D1700011F44EE301C040E26EEE70E18C2F83DCCF
:10D18000112309F440C08091590D90915A0DA0913E
:10D190005B0DB0915C0DB695A79597958795019716
:10D1A000A105B10581F596DD8BE293E89FC0D230F1
:10D1B00051F520916F02222381F0B695A79597959E
:10D1C00087952EE70297A105B10511F44EE301C042
:10D1D00040E263EE70E18C2F56DC1123A1F08091C8
:10D1E000590D90915A0DA0915B0DB0915C0DB695C3
:10D1F000A795979587950297A105B10521F46ADD5A
:10D2000082E393E873C020E030E040E251E46091B3
:10D21000350D7091360D8091370D9091380D0E942B
:10D22000B9B287FF68C08091590D90915A0DA091B5
:10D230005B0DB0915C0DD33061F520916F0222231C
:10D2400081F0B695A795979587952EE70397A10549
:10D25000B10511F44EE301C040E268ED70E18C2F9E
:10D2600012DC111102C025E047C08091590D909148
:10D270005A0DA0915B0DB0915C0DB695A795979551
:10D2800087950397A105B10571F724DD89E393E83C
:10D290002DC0D43041F720916F02222381F0B69542
:10D2A000A795979587952EE70497A105B10511F4E9
:10D2B0004EE301C040E26FEC70E18C2FE4DB112300
:10D2C00091F24091590D50915A0D60915B0D709102
:10D2D0005C0D7695679557954795443051056105E6
:10D2E000710509F0C0CFF6DC86E691E8DF91CF91B9
:10D2F0001F910F912CCD23E04091590D50915A0D63
:10D3000060915B0D70915C0D76956795579547958B
:10D31000822F90E0A0E0B0E0481759076A077B072A
:10D3200088F0822F90E0880F991F0197AA2797FD18
:10D33000A095BA2F8093590D90935A0DA0935B0D31
:10D34000B0935C0D4091590D50915A0D60915B0D59
:10D3500070915C0D76956795579547958091620D14
:10D3600090E00396242F30E0821793074CF48DEF62
:10D37000840F8093620D00936F02DCEFD40FCFEF28
:10D38000CF5FDF5FC43008F4B3CEDF91CF911F9140
:10D390000F91089580E090E0A0E8BFE38093350D01
:10D3A0009093360DA093370DB093380D67CE20E0E3
:10D3B00044E064E184E69DE00E945F29EEDB84E6C0
:10D3C0009DE00C942029F3DF20E040E050E0BA011A
:10D3D0008BED93E8A1CC109267081092660810922A
:10D3E00065081092640810924D0A10924C0AEBCF17
:10D3F00084E69DE00C94202920E030E04EE353E4E5
:10D4000060915E0870915F0880916008909161085A
:10D410000E94BCB418164CF48EE09FE00E948E3F30
:10D4200081E09FE00E948E3F20C0E2DF40E060E0AC
:10D4300084E69DE00E942C2968ED74E084E69DE07E
:10D440000E94D7B142E060E084E69DE00E942C2972
:10D450006FED74E084E69DE00E94D7B160ED77E067
:10D4600080E090E00E9479ADC3DFADCF20E030E0F6
:10D470004EE353E460915E0870915F08809160080C
:10D48000909161080E94BCB418166CF48DEF9EE078
:10D490000E948E3F81EF9EE00E948E3F85EE9EE0CF
:10D4A0000E948E3F20C0A4DF40E060E084E69DE063
:10D4B0000E942C2968ED74E084E69DE00E94D7B1BB
:10D4C00042E060E084E69DE00E942C296FED74E06C
:10D4D00084E69DE00E94D7B160ED77E080E090E0C7
:10D4E0000E9479AD85DF6FCF8091BB0D9091BC0D0F
:10D4F00090936708809366088091B90D9091BA0D5A
:10D50000909365088093640810924D0A10924C0A1B
:10D510005ADF0C94F2218091B50D9091B60D909345
:10D520006708809366088091B30D9091B40D909335
:10D5300065088093640810924D0A10924C0A43DFEC
:10D540000C94F22180919502909196029093670835
:10D55000809366088091930290919402909365085D
:10D560008093640810924D0A10924C0A2CDF0C94A0
:10D57000F22180919102909192029093670880939A
:10D58000660880918F029091900290936508809335
:10D59000640810924D0A10924C0A15DF0C94F22187
:10D5A00080918D0290918E02909367088093660817
:10D5B00080918B0290918C0290936508809364080F
:10D5C00010924D0A10924C0AFEDE0C94F2218091CA
:10D5D000890290918A0290936708809366088091EF
:10D5E0008702909188029093650880936408109256
:10D5F0004D0A10924C0AE7DE0C94F2212F923F92D2
:10D600004F925F926F927F928F929F92AF92BF9252
:10D61000CF92DF92EF92FF920F931F93CF93DF93FE
:10D62000CDB7DEB7A2970FB6F894DEBF0FBECDBF61
:10D6300080916F02811104C08091630D82FFA9C2A5
:10D6400081E89AE00E9476394091590D50915A0D27
:10D6500060915B0D70915C0D413050486105710522
:10D6600040F01092590D10925A0D10925B0D1092CD
:10D670005C0D4091590D50915A0D60915B0D709168
:10D680005C0D76956795579547950091620D10E072
:10D6900020E030E0401751076207730710F4409311
:10D6A000620D4090620D3090630D32FA332430F8F1
:10D6B000512C9C012150310939A328A341102BC0C2
:10D6C00080916F028823A1F08091590D90915A0D9D
:10D6D000A0915B0DB0915C0D23E00297A105B1050F
:10D6E00010F443E001C040E263E770E1852DCBD93F
:10D6F000332089F08091590D90915A0DA0915B0DC6
:10D70000B0915C0D0297A105B10528F4E3DA8EEB28
:10D7100093E718DB3EC265E87AE08FEE9AE00E945C
:10D72000EE108091850A8F3229F031E0431669F0BE
:10D7300022E001C021E0A8A0B9A0C42CD12CE12C8A
:10D74000F12C22242394240C49C080916F02882359
:10D75000C1F08091590D90915A0DA0915B0DB0913F
:10D760005C0DB695A7959795879520E20197A10541
:10D77000B10511F44EE301C040E26FE670E1852D82
:10D7800082D93320A9F28091590D90915A0DA09120
:10D790005B0DB0915C0DB695A79597958795019710
:10D7A000A105B10529F696DAE7D9F3C124115FC1C5
:10D7B00040E050E0B50181E89AE00E94ED3590919B
:10D7C000C70A80916F02992309F49AC081110BC096
:10D7D000311074C0222DF1E0AF1AB1083FEFA3164B
:10D7E000B30621F746C18091590D90915A0DA09131
:10D7F0005B0DB0915C0DB695A79597958795452DD6
:10D8000060E08C159D05AE05BF0561F584E69DE0E1
:10D810000E942C296EE384E69DE00E94D8B165E069
:10D8200084E69DE00E94D8B18091920A882329F075
:10D830001092A40A02E91AE002C005E81AE0B2E177
:10D840009B2EF80161918F01662311F0911060C148
:10D85000992009F4BDCF60E284E69DE00E94D8B132
:10D860009A94F6CF84E69DE00E942C2960E284E63B
:10D870009DE00E94D8B165E084E69DE00E94D8B1A9
:10D880008091920A882329F01092A40A02E91AE0F2
:10D8900002C005E81AE0A2E19A2EF80161918F0119
:10D8A000662311F091103AC1992009F491CF60E2FA
:10D8B00084E69DE00E94D8B19A94F6CF8091590DEC
:10D8C00090915A0DA0915B0DB0915C0DB695A79506
:10D8D000979587958C159D05AE05BF0509F07ACF04
:10D8E000F9D965E87AE081E89AE00E94D939109286
:10D8F000590D10925A0D10925B0D10925C0D49C19A
:10D90000811103C0311071C065CF8091590D909184
:10D910005A0DA0915B0DB0915C0DB695A7959795AA
:10D9200087958C159D05AE05BF05B1F52091C60DF7
:10D930002F8F10E0412F60E084E69DE00E942C29AB
:10D9400060E284E69DE00E94D8B11F5F143091F739
:10D95000452D60E084E69DE00E942C296EE384E67C
:10D960009DE00E94D8B163E9862E6AE0962E72E9A6
:10D97000672E7AE0772E01E010E0F30121913F015C
:10D980002111D2C014E1101B60E284E69DE00E94E8
:10D99000D8B11150C9F7B6CF452D60E084E69DE0BF
:10D9A0000E942C2960E284E69DE00E94D8B180911B
:10D9B000920A882329F01092A50A02E91AE002C00F
:10D9C00005E81AE053E1952EF80161918F01662375
:10D9D00011F09110D8C0992009F494CF60E284E648
:10D9E0009DE00E94D8B19A94F6CF8091590D909104
:10D9F0005A0DA0915B0DB0915C0DB695A7959795CA
:10DA000087958C159D05AE05BF0509F0E3CE62D95B
:10DA100085E89AE09F938F9388E690E19F938F9398
:10DA20008E010F5F1F4F1F930F930E9474BA0F90C8
:10DA30000F900F900F900F900F907E01F5E0EF0E7A
:10DA4000F11CF7018081882349F0992787FD909583
:10DA50000E94B1B9F70181937F01F3CFC8010E9401
:10DA60001B3F84E690E10E948E3FADDC92C02F5FA9
:10DA7000B2CE8091590D90915A0DA0915B0DB0914D
:10DA80005C0DB695A79597958795422F50E060E07D
:10DA900070E084179507A607B70788F0822F90E0FB
:10DAA000880F991F0197AA2797FDA095BA2F8093F9
:10DAB000590D90935A0DA0935B0DB0935C0D80911E
:10DAC000590D90915A0DA0915B0DB0915C0DB695DA
:10DAD000A795979587952091620D30E02D5F3F4F78
:10DAE000482F50E02417350764F42DEF280F2093BA
:10DAF000620D21E020936F02FCEF4F2E480E55245B
:10DB00005A945394439483E0851508F0D7CD41C0CF
:10DB100084E69DE00E94D8B19A9493CE84E69DE07D
:10DB20000E94D8B19A94B9CE452D602F84E69DE02D
:10DB30002AA30E942C292AA1622F84E69DE00E943C
:10DB4000D8B10F5F1F4F0431110509F016CF340112
:10DB50000CE211E08091630D82FD05C08091C60D3D
:10DB60003F8D381749F0015011090115110591F742
:10DB70008FEF881A980AFFCE61E070E080E090E0B5
:10DB80000E9479ADF0CF84E69DE00E94D8B19A94CE
:10DB90001BCFA2960FB6F894DEBF0FBECDBFDF91AC
:10DBA000CF911F910F91FF90EF90DF90CF90BF909A
:10DBB000AF909F908F907F906F905F904F903F902D
:10DBC0002F900895CF92DF92EF92FF920F931F93C1
:10DBD000CF93DF938091590D90915A0DA0915B0DD9
:10DBE000B0915C0D81309048A105B10540F01092D4
:10DBF000590D10925A0D10925B0D10925C0D809190
:10DC0000590D90915A0DA0915B0DB0915C0DB69598
:10DC1000A795979587954091620D50E060E070E080
:10DC200084179507A607B70710F48093620DD0916B
:10DC3000620D1091630D12FB112710F9C0E0BFE0D7
:10DC4000CB2ED12CE12CF12C01E04091590D5091BB
:10DC50005A0D60915B0D70915C0DD1112EC08091B9
:10DC60006F02882371F023E0423051056105710590
:10DC700010F443E001C040E265E470E18C2F0E94A3
:10DC80004365112309F498C18091590D90915A0D63
:10DC9000A0915B0DB0915C0D0297A105B10508F054
:10DCA0008BC118D88EEB93E7DF91CF911F910F9125
:10DCB000FF90EF90DF90CF9045C8D130A9F58091CB
:10DCC0006F02882391F0769567955795479520E2E6
:10DCD000413051056105710511F44EE301C040E288
:10DCE00065E370E18C2F0E944365112309F464C140
:10DCF0008091590D90915A0DA0915B0DB0915C0DE2
:10DD0000B695A795979587950197A105B10509F057
:10DD100053C10E946A66DF91CF911F910F91FF90CE
:10DD2000EF90DF90CF90F7CBD230A9F580916F02C2
:10DD3000882391F0769567955795479520E2423074
:10DD400051056105710511F44EE301C040E266E240
:10DD500070E18C2F0E944365112309F42DC180913D
:10DD6000590D90915A0DA0915B0DB0915C0DB69537
:10DD7000A795979587950297A105B10509F01CC154
:10DD80000E946A66DF91CF911F910F91FF90EF90F3
:10DD9000DF90CF90A9CBD330A9F580916F02882373
:10DDA00091F0769567955795479520E24330510558
:10DDB0006105710511F44EE301C040E267E170E1D5
:10DDC0008C2F0E944365112309F4F6C08091590DF0
:10DDD00090915A0DA0915B0DB0915C0DB695A795F1
:10DDE000979587950397A105B10509F0E5C00E94B5
:10DDF0006A66DF91CF911F910F91FF90EF90DF90B6
:10DE0000CF90B7CBD430A9F580916F02882391F0E1
:10DE1000769567955795479520E244305105610501
:10DE2000710511F44EE301C040E267E070E18C2F10
:10DE30000E944365112309F4BFC08091590D909150
:10DE40005A0DA0915B0DB0915C0DB695A795979575
:10DE500087950497A105B10509F0AEC00E946A66D6
:10DE6000DF91CF911F910F91FF90EF90DF90CF90B6
:10DE700097CBD530A9F580916F02882391F07695E4
:10DE800067955795479520E2453051056105710525
:10DE900011F44EE301C040E267EF7FE08C2F0E9457
:10DEA0004365112309F488C08091590D90915A0D52
:10DEB000A0915B0DB0915C0DB695A7959795879550
:10DEC0000597A105B10509F077C00E946A66DF9148
:10DED000CF911F910F91FF90EF90DF90CF9032CBB9
:10DEE000D630A9F580916F02882391F076956795D9
:10DEF0005795479520E2463051056105710511F4AB
:10DF00004EE301C040E268EE7FE08C2F0E94436543
:10DF1000112309F451C08091590D90915A0DA0918F
:10DF20005B0DB0915C0DB695A79597958795069773
:10DF3000A105B10509F040C00E946A66DF91CF914A
:10DF40001F910F91FF90EF90DF90CF9040CBD73093
:10DF500099F580916F02882391F076956795579592
:10DF6000479520E2473051056105710511F44EE3F4
:10DF700001C040E26FED7FE08C2F0E9443651123CA
:10DF8000D9F08091590D90915A0DA0915B0DB091EF
:10DF90005C0DB695A795979587950797A105B1054F
:10DFA00059F40E946A66DF91CF911F910F91FF9003
:10DFB000EF90DF90CF900FCA8091590D90915A0D3C
:10DFC000A0915B0DB0915C0D4097A105B10540F0AB
:10DFD000C092590DD0925A0DE0925B0DF0925C0DFB
:10DFE0004091590D50915A0D60915B0D70915C0DEF
:10DFF00076956795579547958091620D90E00396C9
:10E00000242F30E0821793074CF48DEF840F809318
:10E01000620D00936F02DCEFD40FCFEFCF5FDF5FB5
:10E02000C43008F412CEDF91CF911F910F91FF9071
:10E03000EF90DF90CF900895DBD941E060E084E677
:10E040009DE00E942C2965E075E084E69DE00E9439
:10E05000D7B142E060E084E69DE00E942C2965E1B2
:10E0600075E084E69DE00C94D7B1C2D942E060E04F
:10E0700084E69DE00E942C296AE275E084E69DE03A
:10E080000C94D7B11F93CF93DF93B2D940E060E0F7
:10E0900084E69DE00E942C2969E375E084E69DE01A
:10E0A0000E94D7B142E060E084E69DE00E942C2906
:10E0B00067E475E084E69DE00E94D7B110E043E09C
:10E0C000612F84E69DE00E942C296BE673E084E6D4
:10E0D0009DE00E94D7B1CAE0D0E00E94201F81E0FD
:10E0E0000E94934A65E570E080E090E00E9479AD7F
:10E0F0002197209791F71F5F143109F7DF91CF9196
:10E100001F9108951F93CF93DF9372D940E060E091
:10E1100084E69DE00E942C2966E575E084E69DE09A
:10E120000E94D7B142E060E084E69DE00E942C2985
:10E1300067E475E084E69DE00E94D7B110E043E01B
:10E14000612F84E69DE00E942C296BE673E084E653
:10E150009DE00E94D7B1CAE0D0E00E94201F81E07C
:10E160000E94934A6EE670E080E090E00E9479ADF4
:10E170002197209791F71F5F143109F7DF91CF9115
:10E180001F9108951F93CF93DF93EC01FB016081F2
:10E1900011810E9498BC612FCE010196DF91CF9131
:10E1A0001F910C9498BCFF920F931F93CF93DF9312
:10E1B0008C01EB010E9490BCF82EC80101960E94D0
:10E1C00090BCF8828983DF91CF911F910F91FF90CE
:10E1D0000895EF92FF920F931F93CF93DF931F92B7
:10E1E000CDB7DEB77B018C01061B170B460FC701AD
:10E1F000800F911FF70161917F0149830E9498BCB4
:10E2000049814E11F4CF0F90DF91CF911F910F9163
:10E21000FF90EF90089581E09091BD0D911180E005
:10E220008093BD0D41E06DEB7DE08FEF9FE0D1DF8E
:10E230000E94579821E047E050E060E070E08DE5F3
:10E2400091E70C948C6681E09091BD0D911180E076
:10E250008093BD0D41E06DEB7DE08FEF9FE0B9DF76
:10E260000E94579821E049E050E060E070E080E7CC
:10E270009DE70C948C66EF92FF920F931F93CF93C0
:10E28000DF931F92CDB7DEB77B018C01061B170B06
:10E29000460FC701800F911F49830E9490BCF70170
:10E2A00081937F0149814E13F4CF0F90DF91CF917D
:10E2B0001F910F91FF90EF900895CF92DF92EF9210
:10E2C000FF920F931F93CF93DF9341E06DEB7DE0BF
:10E2D0008FEF9FE0D0DF8091590D90915A0DA09162
:10E2E0005B0DB0915C0D81309048A105B10540F007
:10E2F0001092590D10925A0D10925B0D10925C0DF8
:10E300008091590D90915A0DA0915B0DB0915C0DCB
:10E31000B695A795979587954091620D50E060E07E
:10E3200070E084179507A607B70710F48093620D75
:10E33000D091620D1091630D12FB112710F9C0E00E
:10E34000BDE0CB2ED12CE12CF12C01E04091590DF8
:10E3500050915A0D60915B0D70915C0DD11130C0E0
:10E3600080916F02882371F023E0423051056105EE
:10E37000710510F443E001C040E260E771E18C2FC9
:10E380000E944365112309F41FC18091590D90919A
:10E390005A0DA0915B0DB0915C0D0297A105B105DE
:10E3A00008F012C10E946A668EEB93E7DF91CF916D
:10E3B0001F910F91FF90EF90DF90CF900C94A26689
:10E3C000D13079F580916F02882391F07695679529
:10E3D000579547952EE7413051056105710511F4B8
:10E3E0004EE301C040E268E671E18C2F0E94436574
:10E3F000112309F4E9C08091590D90915A0DA09113
:10E400005B0DB0915C0DB695A79597958795019793
:10E41000A105B10509F0D8C00E946A6683ED9BE7AB
:10E4200030C0D230C1F580916F02882391F076958B
:10E430006795579547952EE742305105610571055F
:10E4400011F44EE301C040E26BE571E18C2F0E94B4
:10E450004365112309F4B8C08091590D90915A0D6C
:10E46000A0915B0DB0915C0DB695A795979587959A
:10E470000297A105B10509F0A7C00E946A668AEC5F
:10E4800099E6DF91CF911F910F91FF90EF90DF9070
:10E49000CF900C94A766D33079F580916F028823D2
:10E4A00091F0769567955795479520E24330510551
:10E4B0006105710511F44EE301C040E26EE471E1C3
:10E4C0008C2F0E944365112309F47EC08091590D61
:10E4D00090915A0DA0915B0DB0915C0DB695A795EA
:10E4E000979587950397A105B10509F06DC00E9426
:10E4F0006A6688E491E12FC0D430B9F580916F024B
:10E50000882391F0769567955795479520E244309A
:10E5100051056105710511F44EE301C040E269E364
:10E5200071E18C2F0E944365112309F44DC0809145
:10E53000590D90915A0DA0915B0DB0915C0DB6955F
:10E54000A795979587950497A105B105E9F50E94D0
:10E550006A6685E391E1DF91CF911F910F91FF9062
:10E56000EF90DF90CF900C948E3FD53069F580917D
:10E570006F02882391F0769567955795479520E22D
:10E58000453051056105710511F44EE301C040E2CB
:10E590006BE271E18C2F0E9443651123A9F08091F9
:10E5A000590D90915A0DA0915B0DB0915C0DB695EF
:10E5B000A795979587950597A105B10529F40E9420
:10E5C0006A6687E291E1C7CF2091BD0D8091590D18
:10E5D00090915A0DA0915B0DB0915C0D211135C049
:10E5E000D63009F047C020916F02222389F0B695FA
:10E5F000A7959795879520E20697A105B10511F497
:10E600004EE301C040E265E171E18C2F0E94436559
:10E61000112381F18091590D90915A0DA0915B0DBC
:10E62000B0915C0DB695A795979587950697A1052E
:10E63000B10501F50E946A66DF91CF911F910F919C
:10E64000FF90EF90DF90CF90E6CDD63099F42091F7
:10E650006F022223E9F2B695A7959795879520E258
:10E660000697A105B10511F44EE301C040E263E055
:10E6700071E1CBCF8091590D90915A0DA0915B0D16
:10E68000B0915C0D0E97A105B10540F0C092590DF7
:10E69000D0925A0DE0925B0DF0925C0D4091590DB5
:10E6A00050915A0D60915B0D70915C0D7695679558
:10E6B000579547958091620D90E00396242F30E0A6
:10E6C000821793074CF48DEF840F8093620D0093B3
:10E6D0006F02DCEFD40FCFEFCF5FDF5FC43008F401
:10E6E00035CEDF91CF911F910F91FF90EF90DF908A
:10E6F000CF9008958093520D1092510D0895E2E746
:10E70000F2E001900020E9F73197E257F2401E163F
:10E710001F0634F01092860282E080936F02089503
:10E7200080E2E431F105B4F7DF01AE58BD4F8C93C0
:10E730003196F7CF2091B00D211108C044E150E08F
:10E74000BC0182E792E00E9465BAD9CF0895109289
:10E75000830A60E081E89AE00E94D8350E947397AE
:10E7600088E590E10E948E3F81E080933D0A89E632
:10E7700095E0E0DF84E590E10C948E3F8F929F92CC
:10E78000AF92BF92DF92EF92FF920F931F93CF93BE
:10E79000DF931092BE0D8091590D90915A0DA0916A
:10E7A0005B0DB0915C0D81309048A105B10540F042
:10E7B0001092590D10925A0D10925B0D10925C0D33
:10E7C0008091590D90915A0DA0915B0DB0915C0D07
:10E7D000B695A795979587954091620D50E060E0BA
:10E7E00070E084179507A607B70710F48093620DB1
:10E7F000D091620D1091630D12FB112710F9C0E04A
:10E80000DD24D394D11138C080916F028823A9F000
:10E810008091590D90915A0DA0915B0DB0915C0DB6
:10E8200023E00297A105B10510F443E001C040E2E6
:10E8300061E672E18C2F0E9443651123E9F080911B
:10E84000590D90915A0DA0915B0DB0915C0D0297FE
:10E85000A105B10588F40E946A668BED93E8DF910B
:10E86000CF911F910F91FF90EF90DF90BF90AF90ED
:10E870009F908F900C94A2660E9419A94091590D07
:10E8800050915A0D60915B0D70915C0D811104C027
:10E890008091830A882379F1D130A9F580916F02A4
:10E8A000882391F076956795579547952EE74130E7
:10E8B00051056105710511F44EE301C040E26BE5BD
:10E8C00072E18C2F0E9443651123E9F08091590D6C
:10E8D00090915A0DA0915B0DB0915C0DB695A795E6
:10E8E000979587950197A105B10569F40E946A661D
:10E8F00080E79DE736C2D13031F480916F028111FB
:10E9000095C21111A6C28091840A4091590D50916F
:10E910005A0D60915B0D70915C0D882309F4ECC079
:10E9200080916C0C882309F4B6C08091830A8823F7
:10E93000E1F1D23009F074C080916F02882391F028
:10E94000769567955795479520E2423051056105C8
:10E95000710511F44EE301C040E261E472E18C2FD5
:10E960000E944365112309F4DDC08091590D9091F7
:10E970005A0DA0915B0DB0915C0DB695A79597953A
:10E9800087950297A105B10509F0CCC00E946A667F
:10E99000DF91CF911F910F91FF90EF90DF90BF908B
:10E9A000AF909F908F900C94C965D230C9F580913B
:10E9B0006F02882391F0769567955795479520E2E9
:10E9C000423051056105710511F44EE301C040E28A
:10E9D00066E372E18C2F0E944365112309F4A2C003
:10E9E0008091590D90915A0DA0915B0DB0915C0DE5
:10E9F000B695A795979587950297A105B10509F05A
:10EA000091C00E946A66DF91CF911F910F91FF9094
:10EA1000EF90DF90BF90AF909F908F900C94C56562
:10EA2000D33009F07FC080916F02882391F07695F2
:10EA300067955795479520E243305105610571056B
:10EA400011F44EE301C040E268E272E18C2F0E94B3
:10EA50004365112309F466C08091590D90915A0DB8
:10EA6000A0915B0DB0915C0DB695A7959795879594
:10EA70000397A105B10509F055C00E946A66DF91B0
:10EA8000CF911F910F91FF90EF90DF90BF90AF90CB
:10EA90009F908F905CCED23011F003E044C0809103
:10EAA0006F02882391F076956795579547952EE7E5
:10EAB000423051056105710511F44EE301C040E299
:10EAC0006EE172E18C2F0E944365112331F3809136
:10EAD000590D90915A0DA0915B0DB0915C0DB695BA
:10EAE000A795979587950297A105B105B1F60E9464
:10EAF0006A668EEF9AE635C1D23079F680916F0260
:10EB0000882319F376956795579547952EE74230F8
:10EB100051056105710511F44EE301C040E26FE05B
:10EB200072E1D0CF04E08091830A8111DBC00D1324
:10EB300048C080916F028823F1F08091590D909127
:10EB40005A0DA0915B0DB0915C0DB695A795979568
:10EB50008795402F50E060E070E020E28417950731
:10EB6000A607B70711F44EE301C040E26FEF71E171
:10EB70008C2F0E944365112321F18091590D9091B2
:10EB80005A0DA0915B0DB0915C0DB695A795979528
:10EB90008795402F50E060E070E084179507A60746
:10EBA000B70779F40E946A66DF91CF911F910F91A8
:10EBB000FF90EF90DF90BF90AF909F908F900C945C
:10EBC000366AEE24E394E00EED1248C080916F02A5
:10EBD0008823F1F08091590D90915A0DA0915B0D11
:10EBE000B0915C0DB695A795979587958D2E912C34
:10EBF000A12CB12C20E288159905AA05BB0511F4BA
:10EC00004EE301C040E26EEE71E18C2F0E9443653D
:10EC1000112321F18091590D90915A0DA0915B0D16
:10EC2000B0915C0DB695A795979587954E2D50E0C0
:10EC300060E070E084179507A607B70779F40E9493
:10EC40006A66DF91CF911F910F91FF90EF90DF9057
:10EC5000BF90AF909F908F900C94FC69E2E0EE2EF5
:10EC6000E00EED123EC080916F028823F1F080919A
:10EC7000590D90915A0DA0915B0DB0915C0DB69518
:10EC8000A795979587958D2E912CA12CB12C2EE7C9
:10EC900088159905AA05BB0511F44EE301C040E2B1
:10ECA00064EE71E18C2F0E9443651123D1F08091B5
:10ECB000590D90915A0DA0915B0DB0915C0DB695D8
:10ECC000A795979587954E2D50E060E070E08417EA
:10ECD0009507A607B70729F40E946A668DE591E7B4
:10ECE00040C00D5F0D134AC080916F028823F1F080
:10ECF0008091590D90915A0DA0915B0DB0915C0DD2
:10ED0000B695A79597958795402F50E060E070E005
:10ED10002EE784179507A607B70711F44EE301C045
:10ED200040E26CED71E18C2F0E944365112331F1BB
:10ED30008091590D90915A0DA0915B0DB0915C0D91
:10ED4000B695A79597958795402F50E060E070E0C5
:10ED500084179507A607B70789F40E946A668CEAAC
:10ED600096E6DF91CF911F910F91FF90EF90DF908A
:10ED7000BF90AF909F908F900C94A766FF24F39460
:10ED8000F00E4091590D50915A0D60915B0D7091AC
:10ED90005C0D76956795579547958F2D90E0A0E08F
:10EDA000B0E0481759076A077B0788F08F2D90E07D
:10EDB000880F991F0197AA2797FDA095BA2F8093D6
:10EDC000590D90935A0DA0935B0DB0935C0D40913B
:10EDD000590D50915A0D60915B0D70915C0D7695B7
:10EDE0006795579547958091620D90E00396242F83
:10EDF00030E0821793074CF48DEF840F8093620DFF
:10EE0000D0926F02DCEFD40FCFEFCF5FDF5FC43063
:10EE100008F4F8CCDF91CF911F910F91FF90EF9004
:10EE2000DF90BF90AF909F908F90089576956795F3
:10EE3000579547952EE7413051056105710511F44D
:10EE40004EE301C040E261E572E18C2F0E94436510
:10EE500058CD8091590D90915A0DA0915B0DB091B4
:10EE60005C0DB695A795979587950197A105B10576
:10EE700009F049CD0E946A6682EE9DE672CF20912C
:10EE8000B00D211108C044E150E0BC0182E792E0DE
:10EE90000E94D8B934CC0895F2DF81E08093B00DA0
:10EEA0000C94E3691092B00D0895CF92DF92EF9227
:10EEB000FF92CF93CCB1C095CC1FCC27CC1F8091B3
:10EEC000030183FFC260C0905E0DD0905F0DE090A3
:10EED000600DF090610D0E944AADC616D706E80697
:10EEE000F90610F4489B39C0C093630D8091630DFF
:10EEF00081709091630D91FD826090915D0D8917F5
:10EF000021F18130F1F028F0823089F08330A1F0D6
:10EF10001CC0913021F49091C60D9F5F05C09230C6
:10EF2000A1F49091C60D91509093C60D0EC09923F7
:10EF300091F3933051F4F5CF923069F3913029F485
:10EF4000F0CF933041F3992361F380935D0DCF911E
:10EF5000FF90EF90DF90CF900895C460C5CF0E94DE
:10EF6000D7696F98E4E0F1E08081877F8083779AAA
:10EF70009FB7F894E5E0F1E08081886080839FBFCF
:10EF80005098589A60E088E40E946AAC9FB7F89461
:10EF9000E5E0F1E08081846080839FBF8091030180
:10EFA00082FB882780F991E089278093580D7DDFC7
:10EFB0001092C60D0895CF92DF92EF92FF9275DF07
:10EFC0008091030191E082FB882780F989272091B5
:10EFD000580D8217C9F082E080936F02809103017F
:10EFE00082FB882780F989278093580D0E94D76972
:10EFF0008091580D882309F49EC081E89AE00E9410
:10F00000153187ED9EE03BDFC090540DD090550D3B
:10F01000E090560DF090570D0E944AADC616D706E7
:10F02000E806F90608F094C08091C60D482F5527D0
:10F0300047FD509557FF03C0519541955109423006
:10F04000510584F191E090936F0287FD8F5F482F07
:10F050004595552747FD5095652F752F8091590D82
:10F0600090915A0DA0915B0DB0915C0D840F951F8E
:10F07000A61FB71F8093590D90935A0DA0935B0D57
:10F08000B0935C0D1092C60D0E944AAD6856754C47
:10F090008F4F9F4F6093290D70932A0D80932B0DF6
:10F0A00090932C0D8091630D82FF0EC00E944AAD9B
:10F0B0006856754C8F4F9F4F6093290D70932A0DA2
:10F0C00080932B0D90932C0DE0917002F0917102C2
:10F0D0001995C090290DD0902A0DE0902B0DF0903D
:10F0E0002C0D0E944AADC616D706E806F90638F47C
:10F0F00080917002909171028B5D934819F5809117
:10F100006F02823011F40E94F86980916F028823A7
:10F1100019F0815080936F020E944AAD6C597F4F65
:10F120008F4F9F4F6093540D7093550D8093560DE4
:10F130009093570D0DC081E89AE00E94E03189EC70
:10F140009EE061CF0E94E36982E080936F02D7CF97
:10F15000FF90EF90DF90CF90089581E00895809127
:10F16000630D82FB882780F908950F931F93CF9337
:10F17000DF930E94F86940E060E084E69DE00E9431
:10F180002C2967E775E084E69DE00E94D7B141E055
:10F1900061E084E69DE00E942C2962E875E084E647
:10F1A0009DE00E94D7B142E061E084E69DE00E94CC
:10F1B0002C2966E875E084E69DE00E94D7B143E023
:10F1C00061E084E69DE00E942C2969E975E084E60F
:10F1D0009DE00E94D7B141E060E084E69DE00E949E
:10F1E0002C296AEA75E084E69DE00E94D7B100917F
:10F1F000C60D112707FD1095C1E0D0E08091730A7C
:10F200009091740A892B09F071C00E94201F81E03F
:10F210000E94934A2091C60D332727FD3095C801DF
:10F22000821B930B97FF03C09195819591090597D8
:10F230000CF44DC0201731070CF421970217130767
:10F240000CF42196C430D1052CF4209729F4C1E0A8
:10F25000D0E002C0C3E0D0E041E060E084E69DE0A1
:10F260000E942C296DE973E084E69DE00E94D7B1ED
:10F2700042E060E084E69DE00E942C296DE973E0A5
:10F2800084E69DE00E94D7B143E060E084E69DE023
:10F290000E942C296DE973E084E69DE00E94D7B1BD
:10F2A0004C2F60E084E69DE00E942C296AEA75E01C
:10F2B00084E69DE00E94D7B10091C60D112707FD9D
:10F2C000109564E670E080E090E00E9479AD47DF41
:10F2D000882309F493CFD093740AC093730A64EF20
:10F2E00071E080E090E00E9479AD88CF0E94F869DB
:10F2F000DF91CF911F910F910C94E3690F931F93AE
:10F30000CF93DF930E94F86940E060E084E69DE0DF
:10F310000E942C296CEA75E084E69DE00E94D7B13A
:10F3200041E061E084E69DE00E942C2962E875E0FE
:10F3300084E69DE00E94D7B142E061E084E69DE072
:10F340000E942C296DEB75E084E69DE00E94D7B108
:10F3500041E060E084E69DE00E942C296AEA75E0C5
:10F3600084E69DE00E94D7B10091C60D112707FDEC
:10F370001095C1E0D0E00E94201F81E00E94934AD6
:10F380002091C60D332727FD3095C801821B930BB2
:10F3900097FF03C091958195910905970CF441C0A1
:10F3A000201731070CF42197021713070CF421964C
:10F3B000C330D1052CF4209729F4C1E0D0E002C07D
:10F3C000C2E0D0E041E060E084E69DE00E942C29AC
:10F3D0006DE973E084E69DE00E94D7B142E060E011
:10F3E00084E69DE00E942C296DE973E084E69DE0AF
:10F3F0000E94D7B14C2F60E084E69DE00E942C294A
:10F400006AEA75E084E69DE00E94D7B10091C60DDE
:10F41000112707FD109564E670E080E090E00E94FF
:10F4200079AD9DDE882309F4A6CF2197D9F460EC4D
:10F430007DE08DEF9FE00E94D37062EC7DE08BEF6A
:10F440009FE00E94D37064EC7DE089EF9FE00E9412
:10F45000D3708091C40D9091C50D90935608809300
:10F4600055081EC01092C10D1092C00D1092C30D10
:10F470001092C20D1092C50D1092C40D60EC7DE08B
:10F480008DEF9FE00E94C27062EC7DE08BEF9FE009
:10F490000E94C27064EC7DE089EF9FE00E94C27020
:10F4A00064EF71E080E090E00E9479AD0E94F8691D
:10F4B000DF91CF911F910F910C94E369FC01808142
:10F4C00090E02AE030E0B9010E9484B6482FCB01D9
:10F4D000B9010E9484B6805D80932D0D405D4093FC
:10F4E0002E0D10922F0D8DE29DE0089520E030E06A
:10F4F00040E251E4FC0160817181828193810E942C
:10F500008EB50E9428B377FD02C02BE201C02DE228
:10F5100020932D0D9B0177FF04C022273327261B44
:10F52000370BC90168EE73E00E9484B6CB01EAE0B4
:10F53000F0E0BF010E9484B6805D80932E0DC9016A
:10F5400064E670E00E9484B6CB01BF010E9484B6DD
:10F55000805D80932F0DC901BF010E9484B6282FC2
:10F56000CB01BF010E9484B6805D8093300D8EE296
:10F570008093310D205D2093320D1092330D8DE27A
:10F580009DE008958F929F92AF92BF92CF92DF92AB
:10F59000EF92FF92FC0180809180A280B38020E0F6
:10F5A00030E048EC52E4C501B4010E948EB56B0115
:10F5B0007C0120E030E0A9010E94BCB418161CF4C4
:10F5C000C701B60103C0C701B60190580E9428B315
:10F5D0006B017C0120E030E0A901C501B4010E946B
:10F5E000B9B287FF12C08DE280932D0DC701B6011D
:10F5F00028EE33E040E050E00E94B9B6CA01B901FC
:10F600002AE030E040E050E036C0C701B60120E11A
:10F6100037E240E050E00E94B9B6AAE08A2E912C71
:10F62000A12CB12CCA01B901A50194010E94B9B65F
:10F63000662391F0605D60932D0DC701B60128EE41
:10F6400033E040E050E00E94B9B6CA01B901A5011B
:10F6500094010E94B9B613C080E280932D0DC701BA
:10F66000B60128EE33E040E050E00E94B9B6CA018E
:10F67000B901A50194010E94B9B6662311F0605D3D
:10F6800001C060E260932E0DC701B60124E630E0B0
:10F6900040E050E00E94B9B6FAE08F2E912CA12CE8
:10F6A000B12CCA01B901A50194010E94B9B6605DEF
:10F6B00060932F0DC701B601A50194010E94B9B650
:10F6C000662381F0605D6093320DCA01B901A50126
:10F6D00094010E94B9B6605D6093310D8EE2809313
:10F6E000300D15C0CA01B901A50194010E94B9B637
:10F6F000662329F0605D6093310D8EE203C080E2E5
:10F700008093310D8093300D80E28093320D109202
:10F71000330D8DE29DE0FF90EF90DF90CF90BF9092
:10F72000AF909F908F900895FC012081318137FF29
:10F7300007C08DE280932D0D31952195310914C0BC
:10F740002436310574F0C90164E670E00E9484B685
:10F75000CB016AE070E00E9484B6805D80932D0D3D
:10F7600006C080E280932D0D2A30310564F0EAE076
:10F77000F0E0C901BF010E9484B6CB01BF010E9425
:10F7800084B6805D01C080E280932E0DC9016AE0DD
:10F7900070E00E9484B6805D80932F0D1092300D32
:10F7A0008DE29DE00895CF92DF92EF92FF920F934A
:10F7B0001F93CF93DF936091140270911502809193
:10F7C0001602909117020E946B2860933D0D709372
:10F7D0003E0D80933F0D9093400D6091100270910B
:10F7E000110280911202909113020E947728609377
:10F7F000390D70933A0D80933B0D90933C0D8091A1
:10F80000590D90915A0DA0915B0DB0915C0D813016
:10F810009048A105B10540F01092590D10925A0D73
:10F8200010925B0D10925C0D8091590D90915A0DC4
:10F83000A0915B0DB0915C0DB695A79597958795B6
:10F840004091620D50E060E070E084179507A607D4
:10F85000B70710F48093620DD091620D1091630D83
:10F8600012FB112710F9C0E0B7E0CB2ED12CE12C10
:10F87000F12C01E04091590D50915A0D60915B0DB2
:10F8800070915C0DD11130C080916F02882371F0AE
:10F8900023E0423051056105710510F443E001C0D9
:10F8A00040E266EB70E18C2F0E944365112309F45E
:10F8B000D7C08091590D90915A0DA0915B0DB091D8
:10F8C0005C0D0297A105B10508F0CAC00E946A66E6
:10F8D0008DE591E7DF91CF911F910F91FF90EF9010
:10F8E000DF90CF900C94A266D130D1F580916F0259
:10F8F0008823B9F0769567955795479586E698E001
:10F90000413051056105710521F40EDF9C014EE384
:10F9100003C00ADF9C0140E26FEA70E18C2F0E9475
:10F920007A65112309F49CC08091590D90915A0D6C
:10F93000A0915B0DB0915C0DB695A79597958795B5
:10F940000197A105B10509F08BC00E946A6623E307
:10F9500031E040E050E066E678E088EA90E176C089
:10F96000D230D1F580916F028823B9F076956795F2
:10F970005795479584E698E0423051056105710539
:10F9800021F4D2DE9C014EE303C0CEDE9C0140E2B6
:10F9900064EA70E18C2F0E947A65112309F460C03B
:10F9A0008091590D90915A0DA0915B0DB0915C0D15
:10F9B000B695A795979587950297A105B10509F08A
:10F9C0004FC00E946A6623E930E040E050E064E600
:10F9D00078E080EA90E13AC0D33009F041C08091EC
:10F9E0006F028823B9F076956795579547958CE413
:10F9F0009AE0433051056105710521F495DE9C01C3
:10FA00004EE303C091DE9C0140E261E970E18C2F7E
:10FA10000E947A65112321F18091590D90915A0D20
:10FA2000A0915B0DB0915C0DB695A79597958795C4
:10FA30000397A105B105A1F40E946A662FEF30E09B
:10FA400040E050E06CE47AE082E890E1DF91CF9111
:10FA50001F910F91FF90EF90DF90CF900C94F16485
:10FA60008091590D90915A0DA0915B0DB0915C0D54
:10FA70000897A105B10540F0C092590DD0925A0DDA
:10FA8000E0925B0DF0925C0D4091590D50915A0D32
:10FA900060915B0D70915C0D7695679557954795D4
:10FAA0008091620D90E00396242F30E08217930737
:10FAB0004CF48DEF840F8093620D00936F02DCEFA6
:10FAC000D40FCFEFCF5FDF5FC43008F4D3CEDF9128
:10FAD000CF911F910F91FF90EF90DF90CF900895FD
:10FAE000CF92DF92EF92FF920F931F93CF93DF930A
:10FAF00041E06DEB7DE08FEF9FE00E943B7160EC99
:10FB00007DE08DEF9FE00E94D37062EC7DE08BEF93
:10FB10009FE00E94D37064EC7DE089EF9FE00E943B
:10FB2000D3708091590D90915A0DA0915B0DB091B9
:10FB30005C0D81309048A105B10540F01092590D3F
:10FB400010925A0D10925B0D10925C0D8091590D20
:10FB500090915A0DA0915B0DB0915C0DB695A79553
:10FB6000979587954091620D50E060E070E08417B2
:10FB70009507A607B70710F48093620DD091620D28
:10FB80001091630D12FB112710F9C0E0F1E1CF2EA7
:10FB9000D12CE12CF12C01E04091590D50915A0DDE
:10FBA00060915B0D70915C0DD11130C080916F023E
:10FBB000882371F023E0423051056105710510F48E
:10FBC00043E001C040E260ED7FE08C2F0E9443657E
:10FBD000112309F4C3C18091590D90915A0DA09140
:10FBE0005B0DB0915C0D0297A105B10508F0B6C19F
:10FBF0000E946A668EEB93E7DF91CF911F910F9180
:10FC0000FF90EF90DF90CF900C94A266D130D1F5A9
:10FC100080916F028823B9F076956795579547953F
:10FC20008DE592E0413051056105710521F47CDDDF
:10FC30009C014EE303C078DD9C0140E267EC7FE06D
:10FC40008C2F0E947A65112309F488C18091590D87
:10FC500090915A0DA0915B0DB0915C0DB695A79552
:10FC6000979587950197A105B10509F077C10E9485
:10FC70006A6627EE33E04AE050E06DE572E08EEB15
:10FC80009FE03CC0D23009F043C080916F028823CE
:10FC9000B9F0769567955795479586E698E0423096
:10FCA00051056105710521F43FDD9C014EE303C060
:10FCB0003BDD9C0140E267EB7FE08C2F0E947A6580
:10FCC000112309F44BC18091590D90915A0DA091C7
:10FCD0005B0DB0915C0DB695A795979587950297AA
:10FCE000A105B10509F03AC10E946A6623E331E03B
:10FCF00040E050E066E678E080EB9FE0DF91CF9156
:10FD00001F910F91FF90EF90DF90CF900C94F164D2
:10FD1000D330D1F580916F028823B9F0769567953D
:10FD20005795479584E698E0433051056105710584
:10FD300021F4FADC9C014EE303C0F6DC9C0140E2B6
:10FD40006CEA7FE08C2F0E947A65112309F406C1CA
:10FD50008091590D90915A0DA0915B0DB0915C0D61
:10FD6000B695A795979587950397A105B10509F0D5
:10FD7000F5C00E946A6623E930E040E050E064E6A6
:10FD800078E088EA9FE0BACFD430D1F580916F0255
:10FD90008823B9F076956795579547958CE49AE056
:10FDA000443051056105710521F4BEDC9C014EE330
:10FDB00003C0BADC9C0140E269E97FE08C2F0E941D
:10FDC0007A65112309F4CAC08091590D90915A0D9A
:10FDD000A0915B0DB0915C0DB695A7959795879511
:10FDE0000497A105B10509F0B9C00E946A662FEF1A
:10FDF00030E040E050E06CE47AE08AE89FE07ECFBB
:10FE0000D530D1F580916F028823B9F0769567954A
:10FE1000579547958BE592E0453051056105710591
:10FE200021F482DC9C014EE303C07EDC9C0140E2B5
:10FE300063E87FE08C2F0E947A65112309F48EC05D
:10FE40008091590D90915A0DA0915B0DB0915C0D70
:10FE5000B695A795979587950597A105B10509F0E2
:10FE60007DC00E946A6627EE33E04AE050E06BE511
:10FE700072E08CE79FE042CFD630C1F580916F02EF
:10FE8000882391F0769567955795479520E24630FF
:10FE900051056105710511F44EE301C040E26BE6C6
:10FEA0007FE08C2F0E944365112309F457C0809195
:10FEB000590D90915A0DA0915B0DB0915C0DB695C6
:10FEC000A795979587950697A105B10509F046C0B6
:10FED0000E946A6686E69FE0DF91CF911F910F91A5
:10FEE000FF90EF90DF90CF900C948E3FD730B1F51C
:10FEF00080916F02882391F0769567955795479585
:10FF00002EE7473051056105710511F44EE301C03C
:10FF100040E267E57FE08C2F0E9443651123F1F0FA
:10FF20008091590D90915A0DA0915B0DB0915C0D8F
:10FF3000B695A795979587950797A105B10571F493
:10FF40000E946A668CE693E8DF91CF911F910F9132
:10FF5000FF90EF90DF90CF900C94A7662091BD0D9D
:10FF60008091590D90915A0DA0915B0DB0915C0D4F
:10FF7000211136C0D83009F048C020916F022223E9
:10FF800089F0B695A7959795879520E20897A105E2
:10FF9000B10511F44EE301C040E265E47FE08C2F2F
:10FFA0000E944365112389F18091590D90915A0D5A
:10FFB000A0915B0DB0915C0DB695A795979587952F
:10FFC0000897A105B10509F50E946A66DF91CF91F6
:10FFD0001F910F91FF90EF90DF90CF900C942371C1
:10FFE000D83099F420916F022223E1F2B695A795BB
:10FFF0009795879520E20897A105B10511F44EE386
:020000021000EC
:1000000001C040E263E37FE0CACF8091590D909137
:100010005A0DA0915B0DB0915C0D4297A105B10501
:1000200040F0C092590DD0925A0DE0925B0DF092C3
:100030005C0D4091590D50915A0D60915B0D70917E
:100040005C0D76956795579547958091620D90E088
:100050000396242F30E0821793074CF48DEF840F22
:100060008093620D00936F02DCEFD40FCFEFCF5F70
:10007000DF5FC43008F490CDDF91CF911F910F91D5
:10008000FF90EF90DF90CF900895FC0180819181E7
:100090008436910524F164E670E00E9484B6CB01B9
:1000A0002AE030E0B9010E9484B6805D80932D0D76
:1000B00080819181B9010E9484B6CB01B9010E946F
:1000C00084B6805D80932E0D80819181B9010E945C
:1000D00084B6805D80932F0D1092300D23C08A303E
:1000E0009105BCF02AE030E0B9010E9484B6CB0152
:1000F000B9010E9484B6805D80932D0D808191812D
:10010000B9010E9484B6805D80932E0D10922F0D50
:1001100009C06AE070E00E9484B6805D80932D0D76
:1001200010922E0D8DE29DE008958F929F92AF92D6
:10013000BF92CF92DF92EF92FF92CF9320E030E018
:1001400040E251E4FC0160817181828193810E94CF
:100150008EB50E9428B397FD02C02BE201C02DE2AC
:1001600020932D0D6B017C0197FF08C0F094E09463
:10017000D094C094C11CD11CE11CF11CC701B60174
:1001800020E137E240E050E00E94B9B69AE0892EC3
:10019000912CA12CB12CCA01B901A50194010E9496
:1001A000B9B6605D60932E0DC701B60128EE33E04D
:1001B00040E050E00E94B9B6CA01B901A50194011E
:1001C0000E94B9B6605D60932F0DC701B60124E6A9
:1001D00030E040E050E00E94B9B6CA01B901A50183
:1001E00094010E94B9B6605D6093300DC701B601FD
:1001F000A50194010E94B9B6C62FCA01B901A50193
:1002000094010E94B9B6605D6093310D8EE28093D7
:10021000320DC05DC093330D1092340D8DE29DE020
:10022000CF91FF90EF90DF90CF90BF90AF909F90D5
:100230008F900895CF92EF920F937FE1C72EE0E267
:10024000EE2E0FE02EE045E066E284E69DE00E949F
:10025000172A0F91EF90CF900895CF93DF93FC0171
:100260006491EC012196662331F084E69DE00E94C2
:10027000042BCE01F4CFDF91CF9108950F931F93FC
:10028000CF93DF938C01EB0141E061E084E69DE0D8
:100290000E942C29C801E1DF6AE384E69DE00E9408
:1002A000D8B1FE0101900020E9F76C2F6E1B6C5E47
:1002B00041E084E69DE00E942C29BE0184E69DE099
:1002C000DF91CF911F910F910C94D7B1CF92DF9214
:1002D000EF92FF920F931F938091590D90915A0DB9
:1002E000A0915B0DB0915C0D0097A105B10509F4DB
:1002F00042C0BC01882777FD8095982F0E945BB390
:100300002091350D3091360D4091370D5091380DBB
:100310000E948EB59B01AC0160916E0A70916F0ACC
:100320008091700A9091710A0E94E0B160936E0A08
:1003300070936F0A8093700A9093710A1092590D0E
:1003400010925A0D10925B0D10925C0DFEE4CF2EB0
:10035000FAE0DF2EE12CF12C00E81FE32EE63AE074
:100360004AE65AE066E67AE082E69AE00E94909ECB
:1003700081E080936F0280916F02882339F08EE6CE
:100380009AE0B4D8BC0186EC90E178DF8091630DEF
:1003900082FF0EC021E040E050E0BA018EE398E613
:1003A0001F910F91FF90EF90DF90CF900C948C668F
:1003B0001F910F91FF90EF90DF90CF900895CF9312
:1003C000DF931F921F92CDB7DEB78091590D9091A8
:1003D0005A0DA0915B0DB0915C0DB7FF08C0109253
:1003E000590D10925A0D10925B0D10925C0D809178
:1003F000410D9091420DA091430DB091440D40915B
:10040000590D50915A0D60915B0D70915C0D8417E0
:100410009507A607B70744F48093590D90935A0D9A
:10042000A0935B0DB0935C0D80916F028823A9F0BF
:100430008091450D9091460D2091590D30915A0DA6
:10044000820F931F9A838983CE0101966DD9BC01D7
:1004500080914B0D90914C0D11DF8091630D82FFC7
:100460001DC0E091490DF0914A0D8091450D90918C
:10047000460D2091590D30915A0D820F931F918393
:10048000808340914D0D50914E0D60E070E021E071
:1004900080914F0D9091500D0E948C660F900F909F
:1004A000DF91CF9108954F925F926F927F928F92DA
:1004B0009F92AF92BF92CF92DF92EF92FF920F93F3
:1004C0001F93CF93DF934C015B017A018091590D0B
:1004D00090915A0DA0915B0DB0915C0D892B8A2BE8
:1004E0008B2B09F47BC00E94BA41E501CC0FDD1FC4
:1004F000CC0FDD1F8E010E59154F6091590D709173
:100500005A0D882777FD8095982F0E945BB3209124
:10051000350D3091360D4091370D5091380D0E94B8
:100520008EB5F80120813181428153810E94E0B172
:100530002B013C0120E030E0A9010E94B9B2F80192
:1005400087FD05C0408251826282738204C010829E
:10055000118212821382B701882777FD8095982F28
:100560000E945BB36B017C018E010E59154F9B01FC
:10057000AC01F80160817181828193810E94BCB4D9
:1005800018162CF4F801C082D182E282F382109214
:10059000590D10925A0D10925B0D10925C0DCC53B8
:1005A000DA4F20E030E040E752E4688179818A81C7
:1005B0009B810E94C0B2CEE4CC2ECAE0DC2E7B012F
:1005C0008C012EE63AE04AE65AE066E67AE082E6F8
:1005D0009AE00E94909E81E080936F0280916F026A
:1005E000882361F0C501880F991F880F991F8E59C4
:1005F000954F0E94767ABC01C40140DE8091630D64
:1006000082FF18C021E040E050E0BA018EE398E696
:10061000DF91CF911F910F91FF90EF90DF90CF90DE
:10062000BF90AF909F908F907F906F905F904F9012
:100630000C948C66DF91CF911F910F91FF90EF90FA
:10064000DF90CF90BF90AF909F908F907F906F90F2
:100650005F904F90089546ED50E060E070E080ECD0
:1006600090E121CF46EC50E061E070E082EC90E157
:100670001ACF49EC50E062E070E084EC90E113CFD7
:100680000F931F93CF93DF938C01EB0141E060E068
:1006900084E69DE00E942C29C801DFDD6AE384E640
:1006A0009DE00E94D8B1FE0101900020E9F7BE0153
:1006B0006E1B7F0B6B5E7F4F7695679543E084E6FC
:1006C0009DE00E942C29BE0184E69DE0DF91CF9140
:1006D0001F910F910C94D7B1CF93DF9300D01F924D
:1006E000CDB7DEB78091590D90915A0DA0915B0D59
:1006F000B0915C0D0097A105B105F9F02091550866
:1007000030915608280F391F30935608209355080A
:100710002091C40D3091C50D280F391F3093C50DA0
:100720002093C40D1092590D10925A0D10925B0D2A
:1007300010925C0D81E080936F0280916F0288239C
:10074000A9F06091C40D7091C50D882777FD809543
:10075000982F0E945BB369837A838B839C83CE013D
:100760000196E3DCBC0185E29FE08ADF8091630DA6
:1007700082FF08C021E040E050E0BA0180E79DE739
:100780000E948C6660EC7DE08DEF9FE00E94C2705D
:1007900062EC7DE08BEF9FE00E94C27064EC7DE034
:1007A00089EF9FE00E94C2700F900F900F900F9002
:1007B000DF91CF9108958F929F92AF92BF92CF9287
:1007C000DF92EF92FF920F931F93CF93DF93CDB7FA
:1007D000DEB728970FB6F894DEBF0FBECDBF80916D
:1007E000530D882321F081508093530D03C081E085
:1007F00080936F0280916F02882309F459C280911F
:10080000BF0D8F5F8093BF0D8E3129F40E94D76991
:100810001092BF0D0EC06AE00E9463B6911109C02C
:1008200020E044E064E184E69DE00E943C2A0E94CE
:10083000CD6520E030E040E05FE360915E087091BC
:100840005F0880916008909161080E94E0B10E9469
:1008500028B378876F83609166087091670888274E
:1008600077FD8095982F0E945BB320E030E040E058
:100870005FE30E94E0B10E9428B37E836D8340E075
:1008800060E084E69DE00E942C2962E084E69DE021
:100890000E94D8B1CE0107960E94947BBC0184E6E9
:1008A0009DE00E94D7B16FE284E69DE00E94D8B13E
:1008B000CE010596EADBBC0184E69DE00E94D7B13B
:1008C00082E29FE0CADC6CE973E084E69DE00E946E
:1008D000D7B140E06AE084E69DE00E942C2960ECFC
:1008E00075E084E69DE00E94D7B12CEA35EC47E242
:1008F00057E360916A0A70916B0A80916C0A90913B
:100900006D0A0E94E0B169837A838B839C83CE0158
:1009100001960E94C27ABC0184E69DE00E94D7B194
:1009200060E284E69DE00E94D8B141E060E084E6A8
:100930009DE00E942C2920E030E040E05FE36091E0
:1009400058087091590880915A0890915B080E944C
:10095000E0B10E9428B378876F836091640870913A
:100960006508882777FD8095982F0E945BB320E06B
:1009700030E040E05FE30E94E0B10E9428B37E8354
:100980006D8360E084E69DE00E94D8B1CE010796B9
:100990000E94947BBC0184E69DE00E94D7B16FE287
:1009A00084E69DE00E94D8B1CE0105966EDBBC01C5
:1009B00084E69DE00E94D7B18FE19FE04EDC6CE9B8
:1009C00073E084E69DE00E94D7B141E06AE084E6EE
:1009D0009DE00E942C296CE973E084E69DE00E9472
:1009E000D7B166E084E69DE00E94D8B18DE592E043
:1009F0000E94947BBC0184E69DE00E94D7B165E231
:100A000084E69DE00E94D8B169E973E084E69DE048
:100A10000E94D7B142E060E084E69DE00E942C296C
:100A20008CE19FE01ADC8091830A8823A9F18091F0
:100A30006C0C882319F18091160D9091170DA091DF
:100A4000180DB091190D0097A105B105B9F0BC01C1
:100A5000CD016D597F4F8F4F9F4F24E630E040E02E
:100A600050E00E9497B660911E0D70911F0D80910D
:100A7000200D9091210D0E9497B601C020E030E03A
:100A80003A832983CE0101960E94947BBC0184E6BF
:100A90009DE00E94D7B103C088E19FE0DEDB65E204
:100AA00084E69DE00E94D8B168E973E084E69DE0A9
:100AB0000E94D7B142E06AE084E69DE00E942C29C2
:100AC0006CE973E084E69DE00E94D7B167E084E6BC
:100AD0009DE00E94D8B18091700890917108A0911A
:100AE0007208B0917308892B8A2B8B2BE1F10E943D
:100AF0004AAD20E6C22E2AEED22EE12CF12CA7011F
:100B000096010E9497B649015A0160917008709150
:100B100071088091720890917308A70196010E9454
:100B200097B6C401821B930B6CE370E00E9470B611
:100B3000182F6983CE0101960E945E7ABC0184E67B
:100B40009DE00E94D7B16AE384E69DE00E94D8B19F
:100B50001983CE0101960E945E7ABC0184E69DE075
:100B60000E94D7B103C082E19FE077DB6CE973E0BC
:100B700084E69DE00E94D7B143E060E084E69DE01A
:100B80000E942C296AE873E082E792E00E9447BA4B
:100B9000892B09F074C062E97AE089E79DE00E9440
:100BA00047BA892BD1F0E9E7FDE0DF010D90002085
:100BB000E9F7AD014150510949575D4060E070E0EF
:100BC000CF010E9417BA62E97AE089E79DE00E94AE
:100BD00050BA1092AF0D1092AE0DE2E9FAE001901A
:100BE0000020E9F7E359FA40759708F445C00091F1
:100BF000AE0D1091AF0DC12CD12C8091AE0D909106
:100C0000AF0D9801281B390B2431310534F00196C2
:100C10009093AF0D8093AE0D38C0C114D104B9F7D5
:100C2000F801EF57F54F7F019189602F681B43E072
:100C3000911115C084E69DE00E942C29D7015096A1
:100C40006C9184E69DE00E94D8B11092AF0D109295
:100C5000AE0D00E010E0CC24C394D12CCECF84E6BE
:100C60009DE00E942C29F701608984E69DE00E94A6
:100C7000D8B10F5F1F4FC1CF69E77DE002C062E7C7
:100C800072E084E69DE00E94D7B102E712E0D8014D
:100C90008D918D0180322CF460E284E69DE00E940B
:100CA000D8B1B2E006381B0791F78AE08093530D64
:100CB0008091630D82FB882780F99091520D9923D2
:100CC00099F09091510D992339F0811119C010922A
:100CD000510D1092520D14C0882391F00E946A6643
:100CE00081E08093510D0CC0882351F021E040E059
:100CF00050E0BA018EEB93E70E948C660E94D769A0
:100D000080915D0290915E022091590D30915A0DB3
:100D10008436910534F4820F931F853691054CF487
:100D200016C08436910599F0820F931F8436910581
:100D300074F41092590D10925A0D10925B0D10928E
:100D40005C0D84E690E090935E0280935D022091BA
:100D50005D0230915E028091590D90915A0D2436BA
:100D6000310569F48B3091051CF0865A9F4F09C0FC
:100D7000863FEFEF9E078CF482599F4F02C0820F8F
:100D8000931F90935E0280935D021092590D109212
:100D90005A0D10925B0D10925C0D80915D02909146
:100DA0005E028A3091051CF48AE090E005C0883E1E
:100DB000934034F087EE93E090935E0280935D025F
:100DC00028960FB6F894DEBF0FBECDBFDF91CF914E
:100DD0001F910F91FF90EF90DF90CF90BF90AF9059
:100DE0009F908F900895CF93DF93CCEBDEE0FE01D0
:100DF0008491882341F09091C00095FFFCCF8093AF
:100E0000C6003196F5CFEFE5F5E18491882341F0F6
:100E10009091C00095FFFCCF8093C6003196F5CF2E
:100E20008091C00085FFFCCF8AE08093C600FE0160
:100E30008491ECEBFEE0882349F09091C00095FF8F
:100E4000FCCF8093C60031968491F5CF4091CD13AD
:100E50005091CE136091CF137091D01387E595E137
:100E60000E94F73E4091D1135091D2136091D31359
:100E70007091D41384E595E10E94F73E4091D5131B
:100E80005091D6136091D7137091D81381E595E1F5
:100E90000E94F73E4091D9135091DA136091DB1311
:100EA0007091DC138EE495E10E94F73E8091C000C2
:100EB00085FFFCCF8AE08093C600FE018491ECEBB5
:100EC000FEE0882349F09091C00095FFFCCF80930D
:100ED000C60031968491F5CFE4E3F5E1849188234F
:100EE00041F09091C00095FFFCCF8093C6003196F1
:100EF000F5CF8091C00085FFFCCF8AE08093C600CB
:100F0000FE018491ECEBFEE0882349F09091C00053
:100F100095FFFCCF8093C60031968491F5CF409128
:100F2000DD135091DE136091DF137091E0138BE2BB
:100F300095E10E94F73E4091E1135091E2136091D8
:100F4000E3137091E41388E295E10E94F73E40912B
:100F5000E5135091E6136091E7137091E81385E271
:100F600095E10E94F73E4091E9135091EA13609198
:100F7000EB137091EC1382E295E10E94F73E8091B1
:100F8000C00085FFFCCF8AE08093C600FE018491FB
:100F9000ECEBFEE0882349F09091C00095FFFCCF78
:100FA0008093C60031968491F5CFE4E0F5E1849119
:100FB000882341F09091C00095FFFCCF8093C6003C
:100FC0003196F5CF8091C00085FFFCCF8AE08093F9
:100FD000C600FE018491ECEBFEE0882349F090917D
:100FE000C00095FFFCCF8093C60031968491F5CF69
:100FF0004091BD135091BE136091BF137091C01307
:101000008BEF94E10E94093F4091C1135091C213AC
:101010006091C3137091C41388EF94E10E94093F5B
:101020004091C5135091C6136091C7137091C813B6
:1010300085EF94E10E94093F4091C9135091CA1372
:101040006091CB137091CC1382EF94E10E94093F21
:101050008091C00085FFFCCF8AE08093C600FE012E
:101060008491ECEBFEE0882349F09091C00095FF5D
:10107000FCCF8093C60031968491F5CFEDEBF4E17F
:101080008491882341F09091C00095FFFCCF80931C
:10109000C6003196F5CF8091C00085FFFCCF8AE075
:1010A0008093C600FE018491ECEBFEE0882349F0BA
:1010B0009091C00095FFFCCF8093C600319684913B
:1010C000F5CF4091B5135091B6136091B71370915D
:1010D000B81384EB94E10E94F73E4091B113509114
:1010E000B2136091B3137091B41381EB94E10E9439
:1010F000F73E8091C00085FFFCCF8AE08093C60058
:10110000FE018491ECEBFEE0882349F09091C00051
:1011100095FFFCCF8093C60031968491F5CFEEEF1A
:10112000F3E18491882341F09091C00095FFFCCFBA
:101130008093C6003196F5CF8091C00085FFFCCF2B
:101140008AE08093C600FE018491ECEBFEE08823E8
:1011500049F09091C00095FFFCCF8093C600319676
:101160008491F5CF4091B9135091BA136091BB139C
:101170007091BC1385EF93E10E94F73E4091A1135B
:101180005091A2136091A3137091A41382EF93E185
:101190000E94F73E4091ED135091EE136091EF13D2
:1011A0007091F0138FEE93E10E94093F4091AD13CF
:1011B0005091AE136091AF137091B0138CEE93E128
:1011C0000E94F73E4091A9135091AA136091AB136E
:1011D0007091AC1389EE93E10E94F73E4091A51304
:1011E0005091A6136091A7137091A81386EE93E116
:1011F0000E94F73E8091C00085FFFCCF8AE080937B
:10120000C600FE018491ECEBFEE0882349F090914A
:10121000C00095FFFCCF8093C60031968491F5CF36
:10122000E4EDF3E18491882341F09091C00095FFB3
:10123000FCCF8093C6003196F5CF8091C00085FF2A
:10124000FCCF8AE08093C600FE018491ECEBFEE0C7
:10125000882349F09091C00095FFFCCF8093C60091
:1012600031968491F5CF4091560A5091570A60917A
:10127000580A7091590A8BEC93E10E94F73E409115
:101280005A0A50915B0A60915C0A70915D0A88EC81
:1012900093E10E94F73E40915E0A50915F0A60918F
:1012A000600A7091610A85EC93E10E94F73E80919B
:1012B000C00085FFFCCF8AE08093C600FE018491C8
:1012C000ECEBFEE0882349F09091C00095FFFCCF45
:1012D0008093C60031968491F5CFE7EBF3E18491DA
:1012E000882341F09091C00095FFFCCF8093C60009
:1012F0003196F5CF8091C00085FFFCCF8AE08093C6
:10130000C600FE018491ECEBFEE0882349F0909149
:10131000C00095FFFCCF8093C60031968491F5CF35
:10132000409118025091190260911A0270911B02AB
:101330008DEA93E10E94F73E6091140270911502CC
:1013400080911602909117020E946B28AB01BC019C
:101350008AEA93E10E94F73E6091100270911102B7
:1013600080911202909113020E947728AB01BC0178
:1013700087EA93E10E94F73E8091C00085FFFCCF91
:101380008AE08093C600FE018491ECEBFEE08823A6
:1013900049F09091C00095FFFCCF8093C600319634
:1013A0008491F5CFE3E7F3E18491882341F09091B4
:1013B000C00095FFFCCF8093C6003196F5CF809199
:1013C000C00085FFFCCF8AE08093C600FE018491B7
:1013D000ECEBFEE0882349F09091C00095FFFCCF34
:1013E0008093C60031968491F5CF4091330250919D
:1013F0003402609135027091360289E693E10E94D1
:10140000F73E20E030E040E752E460912B0270911B
:101410002C0280912D0290912E020E948EB5AB017C
:10142000BC0186E693E10E94F73E4091460A509146
:10143000470A6091480A7091490A83E693E10E9445
:10144000F73E8091C00085FFFCCF8AE08093C60004
:10145000FE018491ECEBFEE0882349F09091C000FE
:1014600095FFFCCF8093C60031968491F5CFE7E3DA
:10147000F3E18491882341F09091C00095FFFCCF67
:101480008093C6003196F5CF8091C00085FFFCCFD8
:101490008AE08093C600FE018491ECEBFEE0882395
:1014A00049F09091C00095FFFCCF8093C600319623
:1014B0008491F5CF4091420A5091430A6091440AC9
:1014C0007091450A8DE293E10E94F73E20E030E002
:1014D00040E752E46091270270912802809129022E
:1014E00090912A020E948EB5AB01BC018AE293E181
:1014F0000E94F73E8091C00085FFFCCF8AE0809378
:10150000C600FE018491ECEBFEE0882349F0909147
:10151000C00095FFFCCF8093C60031968491F5CF33
:10152000E0EDF2E18491882341F09091C00095FFB5
:10153000FCCF8093C6003196F5CF8091C00085FF27
:10154000FCCF8AE08093C600FE018491ECEBFEE0C4
:10155000882349F09091C00095FFFCCF8093C6008E
:1015600031968491F5CF40914B0A50E060E070E0F5
:1015700086EC92E10E94093F8091C00085FFFCCF7C
:101580008AE08093C600FE018491ECEBFEE08823A4
:1015900049F09091C00095FFFCCF8093C600319632
:1015A0008491F5CF8091720A8823A1F1E3EBF2E1F7
:1015B0008491882341F09091C00095FFFCCF8093E7
:1015C000C6003196F5CF8091C00085FFFCCF8AE040
:1015D0008093C600FE01C491ECEBFEE0CC2349F001
:1015E0008091C00085FFFCCFC093C6003196C491A6
:1015F000F5CF409153025091540260915502709181
:10160000560289EA92E10E94F73E8091C00085FF70
:10161000FCCF11C0EDE8F2E18491882341F0909174
:10162000C00095FFFCCF8093C6003196F5CF809126
:10163000C00085FFFCCF8AE08093C600DF91CF9188
:101640000895AF92BF92CF92DF92EF92FF920F93E5
:101650001F93CF93DF93CDB7DEB7E0970FB6F89423
:10166000DEBF0FBECDBF80E1EBEFF2E0DE01919671
:1016700001900D928A95E1F780E1EBE0F3E0DE0165
:10168000519601900D928A95E1F780E1EBE1F3E04C
:10169000DE01119601900D928A95E1F76E0181E2CB
:1016A000C80ED11C8DECE82E83E1F82E8E010F5E62
:1016B0001F4F6DED73E1AE014F5F5F4F9DEBA92EA4
:1016C00093E1B92E20E030E0F60181919191A19152
:1016D000B1916F01F70181939193A193B1937F0130
:1016E000F80181919191A191B1918F01FB018193B9
:1016F0009193A193B193BF01FA0181919191A1912D
:10170000B191AF01F50181939193A193B1935F01E1
:101710002F5F3F4F24303105B9F60E9429A980E0A0
:1017200090E8ABE3B5E48093B5139093B613A09320
:10173000B713B093B8138093B1139093B213A093DF
:10174000B313B093B4131092B9131092BA1310924A
:10175000BB131092BC1380E29EE4A0E0B0E0809343
:10176000ED139093EE13A093EF13B093F013109238
:10177000A1131092A2131092A3131092A41380E04D
:1017800090E0A0EAB1E48093AD139093AE13A093E0
:10179000AF13B093B0138DEC9CECACECBEE3809334
:1017A000A9139093AA13A093AB13B093AC1380E04A
:1017B00090E0A0EAB0E48093A5139093A613A093C1
:1017C000A713B093A81310925E0A10925F0A1092AA
:1017D000600A1092610A10925A0A10925B0A1092E3
:1017E0005C0A10925D0A1092560A1092570A1092E3
:1017F000580A1092590A82ED90E09093BC0D8093A4
:10180000BB0D82E390E09093BA0D8093B90D1092D6
:10181000B80D1092B70D8FEF90E09093B60D8093B6
:10182000B50D84E690E09093B40D8093B30D1092C3
:10183000B20D1092B10D83E393EBA3E2B2E4809377
:10184000180290931902A0931A02B0931B0260E051
:1018500070E08CE990E40E94652860931402709314
:101860001502809316029093170265E87BE28CEADA
:1018700092E40E9471286093100270931102809389
:101880001202909313020E94D31E80E090E0A0E821
:10189000BFE380930C0290930D02A0930E02B093CD
:1018A0000F0210924B0A80E090E0A0E4B0E4809335
:1018B000330290933402A0933502B093360240E095
:1018C00050E064E372E440932B0250932C02609347
:1018D0002D0270932E021092460A1092470A10921F
:1018E000480A1092490A1092420A1092430A109232
:1018F000440A1092450A40E050E060E071E44093F1
:101900002702509328026093290270932A021092B2
:10191000720A8093530290935402A0935502B0939D
:1019200056020E94024CECEBFEE08491882341F0C9
:101930009091C00095FFFCCF8093C6003196F5CF03
:10194000EBE6F2E18491882341F09091C00095FF8D
:10195000FCCF8093C6003196F5CF8091C00085FF03
:10196000FCCF8AE08093C600E0960FB6F894DEBF05
:101970000FBECDBFDF91CF911F910F91FF90EF90E0
:10198000DF90CF90BF90AF9008951F920F920FB647
:101990000F9211240BB60F922F933F934F935F93A7
:1019A0006F938F939F93EF93FF936091C600209165
:1019B000480E3091490EC90101968F7799274091C1
:1019C0004A0E50914B0E8417950741F0F901E853E8
:1019D000F24F60839093490E8093480EFF91EF91F0
:1019E0009F918F916F915F914F913F912F910F90A8
:1019F0000BBE0F900FBE0F901F9018959A01AB0170
:101A0000211581EE38074105510549F182E08093A7
:101A1000C00060E079E08DE390E00E94B9B621500B
:101A2000310941095109CA01B90122E030E040E021
:101A300050E00E94B9B63093C5002093C400809155
:101A4000C10080618093C1008091C1008860809353
:101A5000C1008091C10080688093C10008951092F8
:101A6000C00020E130E0E7CF20914A0E30914B0ECC
:101A70008091480E9091490E8217930771F0F901F9
:101A8000E853F24F80812F5F3F4F2F7733273093FA
:101A90004B0E20934A0E90E008958FEF9FEF08952C
:101AA00080914A0E90914B0E9093490E8093480E70
:101AB00008954F925F926F927F928F929F92AF9212
:101AC000BF92CF92DF92EF92FF920F931F93CF932B
:101AD000DF93CDB7DEB7A0970FB6F894DEBF0FBE89
:101AE000CDBF5C014115510561057105E9F420E0A8
:101AF00030E040E350E060E070E0A0960FB6F8946C
:101B0000DEBF0FBECDBFDF91CF911F910F91FF9030
:101B1000EF90DF90CF90BF90AF909F908F907F908D
:101B20006F905F904F905BC08E010F5F1F4FC12C75
:101B3000D12C76014801422E512C612C712C8FEF53
:101B4000C81AD80AE80AF80ACB01BA01A30192011F
:101B50000E9497B6CA01F80161938F01A901BC01E7
:101B6000411551056105710551F7F1E0CF1AD10812
:101B7000E108F108F401EC0DFD1D80818A3010F4BC
:101B800040E301C047E3480F552747FD5095652FB7
:101B9000752F20E030E0C50122D081E0C81AD108BD
:101BA000E108F108EFEFCE16DE06EE06FE0611F7AD
:101BB000A0960FB6F894DEBF0FBECDBFDF91CF91D8
:101BC0001F910F91FF90EF90DF90CF90BF90AF905B
:101BD0009F908F907F906F905F904F900895211508
:101BE000310539F48091C00085FFFCCF4093C600D9
:101BF00008952A30310509F424C05BCF9A01462F9D
:101C0000552747FD5095652F752FE9CFCF93DF936B
